:020000040800F2
:1000000000500020559A0008F19A0008398600082F
:10001000F19A0008F19A0008F19A00080000000027
:10002000000000000000000000000000F19A00083D
:10003000F19A000800000000F19A0008557D0008C0
:10004000F19A0008F19A0008F19A0008F19A000864
:10005000F19A0008F19A0008F19A0008F19A000854
:10006000F19A0008657D0008F19A0008F19A0008ED
:10007000F19A0008F19A000865760008F19A0008E4
:10008000F19A0008F19A0008F19A0008F19A000824
:10009000F19A0008F19A0008F19A0008F19A000814
:1000A000F19A0008C1740008F19A0008B1740008C0
:1000B000A574000895740008857400088123000861
:1000C000872300087D23000885230008F19A000893
:1000D000F19A0008597600084D760008F19A000858
:1000E000697D0008F19A0008F19A000800000000FC
:1000F0000000000000000000000000000000000000
:0C01000000000000000000005FF808F1A3
:100110002DE9F04FA3B008F019F818B906F0F4FE75
:1001200008F03AF808F0DCF8B14BB24D1A78B24E4C
:1001300042F001021A70002209920A920B924FF4C7
:10014000E0120C922A68B17B42F480322A60AA69DC
:1001500042F01002AA6106932B6803F400330A935D
:10016000099B013309930A9B1BB9099BB3F5A06F47
:10017000F2D12B6813F4003300F0748302230B9345
:100180009E4B9F481A689F4F42F010021A601A68EF
:1001900022F003021A601A6842F002021A606B68C9
:1001A0006B606B686B606B6843F480636B60964B4D
:1001B0001A6822F070421A60944A1060686820F44D
:1001C0007C106860186840F000401860FB6823F4F9
:1001D0000043FB604FF4E0130C930B9B012B00F0EA
:1001E0006183022B0ED139B10C9BB3F5801F40F017
:1001F00051834FF4A0130C930C9B69680B4343F499
:1002000080336B602B6843F080732B602B689C01FC
:10021000FCD56B6823F003036B606B6843F002034B
:100220006B606B6803F00C03082BFAD16B68784C99
:1002300003F00C03042B00F03983082B00F0388303
:100240006F4B23606B68734AC3F30313D25C23685C
:100250004FF0000AD34023606F4A0B9BDFF8DC911C
:100260001360BB686D4A6E4B0DF18808DA60AA69AD
:10027000039342F00102AA616A6A674B48465A60DA
:100280006A6A0DF1880B42F080726A62AA6942F0D4
:100290001C02AA614FF6FF7228F8402D41468DF8E6
:1002A0004AA001F0B9FB41465E4801F0B5FB41466A
:1002B000544801F0B1FB02228DF837204FF4007250
:1002C0004FF010032BF8542D8DF836305946C9F8ED
:1002D0001020484601F0A0FB534940464A6842F0CE
:1002E00000724A6004F04CF9129A5049039BB2FB29
:1002F000F1F24F49DFF848E10A604FF47A714D4A54
:10030000C2F800A0C2F804A022684446B2FBF1F291
:100310004949013A4A60F02283F823200723C1F8B3
:1003200008A00B60B368CEF800303A4B03F1100C14
:10033000BCE80F000FC4BCE80F000FC4BCE80F00FE
:100340000FC49CE80F0084E80F00AB69402243F023
:100350001003AB61AB69304C43F01003AB61AB6988
:1003600043F01003AB61AB6943F00803AB61AB69C9
:1003700043F00803AB61AB6943F00403AB611023A6
:10038000C9F814302023C9F81430C9F814204FF4E8
:1003900080423A614FF400523A614FF400423A61B0
:1003A000204A5361134610225A615346F246ACF17B
:1003B00040020492CDF80C90191D58F803004144F6
:1003C000059301F029FB059B0833402BF4D1DAF8A3
:1003D00000301B0736D596F81E31012B32D86268E3
:1003E00096F81F3112F08052059201F02F8029E01B
:1003F000681800200010024064080020002002401D
:1004000000127A0000100140041001403400002066
:1004100014000020E0D50008800400200005FA0543
:1004200000ED00E0000C01400000014040420F00E0
:1004300050180020FC17002010E000E000080140E8
:1004400000160020642007F022FCA0220021BA48F8
:100450000DF091F8EB69B94A43F00703EB61AB6922
:10046000DFF8188343F4006343F00C03AB61B44B33
:1004700000211A600222B34B40461A701822DAF8A3
:1004800000700DF078F8012388F80C3096F805809C
:100490001422002158460DF06EF8B8F10E0FC7F384
:1004A000801904D008F0EF08B8F1080F02D1012339
:1004B0008DF83E3096F97831012B00F0EA8796F9F5
:1004C0008031012B00F0EC8700238DF83930C7F321
:1004D00040038DF83A30C7F340338DF83430C7F31A
:1004E000C0338DF8373017F400638DF83C9007D097
:1004F00096F81231A3F1020EDEF1000343EB0E0376
:100500008DF83830C7F300438DF83D3007F0010314
:10051000B6F8D4208DF83530C7F3C0038DF83630E7
:10052000C7F38043FF04ADF842208DF83B3048BF4D
:10053000B6F8DC20B6F8E03048BFADF84220B3F59D
:10054000FA7FADF8403084BF0023ADF8423096F812
:1005500062310D9A23720023A4F809309DF83E30D1
:1005600022F07F42002B22F0FF0214BF022300235F
:1005700002B101334FF0000A049A02EB83031B6DB2
:100580009A1E1A3305920793059A32F8023F059294
:100590004FF6FF72934223D0DAB26B4916018F19DE
:1005A0009DF839101B0A11B1023A012A14D99DF89D
:1005B0003A204AB1049A03983244516E814203D1E1
:1005C000B2F86820082A07D0022B40F0A3819DF8DA
:1005D0003430002B40F0E681079B059A9342D3D13B
:1005E00006220026594BDFF898C1DFF898E11A700F
:1005F00006EB0C0706EB0E031036602E0FCB87E8D8
:100600000F00F5D1524B53491F68534B0A681E68BF
:100610000023524802F4805E0491BEF1000F00F006
:100620003882B6F9041020F8131001330C2BF4D1E2
:1006300050035CBF01224A4B4FF0000058BF1A70B4
:10064000069B069A1B7843F00403137001F0F6FB37
:10065000049B10221E68002106F0020641480CF09F
:100660008AFFDEB1039B01201A680F26002300FADF
:1006700003F131F0080104BF990006FA01F103F11A
:10068000010308BF8A43082BF1D1039B01261A609E
:100690000322344B1A7007229E70DA706B68324F57
:1006A00043F440436B606B69384643F001036B6170
:1006B000AB694FF0070943F40073AB6103F0D9FF56
:1006C0002A4B002512932A4B12A913934FF48073DF
:1006D00018934FF48063199320231A934FF4005317
:1006E000384615961B93149516951C95179503F08F
:1006F000A2FF3B681F4A43F001033B605368013E81
:1007000023F4702323F48073536091681A4BF6B27C
:100710000B4043F4602343F002039360D36A2946FD
:1007200023F4700343EA06564FF01F0E0123DFF84F
:100730003480D66228E000BFA8130020DA09002028
:100740005C160020FC07002040D600085313002050
:100750004C140020001600204814002040160020F1
:100760007C040020000E0020080002404C240140C0
:10077000100E002000240140FDF7F1FF00080020CA
:10078000B803002020D7000801EB0805A87828B39B
:1007900011F808005F1C0928FFB2EE7840F27C8156
:1007A000A0F10A05D2F80CA005EB450509FA05FCF5
:1007B0002AEA0C0C06FA05F545EA0C05D560062B6D
:1007C00000F27781013B556B03EB83030EFA03F6CE
:1007D00025EA06059840284350633B46043110291A
:1007E000D2D1C14B9A6842F480729A609A6842F002
:1007F00001029A609A6842F008029A609A681107AA
:10080000FCD49A6842F004029A60B74B9A68520787
:10081000FCD49A6842F4A0029A60B44BB3F9E800A1
:100820009B46002800F082810022B14B1A7008F02C
:1008300081FCB04908F0D2FC1290BBF9EA0008F044
:1008400079FCAC4908F0CAFC1390BBF9EC0008F045
:1008500071FCA84908F0C2FCA749149012A807F03F
:1008600053FB6DE12A6842F001022A6009932B686C
:1008700003F002030A93099B013309930A9B1BB9F6
:10088000099BB3F5A06FF2D12B689F0701D5012317
:1008900075E4FEE70C9BB3F5E01F7FF4ADAC4FF4BD
:1008A0000013A8E46B6843F46013AAE41368C8E477
:1008B0006B686968C3F38343C80303F1020302D47E
:1008C0008E4A5343BDE469681268890348BF5208E1
:1008D000F7E7039B05927820C7F81080C3F81490BF
:1008E00007F0CAF9039BC7F814807820C3F810906A
:1008F00007F0C2F9059A013296F81F319A42E8DBF7
:10090000636813F080537FF49DAD86F81F3107F0C4
:1009100063FE97E5012B42D19DF83530002B3FF463
:100920005BAEFF2384F8503084F85130049B4FF0C5
:1009300000081E4496F86D30B6F868208DF84A30ED
:10094000022312A9706E84F8548027668DF84B300C
:10095000ADF8482084F80C80C4F81080C4F81480E6
:10096000C4F81880C4F84C8084F8528084F853800E
:1009700001F052F8424696F86A10306E04F0FCFB23
:10098000384603F07DFB5E4B5E4A63665E4BC4F8FF
:100990006C80A366111F384606F004FE1CE6022B8D
:1009A000DAB243D14FF01C0901235FFA8AF109FB47
:1009B00001F904EB090888F85430049B4FF0000B50
:1009C0001E4496F86D30B6F868208DF84A30022340
:1009D00088F855A012A9706E88F856B088F85EB0F5
:1009E000C8F860708DF84B30ADF8482001F014F86D
:1009F0005A4696F86A10306E04F0BEFB384603F093
:100A00003FFB424B4249C8F86430424B09F11402A3
:100A100009F110090A44C8F86830C8F86CB04944B4
:100A2000384606F0BFFD0AF1010AD5E5032A7FF436
:100A3000D3AD9DF83B30384E63B100234FF6FF72C3
:100A4000082194F80A80384601F021F8334B46F823
:100A5000280013E0BDF8401094F80A80B1F5FA7F41
:100A6000BDF842300FD92E4A3846B2FBF1F20821C8
:100A700092B201F00CF82B4B46F82800C360A37A21
:100A80000133A372A8E5284AB2FBF1F2012192B228
:100A9000D9E7B7F90410C6E5156900EB400C09FA6F
:100AA0000CFA25EA0A0A06FA0CF545EA0A05156168
:100AB00085E60C2B0BD8073B156B03EB83030EFA73
:100AC00003F625EA060598402843106385E60D3BAA
:100AD000D56A03EB83030EFA03F625EA0605984070
:100AE0002843D06279E600BF00240140640800205A
:100AF0003800002035FA8E3CD80D002000093D005A
:100B0000E1150008E8040020B9160008BD19000826
:100B1000D4040020B915000878130020C916000875
:100B200000127A00D916000840420F00BBF9EA30E3
:100B3000002B7FF479AEBBF9EC30002B7FF474AE60
:100B40000026DFF84483C04D10223146C8F800600B
:100B5000C8F80460C8F80860BC4884F83461BBF881
:100B6000F0A09BF8EF909BF8F7700CF004FDC4F830
:100B7000386123206E60AE60A4F83561C4F844612A
:100B800007F085F80DF121020121752001F0E2FA4C
:100B9000A5F59C7500B3AE4B0DF12202C4F83C31B3
:100BA000AC4B0121C4F840314323304684F838313E
:100BB00001F0D0FA9DF8223003F07E038DF8223048
:100BC000002800F0F780682B40F0F480012384F8BF
:100BD00035311D2384F83831002194F835219E4B9E
:100BE000042A1970059340F05D84984B9B4A9C4EF3
:100BF0001A609C4A40F2FD1E5A609B4A0393DA60D9
:100C00003268069142F00100306040F202204B460B
:100C10000A2B28BF00230121994011EA000C40F063
:100C20009D8411EA0E0F00F09984904B42F003026C
:100C300083F800C08E4B3260C8F800308D4BC8F886
:100C4000043033689B0702D5D8F8003098474FF03E
:100C50000009039B50461B689847CA46DFF82C8260
:100C600088F800A01FB1BB1E022B00F2E88012AB77
:100C7000012200210C208DF8489001F031FA002863
:100C800000F0DD809DF84830482B40F0D8807A4B4A
:100C90007A4A1A607A4A5A60062388F80030336824
:100CA00043F0080333609BF8E4300BB1059A1370EE
:100CB0009BF8E5300BB16D4A13709BF8E6300BB131
:100CC00088F800309BF8F830042B00F2E5804FF0F4
:100CD000010808FA03F212F0160662D112F0090FA9
:100CE00000F0D8800A2006F0D2FF0DF1230342461F
:100CF000A021772001F0F4F90746002851D04246A0
:100D00001E21772001F02BFA4FF42F6006F0B4FF7C
:100D1000B046DFF87C91A6F1600112AB0222C9B2A5
:100D200077208DF848808DF8498001F0D9F99DF839
:100D300048209DF8493043EA022326F8093002365C
:100D4000102EE8D100231946B5F8562102F00F06FF
:100D500002F47F42A5F8562121F001002844B0F8A2
:100D60004801002818BF002711F0010F1ABFC0B2B8
:100D7000434083EA1023082013F4004F18BF83F484
:100D8000C05301384FEA4303F6D101311029E3D1B2
:100D90003243A5F8562127B9C3F303339E4200F02E
:100DA000E8832022374B1A6195F83431134385F8D4
:100DB000343176E09DF8213003F07E03682B8DF806
:100DC000213036D10223062184F8353112AAD4F815
:100DD0003C31084698479DF84D309DF84B209B00CC
:100DE000520002F0020203F0040313439DF849206D
:100DF00002F001021343DAB263B1012A03D10023E6
:100E000085F83631E8E6022A01D10123F8E702200D
:100E100006F047FFD4F83C310DF1230201210C20EC
:100E200098479DF8233013F00F03F0D0042BECD13A
:100E3000E5E7702B04BF042385F83531CCE6012F9C
:100E40007FF631AF00270BE7B8050020040700202C
:100E500055210008752300080C020020811D0008A0
:100E60009C0700203519000890C1793D70020020D0
:100E7000291E000879190008E801002081220008D5
:100E8000DD2100080008014064020020F00100207C
:100E9000C8050020012B84D0B14A136843F0040335
:100EA00013602368012B07D14022AE4B1A6194F8DE
:100EB0003431134384F8343195F834410CB1204671
:100EC000A6E7A94DA94E2B780F2743F002032B70FC
:100ED0004FF4005373614FF480433361F36819207A
:100EE00083F40053F360F368013F83F48043F360BD
:100EF000F36883F40043F36006F0C9FE192006F09E
:100F0000C6FE17F0FF07E9D14FF480434FF40058B5
:100F100033614FF40043924FC6F8108033613B6851
:100F20001B0709D5924BC6F814801B68984701220D
:100F3000904BC6F810801A708F4B904E1B68187B30
:100F400008F0F8F88E4908F049F98E4908F03EF8A3
:100F500006F062FF8046308808F0ECF8414608F061
:100F60003DF90BF0C5F8884B1880308808F0E2F89E
:100F70000146864808F0E6F9854908F0E3F9854B13
:100F80007F491860844B854ED86808F027F984495A
:100F900008F024F9834B1B221860FF2130460CF027
:100FA000EAFA0022012132703A687F4B12F0020FF8
:100FB0001970304604D07170032119700221B1708C
:100FC000560704D519784E1C1E700326465412F09D
:100FD0000A0F0CD0042105261A788154511CC9B27D
:100FE0004654D11C197006210232D2B28154049A9F
:100FF0001268910604D519784E1C1E7007264654B7
:101000009BF80510082901D00E2904D119784E1C2F
:101010001E700B2646540C27197847544E1C570750
:1010200048BF0231F6B21E7044BF197010214FF054
:10103000120748BF815519784E1CF6B24754570520
:101040001E7006D59BF888711FB1023119701321EB
:101050008155910504D519784E1C1E7015264654ED
:10106000D20504D51A78511C19701A23835498227A
:1010700000214E480CF07FFA012006F01FFB4FF0D4
:101080004C0ADFF8288108B1012C5ED94849494B48
:10109000BBF8DE201960484B484E1A8000233746C3
:1010A000474A484C138093702160474A474910686B
:1010B0000B70BBF82411DFF81C81DFF81CC100F1B4
:1010C00079020FFA81FED8F8004026F813E004F503
:1010D00016744CF823400133122BF4D13C4CC93028
:1010E0002668F30458BFBBF92AE1A7F806E0137895
:1010F000BBB992F802E0D3789E4512D2BEF1000F40
:1011000000F08E800EF1FF3E0EEB8E0E0EEB8E0E7B
:101110000EF5617392F801E09BB20EF1040E27F810
:101120001E3004329042E2D1330740F18E809BF8AA
:101130001E31062B00F28380DFE813F07A00E60010
:10114000E90014012E01480148010AFB04F908EBEB
:10115000090797F84A60002E40D00134E4B292E7C4
:101160009C07002000080140681800200010014082
:10117000E801002004020020581400203A0000205A
:1011800035FA8E3CDB0FC93FA00200200AE81C4163
:1011900000401C466807002004070020A307002029
:1011A000BD37863584020020A2070020F00200200F
:1011B0007A090020400700203C070020900D002005
:1011C0000C160020FC1500203C160020E100002039
:1011D00000160020C40D0020E40000200379B64A68
:1011E00090F9000002EB8303032201960092D3F8EA
:1011F000A0313246012102F057FE039060B14C222B
:10120000314638460CF0B7F9039B48F80930012302
:101210001C4487F84A30E4B2012002F077FE32E73E
:10122000013303EB830303EB830303F5617371E77E
:1012300045F2F052A14B1A8002F08EFF28B9082027
:1012400006F050FF9E4A9F4B1A6022689E4B12F494
:10125000804F04D012219D4819709A49086042F2CB
:101260000106324202F0010102F400500FD044F6B0
:101270002066924A168020B1082295481A70914A39
:10128000106021B10C2293491A708E4A11601A78AD
:10129000043A5A7006F0D4FC8F4B18609BF8053066
:1012A000052B02BF4FF4C8728C4B1A804FF47A7230
:1012B0008B4B1A80C8228B4B1A808B4A137843F0D1
:1012C00008031370894A137823F00203137040F661
:1012D000020223681A420AD0854A864B1A6003220A
:1012E000854B1A700023854A1380854A138001229A
:1012F000844B9B682360844B1A702B7863F07F03C8
:101300002B7023B0BDE8F08F42F6F82292E742F648
:10131000F8226A4B09011A800A2391FBF3F100239A
:101320007A4AA1F5B06142F823100133122BFAD1A9
:10133000644A774940201160634A137006F0BEF991
:1013400000283FF47CAF0123072790F90000714A81
:101350008DE88800704B402102F0A6FD003018BFD8
:1013600001206BE742F6F822544B40201A806B4A6A
:10137000544B1A601022544B1A7006F09FF9002843
:101380003FF45DAF0123002690F90000644A8DE828
:1013900048004FF4E133DEE742F6F822474B4020A5
:1013A0001A80604A474B1A600822474B1A7006F0B1
:1013B00085F900283FF443AF0023012190F9000094
:1013C000594A8DE80A004FF4E133C4E742F6F821A8
:1013D0003A4A062B11804FF00C023B49DFF870812E
:1013E000DFF870C1DFF870E1504F514E51480A707C
:1013F0001FD0002388F800308CF800308EF80030C1
:101400001B233B70052332704FF4E13603704A4AC8
:101410002C4B40201A6006F051F900283FF40FAF22
:101420000122002390F900008DE80C003346434A66
:1014300091E7002188F800108CF800108EF8001059
:1014400021213270397003703D4EE0E7013B092BDA
:101450003EF6F8AF4FF4005214217A618DF84A102D
:1014600002214FF008098DF84B103648414607928B
:10147000ADF8489000F0D0FA039B3C20C3F81090E0
:1014800006F005FC079A4FF400483A61059AFFF709
:1014900033BA2D4B5B88003318BF0123FFF715B813
:1014A0002A4BF7E71023039A136194F8343143F081
:1014B000020384F8343105E4E0D500088A030020F3
:1014C000BD6200082C000020840D00208D62000801
:1014D000AD6200089D620008B0020020581600208E
:1014E000A8010020480700205A16002034160020CA
:1014F0006C090020FC0D0020D4020020D602002040
:10150000D8020020640800207C040020F014002091
:101510005D620008F5630008A086010049620008CA
:101520005163000831620008096300085F08002069
:10153000F7150020600800207D3F0008913F00085B
:1015400090D0030000080140DC090020E4090020DD
:10155000F81500203D0800203C080020012B4FF02A
:1015600000093FF654AB0E4B9DF818201A70FFF798
:1015700068BB42F21073A5F85831A5F85A31094BEF
:10158000C5F85C31084BC5F86031084BC5F86431CB
:10159000074BC5F86831074BC5F86C317CE400BFD8
:1015A00070020020236E0008656E0008196E0008A6
:1015B000556E0008796C000810F80A3C0133DBB264
:1015C0000A2B00F80A3C07D9002310F8131C034A21
:1015D00022F8113000F80A3C704700BF5C1500206B
:1015E000314A70B5136C9068194440F68C23081A80
:1015F00098429160D0605160134639D9117892F9C0
:101600004520914228D10A1F082A25D893F8462060
:10161000182A03D8013283F8462001E083F84410E9
:1016200093F9442091420FD193F8470060B1002014
:101630001E4C1F4D824211DC00241D480B2A13DD75
:101640001C48027801320270012283F847200022F0
:1016500083F845101A7070BD0022DCE754F8046F5F
:1016600025F810600130E5E720F812400132E5E787
:1016700092F84710B9B140F2DA51A0F2EF248C424F
:1016800008D811780B2905D80B1D0131117042F8CB
:10169000230070BD0022104683F8472099180432B9
:1016A000302A0861FAD170BD8C0400209804002013
:1016B0005C150020B6000020024A136C01330B4475
:1016C000136470478C040020024B53F820301B68D1
:1016D0001980704778130020074B53F82030A1F58C
:1016E0007A701A6819894FF47A73414391FBF3F1C8
:1016F00089B21180704700BF781300208C4B70B501
:101700001A68908A80B2C1B2CE073FD5118821F401
:1017100000610904090C1180118889B241F48061CB
:10172000118000211971597931B3997911B9D97999
:10173000FF2921D101219971197A022901BF11884C
:1017400089B241F400611180597A41F0010111829E
:101750001A7A93F90410013291420CD100229A7145
:101760009A7A32B119688A8822F440721204120CF3
:101770008A8000221A7670BD597A01F0FE0111822A
:10178000DA79FF2AE4D0FF221A71E1E78D073ED50E
:10179000BFF35F8F187AC0B2012818D15979B1B15F
:1017A0009979A1B1118821F480610904090C118093
:1017B000BFF35F8F118B1188987289B241F4007169
:1017C0001180918889B241F480619180C0E7118BCA
:1017D000BFF35F8F197A02290FD1597969B19979CD
:1017E00059B1118821F480610904090C1180918894
:1017F00021F480610904090CE7E7197A0329E0D193
:1018000059790029DDD099790029DAD0EFE74C0722
:1018100051D5012199725979002938D09979002937
:1018200035D0197A93F90400022911881ED921F4C0
:1018300080610904090C1180148ADD68E4B22C541B
:10184000C1B2108880B240F400701080881C1871FA
:10185000108A013149B2C0B26854918889B241F40A
:10186000806191801188CE05FCD471E789B241F482
:1018700000711180148ADD68E4B22C54C1B2148A5C
:10188000481C40B2E4B22C5403311971EAE799794B
:1018900009B9197C39B1118889B241F400711180FC
:1018A00019790131F1E7118889B241F48071118011
:1018B00001219971D6E711F040011AD093F9046023
:1018C000118ADD68C9B2F4B2A955601C40B21D7A14
:1018D000C11C8D42187105D1918821F480610904E1
:1018E000090C91801A7A90427FF432AF02341C7155
:1018F0002EE705067FF52CAF93F90400441C0AD0AF
:101900005C69411C205C49B21082187A19718842C6
:101910007FF41EAF6BE71971D979118259790029CB
:101920007FF465AF197A00297FF412AF5FE700BF3B
:10193000F005002037B50F4B04465D686A46062166
:101940001878A847A0B19DF800209DF8013043EA1F
:10195000022323809DF802209DF8033043EA0223EE
:1019600063809DF804209DF8053043EA0223A3809C
:1019700003B030BDB805002013B50F4B04465B68BB
:101980006A4606213B209847A0B19DF800209DF8AB
:10199000013043EA022323809DF802209DF80330A2
:1019A00043EA022363809DF804209DF8053043EA52
:1019B0000223A38002B010BDB805002038B510F88E
:1019C0000E2C044650F8043C5AB9012220F80C1C95
:1019D00000F80E2C997A18680222BDE8384003F00E
:1019E000CBBB002530F80C2C20F80A1C891A89B2D0
:1019F00020F8081C074A10F80F0C22F8101004F801
:101A00000E5C2A46997A186803F0B6FB04F8065C67
:101A100038BD00BF5C1500202DE9F04300234FF0D6
:101A20000F0E01260F8847FA03F2D20723D58C78D0
:101A30004FEAD30814F0100F18BF91F8039003F089
:101A4000070504F00F024FEA850550F828C018BFBB
:101A500042EA09020EFA05F92CEA090CAA4042EA08
:101A60000C02282C40F828200AD1C26806FA03F498
:101A700022EA0402C2600133102BD4D1BDE8F08306
:101A8000482CF8D1C46806FA03F22243F2E72DE9A4
:101A9000F74316460546DFF890920A4699F8194032
:101AA000314600689846631C89F8193005F00AFD34
:101AB0002B8901A9ADF8043018238DF806300223D4
:101AC00068688DF80730FFF7A7FF95F80AE009F17D
:101AD0001C07240127442A684946BEF10C0F43D84D
:101AE000DFE80EF00742424268424242A0424242D0
:101AF000D900138CDFF8349223F001031B041B0C74
:101B00001384138CB2F804C0108B4A4520F0730084
:101B10004FEA00404FEA10409BB21FFA8CFC40F0A5
:101B200070003ED009F500694A453AD009F5406990
:101B30004A4536D009F580694A4532D009F58069B1
:101B40004A452ED023F0020343F00303A2F804C059
:101B50001083A2F834801384138B23F008031B0432
:101B60001B0C43F0080313832B7B43B1B2F84430C2
:101B70006FEA43436FEA53439BB2A2F844301388A1
:101B80009BB243F001031380BEF10C0F00F2B98049
:101B9000DFE80EF0B3B7B7B7BEB7B7B7C2B7B7B7DE
:101BA000C60023F00E032CF4407C43F003034CF4F6
:101BB000807CCBE7138CDFF8749123F010031B04B7
:101BC0001B0C1384138CB2F804C0108B4A4520F40C
:101BD000E6404FEA00404FEA10409BB21FFA8CFCEF
:101BE00040F4E04015D009F500694A4511D023F0D2
:101BF000200343F03003A2F804C01083A2F8388019
:101C00001384138B23F400631B041B0C43F4006345
:101C1000A9E723F0E0032CF4406C43F030034CF4CC
:101C2000806CE8E7138CDFF8049123F480731B04C5
:101C30001B0C1384138CB2F804C0908B4A4520F01F
:101C400073004FEA00404FEA10409BB21FFA8CFC31
:101C500040F0700016D009F500694A4512D023F40F
:101C6000007343F44073A2F804C09083A2F83C8050
:101C70001384938B23F008031B041B0C43F008030D
:101C8000938371E723F460632CF4405C43F4407366
:101C90004CF4805CE7E7138CDFF8909023F48053DA
:101CA0001B041B0C1384108CB2F804C0938B20F41B
:101CB000005023F4E6431B0400041B0C000C4A45AF
:101CC0001FFA8CFC43F4E04340F4405003D009F584
:101CD00000694A4503D12CF4804C4CF4804CA2F8A6
:101CE00004C09383A2F840801084938B23F4006394
:101CF0001B041B0C43F40063C2E70B1902F1340010
:101D0000D861384621448E840A6203B0BDE8F0836E
:101D10000B1902F13800F3E70B1902F13C00EFE771
:101D20000B1902F14000EBE7F0050020002C014008
:101D300013B5104C94F8DC20CAB90F4B1B68B3B133
:101D40001A681AB10D49886902438A619A889868AD
:101D5000ADF8042002228DF8072004220DEB0201C9
:101D60008DF80620FFF758FE012384F8DC3002B01E
:101D700010BD00BFF0050020C40500200010024087
:101D800070B50446FFF7D4FFB4F5807F3DD0BB2C7F
:101D90003DD8612C3DD8292C3DD8132C3DD8092C99
:101DA0003DD8002C0CBF002506251E4C8021A368C1
:101DB0006B209847642005F06AFFA368072168201C
:101DC0009847642005F063FFA36800216B209847C3
:101DD000642005F05CFFA36818211B209847A368C6
:101DE00010211C209847A36829461A209847A36809
:101DF00003211D209847A368002119209847A36854
:101E00001221BDE87040372018470025CDE7012595
:101E1000CBE70225C9E70325C7E70425C5E7052564
:101E2000C3E700BFB805002008B5FFF781FF4FF4F6
:101E30008052014B1A8008BD3A000020012828BFBB
:101E400001202DE9F04F4FF0140E06460EFB00F373
:101E5000704FDFF8D881F918F8586F4B88F8DD60BB
:101E6000DC690A69C8F800002243DA6182880D89BA
:101E700022F440721204120C82800222B1F80AA0ED
:101E80004C6889B045EA0A09C4F8109003A92046B5
:101E90000193ADF80C908DF80F208DF80EE0FFF750
:101EA000BBFD019B00974FF0080B1F46A26815422F
:101EB00000F0A2800A20656105F0DEFE25610A209F
:101EC00005F0DAFEBBF1010BF0D1C4F814A00A2032
:101ED00005F0D2FE65610A2005F0CEFE25610A20DC
:101EE00005F0CAFE0222C4F810A08DF80F201C22B3
:101EF00003A920468DF80E20ADF80C90FFF78CFD5D
:101F0000D8F80040454A03A894423A690BBF42F40E
:101F1000001242F480023A613A610BBF3A693A69B1
:101F200022F4001222F480023A61A38823F4407361
:101F30001B041B0CA38023889BB243F00103238066
:101F4000A58802F01DFB059B354A364825F03F0564
:101F5000B3FBF0F0B3FBF2F3002B08BF01232D0419
:101F60002D0C0543ADB2A58021884FF4967221F067
:101F700001010904090C21804FF47A716FEA43438F
:101F8000424392FBF1F26FEA534301329BB292B2A9
:101F90002284A383238800259BB243F0010323807E
:101FA0002388009A23F4816323F002031B041B0C93
:101FB00023804FF4804323811423012403FB06264E
:101FC000737B03A88DF80C308DF80D508DF80E50F2
:101FD0008DF80F4002F036F8337B9DF80F208DF816
:101FE0000C308DF80D508DF80E504AB103A802F058
:101FF00029F809B0BDE8F08F0A2005F03DFE55E74D
:102000005A09094903F01F0304FA03F3203241F887
:102010002230EEE7CCD70008001002400054004008
:10202000804F120040420F0000E100E0F005002068
:1020300010B5214C2368998A89B211F4706F1CBFC6
:10204000012284F8DE2011F4E06F1FD01A8B9A88E9
:10205000890522F480624FEA02424FEA12429A80D6
:1020600014D41A88920511D41A88D00518D51A8864
:10207000D105FCD41A8892B242F400721A801A88F0
:102080009205FCD494F8DD00FFF7D8FE2268938A0D
:1020900023F470631B041B0C93820023237610BD72
:1020A0001A8892B242F400721A809A8822F440721E
:1020B0001204120C9A80E9E7F0050020064A08B5E0
:1020C000138801339BB21380044B93F8DD00FFF7B4
:1020D000B5FE002008BD00BF98070020F0050020D5
:1020E00010B440001A4CC0B26072E17101200021AE
:1020F00021746071227220762068E360636184F845
:10210000DE1018B383889B0515D40388D9050DD438
:1021100047F230530288920503D5013BFAD110BC37
:10212000CCE703889BB243F48073038083889BB21F
:1021300043F44073838047F23053227E12B1013B57
:10214000FBD1ECE794F8DE0080F0010010BC704792
:10215000F005002013460A4601466820C0E713B583
:102160001D4B400002ACC0B2587204F8012DD97169
:102170000122002118681A745C615971DC601A72BE
:102180001A7683F8DE1070B18288920517D402881F
:10219000D4050FD447F230520188890505D5013A9C
:1021A000FAD1FFF78BFF02B010BD028892B242F461
:1021B00080720280828892B242F44072828047F23A
:1021C0003052197E11B1013AFBD1EAE793F8DE00F3
:1021D00080F00100E7E700BFF005002037B50446B6
:1021E0006B46012202210C20FFF77AFF10B9002074
:1021F00003B030BD9DF80030DA07F8D56B460722F2
:1022000003210C20FFF76CFF0028F0D09DF806306A
:102210009B07ECD19DF801309DF80000174D40EA76
:10222000032000B206F086FF296806F0D7FF07F00A
:10223000B1F99DF8033020809DF8020040EA0320A8
:1022400000B206F077FF696806F0C8FF07F0A2F950
:102250009DF8053060809DF8040040EA032000B23C
:1022600006F068FFA96806F0B9FF07F093F90122AC
:10227000A0800A210C20FFF772FFB9E718000020A8
:1022800013B500220A210C20FFF769FF142005F086
:10229000FEFC0F220A210C20FFF761FF0A2005F047
:1022A000F6FC01AB032210210C20FFF719FF0A20D6
:1022B00005F0EDFC9DF9040006F03CFF4FF086416F
:1022C00006F082FE4FF06E5106F088FF4FF07E510F
:1022D00006F07CFE254906F081FF254C20609DF923
:1022E000050006F027FF4FF0864106F06DFE4FF027
:1022F0006E5106F073FF4FF07E5106F067FE1B49EA
:1023000006F06CFF60609DF9060006F013FF4FF0C9
:10231000864106F059FE4FF06E5106F05FFF4FF018
:102320007E5106F053FE114906F058FF0022A060CE
:102330000A210C20FFF713FF0A2005F0A8FC0DF17D
:102340000303012202210C20FFF7CAFE0DF1030353
:10235000012209210C20FFF7C3FE01220A210C20D3
:10236000FFF7FDFE012002B010BD00BF0000F041EC
:10237000180000200A4601466820F0E6FFF7BEB9C3
:10238000FFF7BCB954E653E62DE9F04F87B003934D
:10239000974B07461E88029116F00206019212D052
:1023A000944BB3F90060B3F90230002EB8BF764207
:1023B000002BB8BF5B429E42B8BF1E46B6F5007FF9
:1023C000A8BF4FF400760025DFF854B207F1010AE8
:1023D0000421884B4FEA450933F91520864B5200FA
:1023E00033F91530002B93FBF1F1B8BF5B42B3F525
:1023F000206F00F3F3805BF82500531A0344B3F514
:102400007A5FA8BF4FF47A537C488342ACBF4BF845
:1024100025304BF825005BF825009AF80A40C011DA
:102420004443A0119AF80040714B54431B884FEA73
:1024300085089B0700900AF1010A4FEAA4143BD0DB
:10244000019B5B429A4203DB019B9342A8BF134668
:1024500042F2107E6A4A6B4839F902209B1A039AAD
:1024600032F91520134458F800201A447245A8BFC9
:102470007246DFF8BCE17245B8BF724648F80020EA
:10248000387A4343387FDB1100EB8000C0F1000E47
:10249000734503DB8342A8BF03469E46BB7CA4EB87
:1024A0000E045A43009B1213981A7043744302EBB4
:1024B000602300930EEB6424534B97F851205B5D2F
:1024C0005943A4EBA1146AB15049204641440592F6
:1024D000049106F02FFE059A049905F047FC07F0D9
:1024E00059F804460420444B39F90310484B39F994
:1024F000032029F803108A1A92FBF0F219180C3302
:1025000058F801E058F8030048F8012070441044DE
:1025100097F8502048F803E052B13E4904928844AD
:1025200006F008FE049A414605F020FC07F032F858
:10253000394B3A4A5B5D01355843009B022D1C44E0
:10254000A4EB601029F802007FF442AF0420029B44
:1025500099790F314B002749B1F904105943264BA3
:102560004911B3F90430002993FBF0F3A1EB030305
:10257000B8BF494232292A4834DC8468797B03FB9E
:102580000141284CA142A8BF2146274CA142ACBF23
:1025900081608460F9784B4324499B1109780329B1
:1025A0000AD9B7F84E10B1F5FA7F05D24C42A342D2
:1025B0001BDB8B42A8BF0B4681686FF0FF0041F325
:1025C0004F31B1F5807FA8BF4FF480718142ACBF1D
:1025D0005B181B18938007B0BDE8F08F00234BF801
:1025E000253018E700218160D4E72346E4E700BFE7
:1025F000A0070020D4120020C407002080C1FFFFE4
:10260000B80D00203013002038130020E012002005
:10261000D00600201C130020501300202813002097
:10262000EC120020FEFFFF0F020000F05313002009
:10263000F0D8FFFF2DE9F04F87B003938F4B029244
:10264000B3F90020B3F90230002AB8BF5242002B80
:10265000B8BF5B429A42B8BF1A460026B2F5FA7F6D
:102660001346A8BF4FF4FA738146B246B3463446C8
:1026700000930196824B67001A8812F003003FD046
:10268000022C39D07D4BD95F029B49005B429942B5
:1026900003DB029B8B42A8BF0B46642579496FF090
:1026A000040EC95F5B1A039931F914100B4499F8B1
:1026B0000810594391FBF5F199F81C500EFB05FBEE
:1026C000594505DB05EB85058D42A8BF0D46AB4698
:1026D0006D4D55F824100B4442F210718B42A8BF87
:1026E0000B466A498B42B8BF0B4699F8121045F861
:1026F00024304B431B130193012801D1022C36D106
:102700005E4BA00033F907A0614B624ED95F81EAAE
:10271000E173A3EBE173B3F5206F00F3A180022C0A
:1027200000F09780502505FB0AF509EB04035B7860
:1027300095FBF3F5042391FBF3F3EB1A35581D4495
:10274000B5F57A5FA8BF4FF47A55534B9D42ACBFA5
:10275000355033504F4B09EB040153F824607D236F
:1027600096FBF3F3CE7A5E43402396FBF3F6910794
:1027700079D5022C77D04FF4FA75009B009903FBB2
:102780000AF871430198C3F5FA720BFB028800FB4B
:10279000021298FBF5F392FBF5F53D4A3F4932F9F9
:1027A0000780042298FBF2F214F8018008FB02F87B
:1027B0006FF04F0298FBF2F899F85120984472B1EB
:1027C0003749404601EB84010592049106F0B2FCC2
:1027D000059A049905F0CAFA06F0DCFE804604204A
:1027E0002B4BD95F2F4BDA5F03F1080E8A1A92FB4D
:1027F000F0F2D95314335EF824C053F824004EF895
:1028000024206044104499F85020A10043F824C0CB
:102810005AB1254B05921944049106F08BFC059A98
:10282000049905F0A3FA06F0B5FE204B454413F8D1
:1028300004801F4B00FB08F04FF0200890FBF8F0DD
:102840000134281A032CD8537FF414AF07B0BDE825
:10285000F08F8AEAEA73A3EBEA73642B7FF762AF27
:102860000023335076E7D30704D5022C02D0019D14
:102870005B4692E7354653468FE700BFD4120020EF
:10288000A0070020B80D002030130020F0D8FFFF73
:10289000C4070020EC12002080C1FFFF3813002085
:1028A000E0120020E40600201C130020501300203A
:1028B000281300202DE9F04F89B00593AA4B8046DC
:1028C00018880C46049206F031FCA84906F086FCF4
:1028D000A74B02901B889B074CD5129BA54ADD890C
:1028E00040F2E633B2F90000401B00F2F3119942C6
:1028F0001146B1F9023040F2E63198BF80EAE07249
:10290000A3EB050398BFA2EBE07203F2F31088BFBC
:102910004FF4FA72884230D883EAE370A0EBE37098
:102920009042B8BF104698F84C504DB3C0F5FA70BD
:1029300006F000FC904906F005FD4FF07E5106F0D0
:1029400043FB0646642090FBF5F006F0F3FB0146DE
:10295000304606F043FC4FF07E5106F037FB002175
:10296000074606F0D9FD58B94FF07E51384606F0BB
:10297000F1FD30B14FF07E5703E04FF4FA70D2E72B
:102980000027231D0024039308F120030193039BD8
:10299000620013F8015B022C03930692774B55D12A
:1029A000B3F904000A35684306F0C4FB744906F025
:1029B000C9FC0546734B6200985E06F0BBFB724B88
:1029C000196C06F00BFC0146284606F0FDFA019B47
:1029D000834653F8046B01936C4B185D06F0AAFB19
:1029E00031460546584606F0F9FB0146284606F0F2
:1029F000F5FB674906F0A6FC98F8512082462AB1FB
:102A0000644901EB840105F0B1F982465946029808
:102A100006F0E4FB019B604E996806F0DFFB5F491E
:102A200006F0DCFB56F8241006F0D0FA5C49A5004D
:102A3000814606F071FD002844D15A49484606F007
:102A400089FD002840D0DFF85C913DE033F9146047
:102A5000049B5842864203DBB342A8BF3346184664
:102A6000514B62009B5EC01A059B33F91430184429
:102A700006F060FB494906F065FC3D4B8246B3F821
:102A8000009019F0010F04D0D8F8441006F0A6FB0E
:102A90008FE705F11400704306F04CFB384906F04F
:102AA00051FC19F0020F054684D0D8F84810504662
:102AB00006F094FB394606F091FB0146284606F0E5
:102AC00085FA76E7DFF8D89046F80590374E5846F5
:102AD000A95906F079FA45F806B0069002994FF028
:102AE0007E5006F02FFC069B194606F077FB8346C6
:102AF00006F10C03EA581836A959104607930692B6
:102B000006F064FA594606F061FA069A079BAA5144
:102B100098F85020864645F803B022B1244929444C
:102B200005F024F986467046224906F00BFC019B0D
:102B3000596906F053FB154B0546185D06F0FAFA85
:102B40000146284606F04AFB114906F0FBFB1A49EC
:102B5000054606F0E1FC98BB1849284606F0FAFC49
:102B600078B3164D2DE000BF54180020BD378635D0
:102B7000A0070020900D00200000FA43D41200208E
:102B800000004842C4070020D0060020DC120020CC
:102B90000000C842E01200205C1300200000204129
:102BA00000007AC300007A43B80D0020140700200B
:102BB0001C13002000004040000096C30000964314
:102BC0000E4D4946504606F001FA294606F0FEF938
:102BD00009F08EFAB0F57A7FA8BF4FF47A70084BEF
:102BE00062009842B8BF18460134064B032C985235
:102BF0007FF4CDAE09B0BDE8F08F00BF000096C3F2
:102C000018FCFFFF281300200022044B1A605A60B2
:102C10000022034B1A605A60704700BF3013002037
:102C200054130020012310B50A4C4FF48060E37068
:102C3000022384F8203005F047FA6421064B1A6815
:102C4000064B9B6E5B7801FB032363612388013392
:102C5000238010BD0C160020C40D0020D0060020DB
:102C60002DE9F74F714B724A93F821809946B8F1DC
:102C7000010F92460CBF002703276E4E116835786E
:102C800001F080616C4CDFF8CCB105F004050091D7
:102C900099F82020052A45D8DFE802F0034C578830
:102CA00098B3002D35D0654AB2F86C10106F0192C0
:102CB00004F086FD0128019A08D14FF0640E916E50
:102CC0002068C9880EFB0101C9F81010009B63B190
:102CD000926E12794AB1FFF7A5FF032289F82020EE
:102CE0004FF47A72C9F81C20D2E7B8F1010F19D05D
:102CF0002268D9F81010914207D2FFF793FF032200
:102D000089F8202040F6B832ECE7012289F820202B
:102D1000BEE7009B4FF480604BB105F0D5F900226F
:102D2000C9F81020002F7BD103B0BDE8F08F05F06B
:102D3000BCF9F4E7B8F1010F01D10522E6E7FFF78E
:102D400071FF20213E4A1170A2E74FF4806005F028
:102D5000ACF95DB1BBF8DE103A4804F031FD10B3B8
:102D6000364A926E5188384AD18002272268D9F8B3
:102D70001410914211D385B13449B1F90020002AD1
:102D8000B8BF5242B2F5FA7F07DCB1F90220002A3F
:102D9000B8BF5242B2F5FA7FC4DD47F23052C9F8EB
:102DA0001C200322B2E705F021FCDEE705F01EFC43
:102DB0002168D9F81C200A44C9F81820042289F88F
:102DC00020204FF4806005F070F961E7B8F1010F41
:102DD00010D12268D9F818109142A3D21C4A127857
:102DE0001AB9DAF80020D3079CD4327822F0020214
:102DF0003270A2E72168D9F81C200A44C9F81820CB
:102E000090E764200D4A2168926ED28800FB02127E
:102E1000C9F81020002289F8202089F80320D0E783
:102E2000384603B0BDE8F04F04F0F2BC0C160020A9
:102E30008C0D002034160020C40D0020D006002088
:102E4000250000207A090020900D0020BE070020F8
:102E5000280000206408002046F2A7132DE9F04F57
:102E6000B14C85B0676FC71B9F4240F25181B4F8E7
:102E70007850606765B3D4F88430D4F880001B784C
:102E8000E26F013BB0FBF3F3082092FBF0F1521A22
:102E90001344E36793FBF0F006F04CF9A34906F006
:102EA00051FAA34909F0B0F901464FF07E5006F0FF
:102EB0008BF8A04906F092F906F06CFB6B1EA4F8A3
:102EC00078300023C4F88800C4F88C30C4F89030FF
:102ED000D4F88450D4F880002B78DFF87CA2013B32
:102EE000B0FBF3F006F022F9904906F02BFA904976
:102EF00009F08AF901464FF07E5006F065F88D49D9
:102F000006F06CF909F0F4F8D4F888306D68C01A4E
:102F100006F010F9294606464FF07E5006F054F8A8
:102F20000146304606F05AF90646D4F8940006F0F9
:102F300001F9294606F052F90146304606F046F8F6
:102F400009F0D6F8C4F894000646DAF8000006F056
:102F5000EDF87949814606F041F9784B80461D68C5
:102F6000CDF804A0002D00F0D680754B986806F0CF
:102F7000E1F88246284606F0DDF80146504606F0A4
:102F8000E1F90546D4F89810284606F027F9494695
:102F900006F024F94FF07C51834606F01FF94146B4
:102FA00006F01CF9D4F88C9082464946404606F05B
:102FB00015F90146504606F009F8D4F8901006F0CD
:102FC00005F86049039006F009F909F091F83046D8
:102FD00006F0B0F8D4F89C800290D8F80CA04FF01E
:102FE0007E50514605F0F0FF029B0146184606F060
:102FF000F5F8039A51460290104606F0EFF8029B4E
:103000000146184605F0E2FF4946C4F890008246A2
:10301000584605F0DBFF00224949B4F878900A6071
:103020004A608A604549C4F88C000A6001990A60C8
:10303000B9F1000F6CD10190504606F0ABFADFF801
:103040001CB1CBF80000D4F8A000301A06F072F8DA
:103050003D4906F0C3F88246384606F067F8014657
:10306000504606F06FF906F095FA40F2DC529042B5
:10307000A8BF1046A2F6B8329042B8BF10460A2147
:10308000C4F8A06004F0B9FE06F054F8D8F808605F
:10309000074631464FF07E5005F096FF0146384610
:1030A00006F09CF8019B07463146184606F096F854
:1030B0000146384605F08AFFC4F88C0009F018F87C
:1030C0000521074604F099FE40F23E621F4B20495D
:1030D00018600B8803F21F339BB2934205D84B88CC
:1030E00003F21F339BB293423AD9D4F8A830C4F804
:1030F000B490987B06F01AF8164906F023F90146B9
:103100004FF07E5005F060FFC4F8B850C8F80C00CE
:1031100005B0BDE8F08F002534E7D4F8AC0052E0EC
:10312000C4F8B0A06CE000BFD006002080E6C54720
:10313000B1DC423ED048874ABD3786357C1400203A
:103140006C1400200000C84200247449C00D002007
:10315000B80D002000007A4478140020EC0700200D
:103160003F4BD4F8B86093F800A01AF0040A04D1D9
:10317000DBF800306433C4F8A4303A4B1B78002BE2
:10318000CBD1DBF80000D4F8A4300A211B1AB3F528
:10319000FA7FA8BF4FF4FA7333489842B8BF184675
:1031A00004F02BFED4F8A8301B795843802390FB01
:1031B000F3F0B0F5967FA8BF4FF49670A3F5D673E1
:1031C0009842B8BF18462022D4F8A810C01B91F826
:1031D0000A90264B00FB09F999FBF2F2B2F5967FB3
:1031E000A8BF4FF496729A42B8BF1A46BAF1000FC0
:1031F00096D0D4F8B0300F7D00FB0730C4F8B00093
:10320000D4F8B0301A48B3F5161FA8BF4FF4161300
:103210008342B8BF03464FF4005993FBF9F9C4F851
:10322000B030887F914405F085FF31460746284637
:1032300005F0CCFE0146384605F0D0FF4FF06C514A
:1032400005F0CCFF06F0A6F99628A8BF96206FF0EF
:1032500095039842ACBFA9EB0009A9EB030944E729
:1032600034160020240000200CFEFFFFD4FEFFFFD8
:103270000080DAFF0F4B10B51B681B0704D4BDE8B4
:103280001040082004F011BF0B4B1C8814F00804F8
:103290000FD1082004F018FF084A094B1268C3F840
:1032A000B040C3F8A42040F2DC52C3F8B440A3F805
:1032B000BC2010BD8C0D0020A0070020EC070020D2
:1032C000D006002014490B7813F0010F03F004021C
:1032D0001CD0FAB91148006840011BD4980715D4D6
:1032E0004FF47A7043F004030B700D4B0D4A1B88AA
:1032F000A2F8BE300C4B19680C4B93F86E3100FBF2
:1033000003130520C2F8C03004F082BA12B90120BC
:1033100004F0A2BA704700BF341600208C0D0020C4
:10332000E8070020D0060020C40D0020640800201B
:10333000034B1B68DA79511CD9711344187A704712
:103340003016002010B5FFF7F3FF84B2FFF7F0FF4F
:1033500004EB002080B210BD10B50446054B214699
:10336000186803681B689847034B1B689A79544098
:103370009C7110BD940700203016002038B504461B
:1033800024200D46FFF7E8FF4D20FFF7E5FF002C56
:1033900014BF21203E20FFF7DFFF0022054C284606
:1033A00023689A71FFF7D8FF236893F84900BDE8B6
:1033B0003840D1E73016002001460020DEE710B586
:1033C0000446C0B2FFF7C8FF200ABDE81040C3E7BB
:1033D00010B5044680B2FFF7F2FF200CBDE81040A4
:1033E000EDE746282DE9F74F044600F020857DD80B
:1033F0002C2800F0728438D8052800F057811AD89C
:10340000022800F03A8104D8012800F02981002028
:103410003FE1032800F040810428F8D10620FFF79F
:10342000CBFF0024AF4D285D0134FFF795FF042C3E
:10343000F9D1002039E2262800F02D840AD822286C
:1034400000F063832428E2D10420FFF7B5FFA64BE8
:10345000986873E0282800F02D842A28D7D101200D
:10346000FFF7AAFFA04B587904E13A2800F0418207
:1034700016D8342800F06C8308D83228C7D1012030
:10348000FFF79AFF984B93F82001F3E0362800F0FD
:10349000B4843828BBD10420FFF78EFF924CD0E3D0
:1034A000402800F07B840FD83B2800F027833D287C
:1034B000ADD18D4C0220FFF77FFF94F86E01FFF72E
:1034C0004BFF94F86D01D5E0422800F07584452843
:1034D0009DD11320FFF770FF0024844D285D013437
:1034E000FFF73AFF0B2CF9D100F0AABC6E2800F0D0
:1034F00005824CD8652800F0078122D84B2800F0BF
:103500001F8407D8492882D10220FFF755FF764B48
:103510009889CAE14D2800F0228464287FF477AFAF
:103520000720FFF749FFE720FFF716FF6E4B58799A
:10353000FFF712FF0020FFF70FFF0420FFF748FFFF
:10354000A6E0692800F0B48111D8662800F08581D2
:1035500068287FF45CAF1020FFF72EFF0024644D35
:10356000285D0134FFF7F8FE102CF9D190E06C28AB
:1035700000F0B1816D287FF44AAF0620FFF71CFFF1
:103580005C4B986DFFF724FF5B4B18888DE1742826
:103590004ED015D8702800F01D82C0F0DC81722852
:1035A00000F0198373287FF432AF0820FFF704FF7F
:1035B0000124E0B20134FFF7CFFE092CF9D167E016
:1035C000A02800F05A8320D8752800F08B82772835
:1035D0007FF41DAF474C0025A07BFFF7EDFE4FF0B9
:1035E0000C08464E04F10F07A37B9D4250D20023E6
:1035F000E85D08FB03F29119925D824200F02F848E
:1036000001331C2BF5D10135EEE7F02800F02883BB
:10361000FE287FF4FCAE0820FFF7CEFE0020FFF767
:10362000CEFE0020FFF7CBFE0020FFF7C8FE00E72C
:1036300000274FF0010BDFF8BC8008F10F0A0024CF
:10364000DFF8B89098F80E309C42C0F2A682BBF129
:10365000000F1DD0F8B2FFF7AFFE4FF0000BEEE702
:103660000320FFF7A9FE0020FFF776FE2046FFF7B4
:1036700073FE0D20FFF770FE0AE00420FFF79CFEAA
:1036800000241F4D285D0134FFF766FE042CF9D19C
:10369000012003B0BDE8F08FFFF78EFE0220FFF798
:1036A0005BFE0020FFF758FE0020E3E71A20FFF73B
:1036B00083FE00240D4D285D0134FFF74DFE0B2CD9
:1036C000F9D100240F4D285D0134FFF745FE082C89
:1036D000F9D1002400200134FFF73EFE072CF9D178
:1036E000D6E700BFA0DA000864080020A5DA0008C9
:1036F000D007002094070020C00D002058D80008F3
:103700009BDA0008B1DA00080B20FFF755FEA64B44
:10371000A64C1878FFF753FEA0880F3480B2FFF74D
:103720004EFE54F8070CC0F3C003C0F380029B00A8
:1037300043EA4203C0F340021343C0F3401243EA9A
:10374000C20300F010001843FFF739FE34F8030CF1
:10375000974910F0010F0CBF4FF000094FF002091C
:1037600010F0020F0CBF4FF000084FF0040810F0EB
:10377000040F0CBF00231023D1F800A000F00802B2
:103780000AF4475111430AF4804211430AF40042FB
:1037900011430AF4803211430AF4003211430AF44F
:1037A000802211430AF4002211430AF480121143CB
:1037B000804A10F0400F12780CBF4FF0000C4FF011
:1037C000200C0AF0007A10F0100F0CBF4FF0000E22
:1037D0004FF4007EC2F3800210F0200F4AEA01018C
:1037E0000CBF00274FF480670A4310F4807F0CBFA2
:1037F00000264FF4006642EA090210F4007F42EA14
:1038000008020CBF00254FF4001510F4806F43EA46
:1038100002034FF000000CBF00224FF0806243EA29
:103820000C0343EA0E033B4333432B43134301256D
:10383000024614F8016CB24205D3FFF7C9FD5E4B96
:1038400093F8EC0416E7115D05FA01F119421CBF6B
:1038500005FA02F108430132EDE71220FFF7ACFD53
:10386000564B00251B88514CB3F5806F94BF012641
:10387000082604F12A0737F91500013590FBF6F008
:1038800080B2FFF79CFD032DF5D1208EFFF797FD49
:10389000608EFFF794FDA08EFFF791FDE08EFFF79D
:1038A0008EFD208FFFF78BFD608FFFF788FDEFE621
:1038B000434D00242878434E400000F0FE00FFF7FF
:1038C0007BFD2B789C42BFF4E3AE36F81400FFF783
:1038D00076FD0134F5E73C4C0620FFF76DFD2088AE
:1038E000FFF76DFD6088FFF76AFD304BB3F85400B9
:1038F000DBE70420FFF760FD00201FE60720FFF74D
:103900005BFD324B4FF6FF751888284CFF28A8BF87
:10391000FF20C0B2FFF720FDE06DA842A8BF2846F7
:1039200020EAE07080B2FFF74AFDB4F86000FFF7CC
:1039300046FD214B93F813314BB10A20636E584377
:10394000A842A8BF284620EAE07080B2ADE7606ECA
:1039500000F30F00F9E71E4C0B20FFF72DFD236845
:1039600000251878FFF7F8FC23685878FFF7F4FC77
:1039700023682B4418790135FFF7EEFC032DF7D1AE
:103980002368D879FFF7E8FC23689878FFF7E4FC10
:103990002368D878FFF7E0FC23685889FFF70FFD0C
:1039A0002368187A66E600BF2500002094070020EF
:1039B0008C0D002034160020640800203A000020FE
:1039C000840D0020900D0020B80D0020A80E0020CE
:1039D000BC0D0020D04C1E20FFF7EEFC2368002514
:1039E0001B78022B6BD1DFF83C83CC4FCC4E236885
:1039F00005F1080253F82200414605F0EFFB08F0FC
:103A000077FB80F30800C0B2FFF7A6FC23683946B5
:103A100003EB8503D86A05F0E1FB08F069FB80F34E
:103A20000800C0B2FFF798FC236805F10E0231468A
:103A300053F8220005F0D2FB08F05AFB80F308008F
:103A4000C0B20135FFF788FC032DD0D1B54E072D4C
:103A5000236827D13146586C05F0C0FB08F048FBBD
:103A600080F30800C0B2FFF777FC23683146986CFA
:103A700005F0B4FB08F03CFB80F30800C0B2FFF790
:103A80006BFC236893F84C0005F050FB08F030FB0A
:103A9000FF28A8BFFF20C0B20135FFF75DFC0A2D4B
:103AA000D5D1F5E52B445878FFF756FC23682B4415
:103AB000D87AFFF751FC23682B44587DECE7236844
:103AC0002B445878FFF748FC23682B44D87AFFF73B
:103AD00043FC23682B44587D0135FFF73DFC0A2D3C
:103AE000EDD1D5E52F20FFF767FC8F4C14F8010FBF
:103AF00000283FF4CDADFFF72FFCF7E70120FFF7DB
:103B00005BFC854B1B681878B4E55020FFF754FC2C
:103B100000250C27DFF80082844ED8F8004004EB23
:103B2000850494F87930013507FB0363187AFFF7B1
:103B300013FC94F87A00FFF70FFC94F87B00FFF772
:103B40000BFC94F87C00FFF707FC142DE5D19FE5F2
:103B50004820FFF731FC002506266F4F3C6806FB26
:103B6000054494F8CE00FFF7F7FB94F8C900FFF77F
:103B7000F3FB94F8CA00FFF7EFFB94F8CB00FFF7D4
:103B8000EBFB94F8CC00FFF7E7FB013594F8CD0090
:103B9000FFF7E2FB0C2DE1D17AE500230C2514F8A8
:103BA0000A0005FB03F202EB090112F80920824228
:103BB00000F04A8101331C2BF3D1013442E51F444C
:103BC000FBE715F8010B0193FFF7C6FB019BAA1B4E
:103BD0009A42F6DBF1E7564C1620FFF7EDFBB4F8FE
:103BE0002401FFF7ECFBB4F8D000FFF7E8FBB4F8D2
:103BF000D200FFF7E4FBB4F8D400FFF7E0FBB4F821
:103C00006601FFF7DCFB0020FFF7A6FB0020FFF7B3
:103C1000A3FB0020FFF7A0FB94F81301FFF79CFB28
:103C200094F82001FFF798FB0020FFF795FB3A4B33
:103C30001B68B3F956000A2390FBF3F080B2FFF73C
:103C4000BEFB94F80801FFF787FB94F80C01FFF71F
:103C500083FB94F80B01FFF77FFB94F80D0109E556
:103C60002D4C0420FFF7A8FB2368B3F85A00FFF798
:103C7000A6FB2368B3F8580017E60C20FFF79CFB5F
:103C80002C4B1868FFF7A4FB2B4B1868FFF7A0FB21
:103C90002A4B186852E4264C0620FFF78DFBB4F837
:103CA000E800FFF78CFBB4F8EA00FFF788FBB4F8F4
:103CB000EC00FAE51E4C0720FFF77EFBB4F80E017E
:103CC000FFF77DFBB4F81001FFF779FB94F81201C0
:103CD000FFF742FBB4F81401E7E5154C0C20FFF7A1
:103CE0006BFB94F81E01FFF737FBB4F82801FFF7D0
:103CF00066FBB4F82401FFF762FBB4F82601FFF776
:103D00005EFB94F81F01FFF727FBB4F82A01FFF7C9
:103D100056FBB4F82C01C8E53C1600200000C84250
:103D200000007A4400002041F3D7000858D800086A
:103D300064080020E8F7FF1FECF7FF1FF0F7FF1FF4
:103D4000554C0420FFF738FB94F86401FFF704FB9F
:103D500094F86501FFF700FBB4F86601A5E54F4C48
:103D6000002620784E4D00EB4000C0B2FFF724FB48
:103D7000237802359E42BFF48BAC15F8020CFFF796
:103D8000EBFA15F8010C013600EB800000EB800027
:103D900000F2EE2080B2FFF712FBE9E70820FFF700
:103DA0000BFB00243C4D631993F816010134FFF717
:103DB000D3FA082CF7D16BE4374C1020FFF7FCFA4C
:103DC0006079FFF7C9FAA068FFF702FB94F81E01BB
:103DD000FFF7C2FAB4F8E800FFF7F1FAB4F8EA0026
:103DE000FFF7EDFAB4F8EC00FFF7E9FAB4F80E01CA
:103DF000FFF7E5FAB4F8100157E52A4D264C95F87F
:103E0000680004F11006C0EBC000C0B2FFF7D4FA9E
:103E100094F9780195F96C30834225D095F9783082
:103E2000834221D00834A6423FF432ACF0E70D20A3
:103E3000FFF7C2FA0020FFF78FFA0020FFF7C8FA59
:103E40000020FFF7C5FA57E54E68304604F000FC45
:103E50000346BBF1000F7FF4B2AE3546B7E6087AF1
:103E6000FFF77AFAFFF7CFBBC0B2FFF775FAB4F8E5
:103E70007A01FFF7A4FA94F87C01FFF76DFA94F841
:103E80007D01FFF769FA94F87F01FFF765FA94F86E
:103E90007E01FFF761FAC5E764080020840D002069
:103EA0009209002094070020F7B50546144C0E46F1
:103EB00094F96C001146A8421A469DF824709DF8AA
:103EC000203011D094F97800A84217D0002013E0D8
:103ED0000C48009700F0FFFF70B10571267260601A
:103EE0000AE000970848F5E76C34207A0028EDD105
:103EF000002DEDD0012DF4D003B0F0BD7834F4E7FF
:103F0000940700200038014000440040F0B500252F
:103F10000E4B0F4C196894F88430DAB2012A04D998
:103F20000DB184F884200020F0BD5E1CDB00CF18AA
:103F3000BF8801320742D2B24FF0010504D00233EC
:103F400084F88420C818F0BD3346E6E75C160020EC
:103F500094070020084BDA68D10709D4DA685207C1
:103F600008D4DB6813F0100F14BF0320042070473F
:103F700001207047022070470020024003788B42E6
:103F800086BF024B33F81100002070472008002044
:103F900070B5054603F054FE294CA369A061C31A0D
:103FA000B3F5FA5F82BF002323776377237F1BB9C2
:103FB000A12D04BF01226277627F22B1E218EDB227
:103FC000013395772377227F94F83F309A4208D1C6
:103FD00094F84030052B05D0062B06D000236377DC
:103FE000237770BD002002F02BFAE37F1E2BF5D162
:103FF0000025294694F83F20013AEBB2934207DBB3
:104000002244937F9942E9D1032002F019FAE5E7AF
:10401000082023449B7FDBB281EA030616F0010FE0
:104020004FEA530300F1FF300CBFDBB283F08C0387
:1040300010F0FF00C1F34701EED101351946DCE76E
:10404000200800200C4B0D49DB68DB43C3F302233F
:10405000C3F104024378934002781B018818DBB255
:1040600080F800330123500902F01F0203FA02F224
:1040700041F82020704700BF00ED00E000E100E0C3
:1040800073B505460124002601220021006803F0D3
:1040900019FA2A6801A813889BB243F00103138020
:1040A000EB7A8DF805408DF804308DF806608DF8B8
:1040B0000740FFF7C7FFEB7A1B2B0BD1192301A891
:1040C0008DF804308DF805408DF806608DF80740B6
:1040D000FFF7B8FF02B070BD10B50F4C12220021DF
:1040E00004F5DD7009F047FA05230421012284F864
:1040F000C03184F8C23184F8C83184F8CA315223FF
:1041000084F8C11184F8C42184F8C91184F8BA3143
:10411000A4F8BE2110BD00BF200800200C4B03F501
:104120008A72C3F85825C3F85C1500F15003027871
:104130001AB98178C278914208D304309842F6D1F6
:104140000023044A83F00103137070470123F8E74A
:10415000200800202800002007B51C4B03F2645201
:10416000C3F8602593F862212AB3012A0AD10321FA
:1041700083F86615072183F868250C2283F86715F4
:1041800083F86425124A134B40205A6003F096FAD4
:1041900070B10122002390F9000040218DE80C004D
:1041A0004FF4E1330C4AFFF77FFE003018BF0120C7
:1041B00003B05DF804FB022183F86615032183F840
:1041C000682583F867150722DAE700BF200800207A
:1041D0000962000828000020C162000800210120B7
:1041E000FFF7CCB870B5CF4DAB68013B062B00F2A2
:1041F000C481DFE813F007007600A400FA00240170
:1042000045019B010126C84C3046D4F86C35A4F812
:104210006A6543F00803C4F86C3503F055FF40F2BB
:10422000A363B4F976259A4240F3A781B4F8943594
:10423000B3F5AF7FC0F0A181D4F86C3583F00803EB
:10424000C4F86C35B4F89635052BB4F99A3508BF27
:10425000A4F89665642B32DCB4F89835FA339BB237
:10426000B3F5FA7F2BD85522D4F89C355A710B231D
:10427000A4F8963540F26B73B4F976259A4240F370
:104280007C81D4F8A035952B40F37781012003F091
:104290000CFF40F24C43A4F876354FF47A73A4F83F
:1042A00072350223AB60B4F89635022B02D103239A
:1042B000A4F89635D4F8A435C4F8A83570BD40F2FA
:1042C0006B739A4240F35981D4F8A035772B40F3B1
:1042D00054810523AB60B4F89635022BEAD1042350
:1042E000E6E70226904C0120D4F86C35A4F86A6504
:1042F00083F00803C4F86C3503F0D7FE40F24C435A
:10430000A4F876354FF47A73A4F87235B4F99A3577
:10431000B3F5E17F02DD0323AB60CBE7D4F8A4352E
:10432000D4F8A825AE609B1AB3F5FA6FC0F02581CA
:1043300001230022AB607C4BC3F8A82570BD03238A
:10434000794CA4F86A35B4F99A352646B3F5E17F7D
:1043500019DDD4F86C35012083F00803C4F86C35FE
:1043600003F0A3FE40F24C43A4F876354FF4D26339
:10437000D4F8A825A4F87235D4F8A4359B1AB3F55F
:10438000FA6FD5D270BD9BB2B3F5E17F00F2F58034
:10439000B4F89835FA339BB2B3F5FA7F00F2ED80AA
:1043A000D4F86C35012043F00803C4F86C3503F0F1
:1043B0008BFEB4F89435B3F5B97F40F2DC5388BF77
:1043C000A4F87635A4F87235D4F8A43598BF40F235
:1043D000A462C4F8AC354FF0040398BFA4F8762566
:1043E000AB600523A6F8963570BD04264E4C01201F
:1043F000D4F86C35A4F86A6543F00803C4F86C354A
:1044000003F062FE4FF4FA63A4F8763540F2DC5311
:104410004B22A4F87235D4F89C355A71D4F8A435DF
:10442000D4F8AC259B1AB3F57A7F01D8AE6070BD85
:104430000123AB600523A4F8963500233CE705264D
:10444000394C0120A4F86A6503F02FFE40F24C437A
:10445000A4F876354FF4FA63A4F87235B4F99A35B6
:1044600013F5E17F01DA062356E7D4F8A435D4F832
:10447000A825AE609B1AB3F5FA6FBFF459AF70BDB3
:104480000623294CA4F86A35B4F99A35264613F563
:10449000E17F1ADAD4F86C35012083F00803C4F800
:1044A0006C3503F002FE40F24C43A4F876354FF42D
:1044B000A563D4F8A825A4F87235D4F8A4359B1ABE
:1044C000B3F5FA6FBFF434AF70BD03F5E1739BB27F
:1044D000B3F5C87F51D8B4F89835FA339BB2B3F529
:1044E000FA7F4AD8D4F86C35012043F00803C4F8A9
:1044F0006C3503F0E9FDB4F89435B3F5B97F40F2BB
:10450000DC5394BF40F2A462A4F87635A4F8723567
:10451000D4F8A43598BFA4F87625C4F8AC350723A1
:104520005EE700BF28000020200800200726134C6B
:104530000120D4F86C35A4F86A6543F00803C4F888
:104540006C3503F0C1FD4FF4FA63A4F8763540F200
:10455000DC534B22A4F87235D4F89C355A71D4F848
:10456000A435D4F8AC259B1AB3F57A7F7FF65EAFFD
:104570000123AB600523A4F8963570BD2008002008
:104580001F4A10B5536803F00C03042B21D0082BED
:1045900022D01C4B036053681B49C3F30313CC5C4C
:1045A0000368E34043605468C4F302240C5D23FABB
:1045B00004F484605468C4F3C2240C5DE340C36017
:1045C0005268C2F3813211440A7CB3FBF2F30361F7
:1045D00010BD0E4BDB68DDE753685168C3F38343BE
:1045E000C90303F1020302D409494B43D2E75168DE
:1045F00011F4003F0549C96818BF4908F5E700BF35
:104600000010024000127A0024D800082800002080
:1046100000093D0010B50446FFF79CFC012806D1B7
:104620000CB9052010BDFFF795FC013CF6E7002C06
:1046300008BF052010BD8B6810B50C6A02682343C3
:104640000C6922F4FF4223434C6922F07002234399
:104650008C692343CC6923434C6A23438C6A2343EC
:1046600013430360CB6843600B6883604B68C3608F
:1046700010BD036823F001031B041B0C036000231F
:10468000036043608360C360284B984204D1284A8A
:10469000536843F00F0326E0264B984204D1244A86
:1046A000536843F0F0031EE0234B984204D1204AA4
:1046B000536843F4706316E0204B984204D11C4ABF
:1046C000536843F470430EE01D4B984204D1184ADE
:1046D000536843F4702306E01A4B984205D1144AFC
:1046E000536843F4700353607047174B984204D1EA
:1046F0000F4A536843F07063F5E7144B984201D1B9
:10470000134AC5E7134B984201D1114AC8E7124B2F
:10471000984201D10E4ACBE7104B984201D10C4A86
:10472000CEE70F4B9842DFD1094AD1E7080002409B
:10473000000002401C0002403000024044000240E1
:10474000580002406C000240800002400804024011
:10475000000402401C0402403004024044040240B1
:10476000580402400F4B1A6842F001021A6059685F
:104770000D4A0A405A601A6822F0847222F480328C
:104780001A601A6822F480221A605A6822F4FE0223
:104790005A604FF41F029A604FF00062034B9A6018
:1047A000704700BF001002400000FFF800ED00E07D
:1047B0002DE9F8435B4C0368023AC4F8B0358388AE
:1047C0000D46A4F8B435062A05D8DFE802F0767D58
:1047D000848B969CA300B4F8B0350B80B4F8B23546
:1047E0006B80B4F8B435AB804F4B1B7C002B62D18F
:1047F000B5F9000004F09EFC8046B5F9020004F013
:1048000099FC0746B5F9040004F094FCD4F8B815F7
:104810000646404604F0E2FCD4F8C415814638460A
:1048200004F0DCFC0146484604F0D0FBD4F8D01577
:104830008146304604F0D2FC0146484604F0C6FBEF
:1048400007F056FCD4F8BC152880404604F0C6FC9E
:10485000D4F8C8158146384604F0C0FC01464846E5
:1048600004F0B4FBD4F8D4158146304604F0B6FC0D
:104870000146484604F0AAFB07F03AFCD4F8C015FC
:104880006880404604F0AAFCD4F8CC15804638462F
:1048900004F0A4FC0146404604F098FBD4F8D81577
:1048A0000746304604F09AFC0146384604F08EFB79
:1048B00007F01EFCA880BDE8F883B4F8B2350B8081
:1048C000B4F8B0355B428BE7B4F8B0355B420B808F
:1048D000B4F8B235F6E7B4F8B2355B420B80B4F801
:1048E000B0357DE7B4F8B0355B420B80B4F8B23533
:1048F0006B80B4F8B4355B4275E7B4F8B2350B8021
:10490000B4F8B035F4E7B4F8B0350B80B4F8B2358C
:104910005B42EDE7B4F8B2355B420B80B4F8B035DA
:10492000F6E700BF200800202800002040F2AD126A
:1049300040F6FF714243B2FBF1F244F6FB710A4BC1
:10494000A3F89425D3F8DC25137803EB431300FB7D
:1049500003105378C3EB0333B0FBF3F09378B0FB51
:10496000F3F080B2704700BF200800202DE9F74F18
:10497000794C94F8E13504EB4303B3F8F085B4F9CE
:1049800002361FFA88F80A2B1CBF002384F8003671
:1049900094F80036A4F8F885002B61D16F4B4FF0E6
:1049A0009749C4F80436C4F80C364FF07E53C4F867
:1049B00010366B4B4FF0000AC4F81436694B4FF0B9
:1049C0007C57C4F8183640F2DC53C4F85436102330
:1049D000A4F852361823644D644AA4F85036C4F83B
:1049E0000826EE1805F1300B4946286904F0F6FB5D
:1049F0005146019004F090FD019B3946002800F0DB
:104A0000A380184604F0E0FA04F05AFEC6E9080153
:104A1000494655F8040F04F0E1FB5146019004F0BB
:104A20007BFD019B3946002800F09280184604F077
:104A3000CBFA04F045FEE6E902015E45D4D10A2333
:104A4000A4F80236A8F2DC531B04C4F87036C4F88C
:104A50007C36C4F87436C4F88036012384F80036F6
:104A6000414BD4F854A6B4F95256A8EB0A005A6A3E
:104A700000FA05F14A43186A4FEAE179D4F87076F2
:104A800000FB0922C4F87016A0FB0101D4F87C6673
:104A900011445A6CD3F8408072434FEAE67908FB20
:104AA0000922A8FB06899144DA6AD4F880C67A43C1
:104AB000B0EB0800C4F880669E6A61EB09014FEA1A
:104AC000E779D4F874E606FB0922C4F87476A6FBED
:104AD00007671744DA6C36180CFB02F2986C4FEA41
:104AE000EC794F4100FB0922A0FB0C01301A7646FD
:104AF000114467EB0101F7171E6B5B6BC4F878E696
:104B00000EFB03F306FB0733A6FB0E671F44801959
:104B1000C4F884C6B4F95026794103F0A1FD0123FD
:104B20006A1E9340C4F87C06C01841EBE3712A4624
:104B300003F096FD10EB0A0080B2FFF7F7FEA4F831
:104B4000880603B0BDE8F08F184604F03FFA5BE733
:104B5000184604F03BFA6CE72008002056157D3912
:104B60006350FABF0CE0743F200E00205615FD394B
:104B7000F8B53C4C0546B4F88A36322B4ED1D4F801
:104B80008C361A88A4F890265A889B88A4F8922616
:104B9000A4F894360388A4F896364388A4F8983687
:104BA00000231946304AD4F88CE602F10C06B4F81A
:104BB0008A069F00322808BF42F8231036F913C036
:104BC000D05926F813106044D0512EF81310013339
:104BD000032BECD1B4F88A36012B19D14FF0000227
:104BE0000C2084F8AE2684F8AF3602F011FED4F81B
:104BF0008C36B4F890261A80B4F892265A80B4F80D
:104C000094269A80B4F896362B80B4F898366B8048
:104C1000B4F88A36013BA4F88A3601E0002BBFD1F4
:104C200094F8B036EBB13220D4F89C36002293FBD6
:104C3000F0F3D4F88C1684F8B0260B80D4F8A036A4
:104C400093FBF0F34B80D4F8A43693FBF0F30748C2
:104C5000408A1B1A8B802A806A80BDE8F84003F0E6
:104C6000BBBCF8BD20080020BC0E0020280000209E
:104C700010B5046B0346C168406944B11A6C8C1AC4
:104C8000013A08BF0A46005D1A64C0B210BD1A6A34
:104C9000805C01328A4228BF2246C0B21A6210BD2F
:104CA000436B13B190F844007047836A406A1B1A43
:104CB000584258417047416A826A0369914238BF3D
:104CC000C9188A1A416B21B149680A44591E8A429F
:104CD00003D2581E801AC0B2704700207047036B81
:104CE0005BB15B68026C9342A3EB020301D3D8B2C1
:104CF0007047C0681844C0B27047C369026A9342E3
:104D000037BFC068981AC018801AF4E770B5054616
:104D1000046D8668A38986B023F400531B041B0C22
:104D2000A3818379697913F0020F14BF4FF4005205
:104D3000002213F0040F14BF4FF48060002011F024
:104D4000010F14BF042300238907218A48BF43F0C1
:104D5000080389B221F4405111432182A28922F42F
:104D6000B05222F00C021204120C02431343A3812E
:104D7000A28A01A822F440721204120CA282FFF748
:104D8000FFFB204A039B0499944218BF194619223D
:104D9000A3894A4313F4004F14BF7100B100B2FB62
:104DA000F1F16426B1FBF6F3A2891801120406FBA7
:104DB00013131FD5DA003232B2FBF6F202F007020B
:104DC00042EA00039BB22381AB792A6D13F0080FEE
:104DD000938A0BBF23F008039BB21B0443F0080324
:104DE00008BF1B0C938293899BB243F400539381B9
:104DF00006B070BD1B013233B3FBF6F303F00F03B3
:104E00000343DFE70038014041717FE781607DE7C0
:104E1000026D70B515880446ADB2A90606D5036BC0
:104E200023B9C36AA3B1908880B298472B0620D5D6
:104E3000636AA26A9A42236D17D0511CA069A162CD
:104E4000825C9A802369994213D30023A36270BDC8
:104E5000E169928840694E1CD2B2E6614254E16930
:104E6000E268914228BFE361E0E7DA6822F080025D
:104E7000DA6070BD836A8169426B1944D160416A0E
:104E80008B4229BF0169CB1ACB1A53602ABF00237A
:104E9000536083624FF0000380F84430136838BFDA
:104EA000816243F0010313607047436A8269D15401
:104EB000436A02690133934228BF00234362436B74
:104EC0001BB11B68DB0705D4D4E7026DD36843F040
:104ED0008003D36070472DE9F0431E469B4B8DB095
:104EE0009842894690469DF8507040F0CE80984B8D
:104EF000984AC3F808801A60974A18655A6102F503
:104F000080729A614FF48072DA601A61934A5A6330
:104F1000A2F54842403A9A64914B9A6942F4804221
:104F20009A615A6942F001025A6102238DF80330F6
:104F30004FF400733A07ADF8003040F194801C2321
:104F4000694688488DF80230FCF766FD01240E237F
:104F5000002501A88DF804308DF805408DF8074034
:104F60008DF80650FFF76EF8252301A88DF805404F
:104F70008DF807408DF804308DF80650FFF762F881
:104F8000734C00250123256284F84430E561A56255
:104F90006562C4F82C906671C4F80880A771204639
:104FA000FFF7B4FEF20729D5206B002800F0BC8083
:104FB000E36C039501934FF480530A938023069387
:104FC000E368059504932023099363690795029389
:104FD00008950B95FFF74DFB01A9206BFFF72BFB05
:104FE000226B216D136843F0010313608B8A9BB21F
:104FF00043F040038B8253689BB22364B30728D5E8
:10500000606B002800F09980A36C002501934FF499
:1050100080530A93802306932369029504931023F7
:10502000059503930795089509950B95FFF721FBC7
:1050300001A9606BFFF7FFFA636B1A6842F0020286
:105040001A60226D5D605D60938A9BB243F08003BD
:1050500093822046226D93899BB243F4005393813F
:105060000DB0BDE8F083B30706D5182369463D4867
:105070008DF80230FCF7D0FCF5077FF567AF4FF4F1
:105080008063ADF8003048235AE7374B98425AD135
:10509000364B304AC3F808801A604FF48072DA60E9
:1050A0001A61334A18655A6102F580729A61314A71
:1050B0003C079A64DA642A4BDA6942F40032DA6116
:1050C0005A6942F001025A614FF002038DF8033031
:1050D0004FF00403ADF8003016D51C236946214873
:1050E0008DF80230FCF798FC262300228DF804305E
:1050F000012301A88DF805308DF806208DF80730C2
:105100001A4CFEF79FFF3CE7B00706D51823694607
:1051100014488DF80230FCF77FFCF107E4D5082332
:10512000ADF800304823D9E74FF6DF72236D1A80BF
:10513000DA6842F02002DA6060E7226DD36843F05B
:105140008003D36085E700208AE700BF0038014074
:10515000A81700203CD80008D10E002044000240CF
:105160000010024000080140004400405417002095
:10517000D11000200444004010B57C4B1B78012B5B
:1051800014BF00240324038C002938D123F0010329
:105190001B041B0C0384018B038C89B221F0F301E7
:1051A00041F0010141EA0411714C9BB2A04242F06E
:1051B000010212D004F50064A0420ED0B0F1804F7D
:1051C0000BD0A4F59834A04207D004F58064A04227
:1051D00003D004F58064A0420ED123F002031343F0
:1051E00001830384038B23F00C031B041B0C038338
:1051F000038B9BB2038310BD23F00A03EFE704295E
:1052000038D123F010031B041B0C0384018B038C87
:1052100021F440710905090D41F4807141EA04311E
:10522000534C9BB2A04212D004F50064A0420ED0B1
:10523000B0F1804F0BD0A4F59834A04207D004F50C
:105240008064A04203D004F58064A0420CD123F016
:10525000200343EA021292B242F010020183028458
:10526000038B23F44063C0E723F0A00342F0100255
:105270001A43F3E708293DD123F480731B041B0C68
:105280000384818B038C89B221F0F30141F0010189
:1052900041EA0411364C9BB2A04212D004F50064DE
:1052A000A0420ED0B0F1804F0BD0A4F59834A042AC
:1052B00007D004F58064A04203D004F58064A042C6
:1052C00012D123F4007343EA022292B242F48072B4
:1052D00081830284838B23F00C031B041B0C8383C8
:1052E000838B9BB2838310BD23F4206342F48072CE
:1052F0001A43EDE723F480531B041B0C0384818BBA
:10530000038C21F440710905090D41F4807141EAD3
:105310000431174C9BB2A04212D004F50064A042A5
:105320000ED0B0F1804F0BD0A4F59834A04207D036
:1053300004F58064A04203D004F58064A0420CD13F
:1053400023F4005343EA023292B242F48052818342
:105350000284838B23F44063BFE723F400735B0470
:105360005B0C42F480521A43F1E700BF880400202E
:10537000002C01402DE9F04F87B00493854B074680
:105380001B8802929C0740F1D78040F2E6328248A7
:10539000109BDD89B0F900305B1B03F2F3149442DB
:1053A00004469CBF83EAE370A0EBE37040F2E6336F
:1053B000B4F9022088BF4FF4FA70521B02F2F314C2
:1053C0009C4200F2B68082EAE273A3EBE27383426E
:1053D000B8BF03460522C3F5FA7393FBF2F30A2222
:1053E000643B5A433B7FDB105343642293FBF2F34D
:1053F000134423EAE3735BB200244FF06408DFF840
:10540000BC9100930B1D019309F1100B019B6100EE
:1054100013F8012B022C01930391604B40F08E8016
:10542000B3F904501B3255436D115D4B62009B5E16
:10543000042293FBF2F307EB040A9AF80160ED1AD9
:1054400005FB06F314F8096097F851205E4396FBBC
:10545000F8F6F61172B15349304601EB840105921A
:10546000039103F067FE059A039902F07FFC04F0B4
:1054700091F806464C4B9AF80B2018884B4905FBCF
:1054800000F3DB12534319F8042000095A4392FB3E
:10549000F8F25BF824304FEA840C1A44B2F5001F8E
:1054A000A8BF4FF40012424B9A42B8BF1A4653139A
:1054B0004BF824204FF6FF72B2FBF0F0039351F843
:1054C000243001F10C02EB1A434341F8245001F15E
:1054D000180552F824E09B1155F8240042F82430B6
:1054E00097F850207044184445F824E05AB124310C
:1054F00001EB0C05059203F01DFE059A294602F00A
:1055000035FC04F047F89AF815306200434319F867
:1055100004000134584390FBF8F0039B032C1E4415
:10552000244B06EB20269E527FF470AF07B0BDE8F7
:10553000F08F4FF4FA734DE764235DE733F91450AD
:10554000029B69005B42994203DB029B8B42A8BF2E
:105550000B4619496000095E5B1A049931F9141071
:1055600019440C4B1B88D8070FD41B3255439B079B
:105570004FEA25157FF559AFBB7C009A4B43534347
:1055800093FBF8F305EB23154FE73D7A4D432D11BF
:105590004BE700BFA0070020900D0020D412002090
:1055A000C4070020E012002054180020F812002048
:1055B0000000E0FF28130020B80D0020DC120020BE
:1055C0002DE9F04FB54D89B00492B5F9002006934E
:1055D000B5F90230002AB8BF5242002BB8BF5B4277
:1055E0009A42B8BF1A460027B2F5FA7F1346A8BF01
:1055F0004FF4FA7380463C46059100930297039757
:10560000019705F1180AA64B198811F0030C40D038
:1056100035F91420049B52005B429A424FEA44063B
:1056200003DB049B9342A8BF13469E4A6FF0040E0F
:10563000B25E64269B1A069A32F91420134498F835
:1056400008205A4392FBF6F298F81C600EFB06F015
:105650008242019005DB06EB86069642A8BF1646FD
:105660000196914E56F82420134442F21072934250
:10567000A8BF13468D4A9342B8BF134698F812202C
:1056800046F824305343BCF1010F4FEA2333039310
:1056900034D035F914300293854B33F9142082EA63
:1056A000E273A3EBE273B3F5206F00F3E6805023BF
:1056B0000298434308EB0400407893FBF0F3042086
:1056C00092FBF0F29B1A5AF824201344B3F57A5F48
:1056D000A8BF4FF47A53774A9342ACBF4AF82430BC
:1056E0004AF824207D235AF8247008EB040297FB23
:1056F000F3F3D77A5F43402397FBF3F78A0740F130
:10570000C0804FF4FA76009B0299C3F5FA7203FB4E
:1057100001F90099019B7943039803FB029900FB6F
:10572000021299FBF6F392FBF6F662000792604ACA
:10573000614932F91490042299FBF2F214F80190B5
:1057400009FB02F96FF04F0299FBF2F998F851202A
:1057500099446AB1583901EB840B4846079203F02B
:10576000E9FC079A594602F001FB03F013FF81465A
:1057700004204F4B6200D15E504B4FEA840BD25E47
:1057800003F1040E8A1A92FBF0F203F10C0C600094
:10579000C1525EF824105CF824004EF8242008441E
:1057A000104498F850204CF8241052B1203B9B44F0
:1057B000079203F0BFFC079A594602F0D7FA03F0AC
:1057C000E9FE3F4B4E4403F1280212F804906200B8
:1057D00000FB09F04FF0200990FBF9F00134301A7A
:1057E000022CD0527FF40FAF0421059B9A790F321F
:1057F0005300B5F904205A432D4B5211B3F904302C
:10580000002A93FBF1F3A2EB0303B8BF5242322A02
:105810003EDC296A98F80D2003FB021229498A42CE
:10582000A8BF0A4628498A42ACBF2A62296298F872
:105830000320534395F87F209B11032A0AD9B8F817
:105840004E20B2F5FA7F05D251428B4223DB9342C0
:10585000A8BF13462A6A6FF0FF0142F34F32B2F538
:10586000807FA8BF4FF480728A42ACBF9B185B1840
:10587000A5F8583009B0BDE8F08F00234AF824306D
:1058800030E7CB0759BF3E46029B039E019B4CE786
:1058900000222A62CBE70B46DCE700BFD4120020CF
:1058A000A0070020B80D002030130020F0D8FFFF23
:1058B000C407002080C1FFFF381300203C130020E4
:1058C00028130020FEFFFF0F020000F02DE9F04F2B
:1058D000054690F850008BB0089105920993002876
:1058E00000F0BD803228A8BF322003F023FC01461F
:1058F000614803F027FD0446604B1888002808BF64
:10590000012003F017FC5E49069003F067FC014696
:105910000090204603F05AFB0146009803F012FD68
:10592000584B07901B88980740F1A080564AB2F95F
:105930000030B2F9020083EAE37180EAE072A1EB81
:10594000E371A2EBE07291420C46B8BF1446B4F585
:10595000E17F80F28D80914280F283800028D8BF61
:10596000404203F0E7FB494903F0ECFC07464FF0E7
:1059700000090024444ECDF8049063000293444B88
:1059800033F914301846049303F0D4FB414903F073
:1059900025FC03F0FFFD03F0CDFB3F4903F01EFCA7
:1059A000029036F9140003F0C5FB364B80461B8885
:1059B0009907039300F08E80014603F007FB03F084
:1059C000E9FD059B5B42984203DB059B8342A8BF30
:1059D0000346324A6100885E099A1B1A32F91400A4
:1059E000184403F0A7FB8246287F03F09FFB2C4955
:1059F00003F0F4FB8346287A03F098FB514603F04A
:105A0000EDFB284903F0EAFB03F0C4FD81460BF1EE
:105A1000004003F0BFFD814505DB584603F0BAFDA9
:105A20004845A8BF484603F085FBDFF888905146FB
:105A30000190009803F0D2FB59F8241003F0C6FA45
:105A400019494FEA840B824603F066FDA0BB174953
:105A5000504603F07FFD88B3DFF850A02EE0144CD1
:105A60004AE7002BCCBF184658427AE700277EE76A
:105A70004FF07E577BE700BF83F9223E5418002089
:105A8000BD378635A0070020D41200200000E14376
:105A9000C40700200000A03ECDCC4C40B80D002033
:105AA0000000A0406F12033C0000F0C10000F04174
:105AB000AF4C593C54130020DFF8F0A249F80BA07A
:105AC000A87C03F033FB514603F088FBA94903F09F
:105AD00085FB8146039BDA0700F12481049B002BA0
:105AE000B8BF5B42B3F5206F4FEA8403049340F3E1
:105AF000ED800022A04B43F824202B19D87A03F024
:105B000015FB9D4B53F8241003F068FB9B4903F0F1
:105B100065FB039B82469B0715D50199404603F020
:105B200053FA394603F05AFB019903F04FFA4946FC
:105B30008046504603F048FA394603F04FFB494689
:105B400003F044FA8246DFF868B21BF8040003F061
:105B5000F1FA029903F042FB894903F03FFB014649
:105B6000404603F031FA95F85120034632B1ABF1CB
:105B7000580101EB840102F0F9F803460393814BCD
:105B8000029853F8241003F01FFA009903F0DAFB8F
:105B90007C4B029A03F1080858F824B043F82420FB
:105BA000594603F011FA079903F018FB594603F020
:105BB0000DFA039B48F8240051468346184603F02B
:105BC00005FAA8F120020290105D03F0B3FA5946DD
:105BD00003F004FB6C4903F001FB029B01461846ED
:105BE00003F0F2F906F084FA63000134A8F14808E2
:105BF000022C28F803007FF4C0AE069803F0CAFC1C
:105C000020F0030003F096FA604903F09BFB089B29
:105C100095F853800446DFF89C91B6F904709B799F
:105C2000B8F1000F00F0C88087EAE778A8EBE778C2
:105C300008FB03F0564B90FBF3F0EB7864305843CD
:105C4000642390FBF3F003F075FA0090B9F90400B7
:105C500003F070FA4FF07A5103F0C0FA06F048FAF8
:105C6000834603F067FA009B194603F0B7FA4949E7
:105C700003F068FB8146384603F05CFA494603F0BE
:105C8000A3F98BEAEB73A3EBEB73B3F5207F8146AB
:105C900002DCB8F1640F49DD0023336295F851202E
:105CA00022B148463C4902F061F8814651464846D7
:105CB00003F08CF903F06EFC00B203F03BFA06F03F
:105CC00017FAA6F858000BB0BDE8F08F33494046EC
:105CD00003F084FA2B198246587803F027FA01461C
:105CE000504603F02FFBDFF890A0029903F06CF907
:105CF000009903F073FA5AF8241003F067F9284961
:105D0000834603F009FC38B92649584603F022FCC3
:105D100020B1DFF890B001E0DFF884B0A3004AF8CA
:105D200003B0EAE6CA46DDF804800CE7502047439A
:105D3000E87897FBF0F0A0EB0B0003F0FBF92146AD
:105D400003F04CFA03F026FC336A1844B0F57A5F8E
:105D5000A8BF4FF47A50144B9842B8BF18467D2321
:105D6000306290FBF3F06B7B5843801103F0E2F953
:105D7000824693E70AD7A33D5C1300200AD7233C51
:105D8000A69B443B68130020F7CC923800803B452B
:105D90000CFEFFFF0000A042E81200200000A0431C
:105DA000000040C30000404380C1FFFF0000F0C17D
:105DB00038130020C40700205B002833B9F9040021
:105DC0005F4303F0B7F94FF07A5103F007FA06F09A
:105DD0008FF97F11381A03F0ADF9002FB8BF7F4259
:105DE000322F814632DDC6F82080336A6FF0FF0023
:105DF0005B13B3F5807FA8BF4FF480739842B8BFA0
:105E0000184603F097F98246484603F0C3FBEB7847
:105E10005843801103F08EF996F87F308146032BAA
:105E20007FF63CAFB5F84E40B4F5FA7FBFF436AF1D
:105E300003F0B0FB6342984203DBA0420346A8BFD5
:105E40002346184603F076F9814627E7687B03F07E
:105E50006DF9494603F0C2F9214603F0BFF903F09A
:105E600099FB336A1844054B9842A8BF1846044B67
:105E70009842ACBF30623362B7E700BFFEFFFF0F4E
:105E8000020000F02DE9F74F264C0025A046264FD2
:105E900094F87F60E8B2B04211D3244B1B685B03D7
:105EA0000AD500244FF0500921464FF0280AA34696
:105EB0001F4FE3B29E420FD803B0BDE8F08F04EB52
:105EC0008003D3F8A4302BB10B2803D8DB6837F854
:105ED000101098470135DBE757F82430A2005D68C1
:105EE0008D4217D02846019201F040FBEFF3128358
:105EF00089F31288A98C0AFB008089B20131C0F8AD
:105F0000F810A98ADBB289B241F00101A98283F3BA
:105F10001188019ABB5801341B682946A3F800B0C8
:105F2000C7E700BFD4120020D007002000160020D1
:105F3000781300200F4B10B51B680F4C13F4805FD3
:105F40000E4B14BFD3F87421D3F8782193F87F1047
:105F50000023B2F90420D8B2884206D3FFF792FF9B
:105F6000BDE81040322001F092BE24F81320013326
:105F7000F1E700BF00160020D0070020D412002057
:105F80002DE9F047304E0446D6F87C512F4928467B
:105F900003F01CF801F040FF8046284601F03CFF6A
:105FA000D6F8806105462949304603F00FF801F024
:105FB00033FF8246304601F02FFF2168814650466C
:105FC00003F00CF96768A66839460446284603F0D2
:105FD00005F9494603F002F90146204602F0F6FFB2
:105FE00031460446484603F0F9F8414603F0F6F816
:105FF0000146204602F0EAFF41460446384603F0D7
:10600000EDF831460746284603F0E8F801463846E1
:1060100002F0DAFF214606F0F5F80D4903F0DEF84C
:106020000C4903F08FF9002102F0D0FF0A4903F078
:1060300089F906F05DF803B2002BBCBF00F5B4701F
:1060400003B21846BDE8F087D4120020DB0FC93F29
:106050000000E144DB0F494000002041F0B587B06B
:10606000064603F063F84F4903F0B8F84E4C074674
:10607000D4F87C314D4D03F100430393D4F88031C3
:1060800003F1004304934A4BB3F9000003F052F8C4
:10609000484900F1004003F0A1F80590B5F900006F
:1060A00003F048F80090B5F9020003F043F80190BE
:1060B000B5F9040003F03EF803A90290684601F028
:1060C000A1FFD4F884315B78012B67D13A4B1B7860
:1060D0005B070ED44023D4F8880190FBF3F3C01A79
:1060E00003F028F8029902F071FF03F053FAC4F8A4
:1060F00088014023D4F8880190FBF3F003F01AF8EC
:106100000146029802F060FFD4F8901102903846E0
:1061100002F05CFF0146384603F014F9D4F88C51C4
:1061200007462946029802F04FFF0146384603F021
:1061300055F8294602F04AFF0746C4F88C0100983A
:1061400005F0D6FFD4F89451297801F056FED4F822
:1061500098311844C4F89801019805F0C9FF2978CE
:1061600001F04BFED4F89C311844C4F89C01384629
:1061700005F0BEFF697801F040FED4F8A031184464
:10618000C4F8A001D4F8A831D4F8A40101333044F4
:10619000C4F8A401C4F8A83107B0F0BD074B1888B3
:1061A000ACE700BFBD378635D4120020BE07002003
:1061B000E807002035FA8E3C341600203A00002013
:1061C00001380A4B042804D8DFE800F006080A0C5E
:1061D0000E00074A1A607047064AFBE7064AF9E7CD
:1061E000064AF7E7064AF5E7064AF3E73C000020CF
:1061F0003526000875530008B528000889230008D3
:10620000C1550008CD58000803788B420AD9064BC7
:106210001A78064B53F8210002B1400800F5777058
:1062200080B2704700207047880D00208014002045
:1062300007298FBF0020034B03EB8101086B80B25D
:10624000704700BF80140020034B03EB4101B1F8FD
:106250005000C008704700BF8014002008B5084BEC
:1062600003EB8101086F02F061FF064902F0B6FFFF
:10627000054902F0ABFE03F0B3F980B208BD00BFE0
:10628000801400200000203F00005C44024B03EB20
:106290004101B1F8B800704780140020024B03EBB5
:1062A0004101B1F8DC00704780140020024B03EB81
:1062B0004101B1F8DC0070478014002000207047D5
:1062C00010B5044601F0BCFC41F288310D4BE4B23C
:1062D000D3F8F420C3F8F400821A8A4284BF002263
:1062E00083F8F82093F8F8200F2A03EB02010CBF83
:1062F0000122013281F8F94014BF83F8F82083F8B5
:10630000092110BD8014002010B5044601F098FC4E
:1063100041F288310D4BD3F80C21C3F80C01821ADD
:106320008A4284BF002283F8102193F81021142A96
:1063300003EB02010CBF0122013281F8114114BFAD
:1063400083F8102183F8262110BD00BF801400209F
:1063500010B5044601F074FC254BD3F82821C3F88E
:106360002801821AB2F57A6F84BF002283F82C21AB
:1063700093F82C214AB9A82C38D183F82D21A3F801
:106380002E21991881F8314106E0022A02D183F8C2
:106390003041F6E7242AF4D993F830110132023162
:1063A000D2B249008A4283F82C2116DA082241F23F
:1063B0002101B3F82E01E4B280EA042010F4004F6A
:1063C00002F1FF324FEA400018BF484012F0FF02CE
:1063D00080B2F3D1A3F82E0110BD01318A4201BF72
:1063E000002283F82C21012283F82D2110BD00BF4B
:1063F0008014002010B5044601F022FC40F6AC5198
:106400000E4BD3F85821821A8A42C4BF002283F867
:106410005C2193F85C21991881F85D411AB90F2C21
:106420000BD1C3F858010132D2B2192A83F85C218A
:106430000CBF0122002283F8762110BD80140020B9
:106440000022F0B5234D13462C4641F221070826C1
:106450008118695C83EA012313F4004F4FEA43017A
:1064600006F1FF3618BF794016F0FF068BB2F3D164
:106470000132192AEBD100F11902A15C00F11A02D4
:10648000A25C02EB012292B29A420DD14FF4AF67A7
:106490001149334691F87751104E0130DAB29542E6
:1064A00003D8012381F87831F0BD00EB42025FFA96
:1064B00082FE14F80EC00EF1010E14F80E2002EB4D
:1064C0000C2292B27A43121302F5487226F8132076
:1064D0000133E3E73E08002080140020200800205C
:1064E000114910B5D1F87C3103EB4002147E2CB178
:1064F000022C0DD00D4B33F8100010BD022805D929
:106500000328F7D1D1F88021D2040AD5D88910BD4B
:10651000507E00EB800000EB800000F2EE2080B2A5
:1065200010BD4FF4966010BD80140020900D002027
:1065300008B501F085FB0222064B83F88821064A44
:10654000C3F884011268C3F89421012283F8AD21B5
:1065500008BD00BF80140020C40D002008B501F064
:106560006FFB0222074B00F5B71083F88821D3F8A0
:10657000942100F5587002F2DC52C3F88401C3F88C
:10658000942108BD801400202DE9F047CA4D8AB03F
:10659000D5F8B0212C4692F849304A2B00F02581DD
:1065A00076D8352B00F0BD8132D8292B00F0A4829B
:1065B00021D8252B00F07382272B00F07D82232B1E
:1065C00040F08B80FCF7B4FE1328064610D8D5F8AF
:1065D000BC510C27FCF7ACFE0023B84907FB0312A3
:1065E00092F808E0864500F0298301331C2BF5D191
:1065F000FDF7F4FDB7E02D2B00F09082332B00F077
:10660000D9822B2B69D1FCF793FEAD4B5871AAE0D0
:106610003E2B00F0E08028D8392B00F05B823C2B29
:1066200000F0E880372B58D107265379B3FBF6F2F8
:10663000C2EBC2029A1A12F0FF0FD9D1B3FBF6F6E1
:10664000013EF6B2FF2E00F08E80FCF771FED4F80A
:10665000DC5140B295F90230834200F0D98295F9BD
:106660000A308342C4D10A35D3E2432B00F0A8821A
:10667000442B00F0DF82412B2FD10024904DFCF7FA
:1066800057FE63190134082C83F81601F7D16AE02C
:10669000CF2B00F0A98122D8CA2B00F0B68014D8E5
:1066A0004E2B00F05F82C82B61D04C2B15D1FCF72C
:1066B0003FFE834C84F86401FCF73AFE84F86501E0
:1066C000FCF740FEA4F866014DE0CD2B00F0D1812F
:1066D00000F2D981CC2B00F04B81002029E0D42B93
:1066E00041D00BD8D22B27D039D8D02BF5D195F863
:1066F000B431580737D400F007FC2BE0EF2B5DD006
:106700000CD8D62BE9D1002405F5E075FCF71AFE6C
:1067100025F814000134082CF8D124E0F22B22D003
:10672000FA2BDAD195F8B4315B0713D5FDF756FD96
:1067300001200AB0BDE8F08795F8B43113F00404E5
:1067400011D1FCF7F5FD5E4B022894BF83F8EC04F1
:1067500083F8EC4401F020FD01F0C2FD03E0FCF7FA
:10676000F1FDA5F8B6010020FCF726FEE0E755791B
:106770006D08122D3FF63CAF002601AFAE420DD39F
:106780002A4600234F4901A89D420DDC00214D4BB4
:10679000122A0FD1012384F8B831E4E7FCF7D2FDC7
:1067A00027F816000136E9E730F8136021F8136086
:1067B0000133E9E723F812100132E9E7D5F8BC41CB
:1067C000FCF7C0FDA4F85A00D5F8BC41FCF7BAFDAF
:1067D000A4F85800C7E7FCF7ABFD394C84F86E010C
:1067E000FCF7A6FD84F86D01BDE7FCF7ABFD344B6B
:1067F0009881B8E7D5F8BC41FCF79AFD2070D5F830
:10680000BC311878FFF7DCFCADE7D5F8BC310025CA
:106810001B78022B6FD1DFF8B490DFF8B4802A4FD9
:10682000D4F8BC61FCF784FD02F080FC494602F01C
:1068300089FD05F1080A46F82A00D4F8BC61FCF786
:1068400077FD05F10A0306EB830602F06FFC414673
:1068500002F078FD7060D4F8BC61FCF769FD02F0CD
:1068600065FC394602F06EFD05F10E0A0135032D77
:1068700046F82A00D4D1154F072DD4F8BC6129D190
:10688000FCF756FD02F052FC394602F05BFD7064E5
:10689000D4F8BC61FCF74CFD02F048FC394602F02C
:1068A00051FDB064D4F8BC61FCF742FD86F84C00A1
:1068B00001350A2DE0D156E78014002058D8000891
:1068C000640800203815002000007A4400002041B0
:1068D0000000C842FCF72CFD2E447070D4F8BC6157
:1068E000FCF726FD2E44F072D4F8BC61FCF720FDC5
:1068F0002E447075DCE7D4F8BC61FCF719FD2E441A
:106900007070D4F8BC61FCF713FD2E44F072D4F81B
:10691000BC61FCF70DFD2E4401350A2D7075EAD1DE
:1069200021E7FCF705FD0B2804463FF661AED5F8DC
:10693000BC51FCF7FDFC03283FF65AAE062303FBCF
:10694000045484F8CE00FCF7F3FC84F8C900FCF78B
:10695000EFFC84F8CA00FCF7EBFC84F8CB00FCF7F2
:10696000E7FC84F8CC00FCF7E3FC84F8CD00FAE601
:106970005379092B7FF63CAEBC4D2E68FCF7D8FC52
:1069800030702E68FCF7D4FC7070FCF7D1FC6428E2
:10699000A8BF64202B681871FCF7CAFC6428A8BF44
:1069A00064202B685871FCF7C3FC2B689871FCF7C6
:1069B000BFFC642828BF64202E68F071FCF7B8FC87
:1069C000B0702E68FCF7B4FCF0702E68FCF7BAFCCF
:1069D000D4F8B03170815B790A2B7FF6C4AE2C6895
:1069E000FCF7A6FC2072BEE6FCF7ACFC6FF4AF65CA
:1069F00043199BB29E4DC62B98BFA5F82401FCF706
:106A0000A1FCA5F8D000FCF79DFCA5F8D200FCF78E
:106A100099FCA5F8D400FCF795FCA5F86601FCF7F5
:106A200087FCFCF785FCFCF783FCFCF781FC85F810
:106A30001301FCF77DFC85F82001FCF779FCD4F804
:106A4000BC41FCF77FFC00EB80004000A4F856003E
:106A5000FCF76EFC85F80801FCF76AFC85F80C0170
:106A6000FCF766FC85F80B01FCF762FC85F80D016C
:106A700079E695F8B43159073FF575AE4FF4C87310
:106A8000A5F8D8316FE695F8B4315A073FF56BAEEB
:106A900095F8DA3143F0040385F8DA3163E6002231
:106AA000734B9A60FCF74EFC0446FCF74BFC04EB7E
:106AB000004001F01FFB56E6FCF744FC6C4CA4F8C8
:106AC000E800FCF73FFCA4F8EA00FCF73BFCA4F864
:106AD000EC0048E6FCF72CFC654C84F80801FCF758
:106AE00027FC84F80C01FCF723FC84F80B01FCF76D
:106AF0001FFC84F80D0136E6FCF724FC5C4CA4F87E
:106B00000E01FCF71FFCA4F81001FCF711FC84F83F
:106B10001201FCF717FCA4F8140124E6FCF708FCAA
:106B2000534C84F81E01FCF70DFCA4F82801FCF777
:106B300009FCA4F82401FCF705FCA4F82601FCF7E5
:106B4000F7FBD5F8B03184F81F015B79082B7FF68D
:106B50000AAEFCF7F7FBA4F82A01FCF7F3FBA4F854
:106B60002C0100E603235479B4FBF3F4122C3FF616
:106B70003FAD002640F6CA0740F2EE284FF0190953
:106B80003C4DA64205F10205BFF4EDADFCF7D0FB8C
:106B900005F8020CFCF7D6FBB842A8BF38464045C2
:106BA000B8BF4046A0F2EE2090FBF9F0013605F8A0
:106BB000010CE6E7FCF7BCFB2D4B83F82001D2E586
:106BC000FCF7B6FB00232A4CA3606071FCF7BAFB0C
:106BD0000546FCF7B7FB05EB004001F08BFAFCF72C
:106BE000A7FB84F81E01FCF7ADFBA4F8E800FCF756
:106BF000A9FBA4F8EA00FCF7A5FBA4F8EC00FCF75D
:106C0000A1FBA4F80E01FCF79DFBA4F81001AAE576
:106C100002352870FCF796FB6880FCF789FB287129
:106C2000FCF786FB6871FCF783FBE871FCF780FBDF
:106C3000A87105E5012385F8E03194E5137805EBAB
:106C4000860585F87930FCF773FB85F87A00FCF748
:106C50006FFB85F87B00FCF76BFBD4F8BC1185F863
:106C60007C0001F17900FDF759FA7CE5BC0D0020AC
:106C700064080020920900202DE9F04F0022002531
:106C8000624B634EB3F80AC087B034684FEA0C2AEF
:106C900005901889B4EB0A0A65EB020BA0FB0A45C4
:106CA00000FB0B55B3F80480E00940EA45604FEA69
:106CB00008440719D8888E464FEAE511A0FB0A451B
:106CC00000FB0B5541EB0208CDE90278B3F80280D6
:106CD000200A40EA05604FEAC83410EB04084FEA86
:106CE000252141EB02099A89B446A2FB0A0102FB65
:106CF0000B11C20D42EA412212F5FA604FEAE1534C
:106D000043F10001B0F5FA6FCDE9000171F1000126
:106D10005DDADDE902670524A2FB040104FB03112F
:106D200000FB03F402FB0144A0FB020121444D10CF
:106D30004FEA3004361B4FEA900467EB050744EA3C
:106D400081748D104FF0FF313248B8EB040869EBC5
:106D50000509DDE90045844275EB0101CDE90267D3
:106D600022DA40F6AC50002112184B4102FB03F12D
:106D7000A2FB022303EB4103D900D000101A41EA21
:106D8000527163EB0101341847EB0105CDE902456F
:106D90000B24A2FB040104FB031149104FEA30004D
:106DA000B8EB000869EB01090AFB0BF3DDE9000110
:106DB000AAFB0AAB0BEB430B4FEADA7242EA4B0237
:106DC000801A4FEAEB7361EB0301CDE90001DCF8B7
:106DD0000410A1FB082301FB0933540D44EAC3242A
:106DE0005D15DDE90223A21A65EB03031D46D30BF3
:106DF000059A43EA454302B11360BEF1000F02D089
:106E0000009BCEF8003007B0BDE8F08FC805002029
:106E10006416002024FAFFFF012248217720FBF7A7
:106E20009EB9012258217720FBF799B907B50322B3
:106E300001AB00217720FBF753F99DF805309DF851
:106E400004001B0243EA00439DF80600184303B008
:106E50005DF804FB08B5FFF7E9FF014B586008BD7A
:106E60006416002008B5FFF7E1FF014B186008BD6C
:106E7000641600202DE9F047064689464FF000478A
:106E80004FF00008038A8589ADB21D400DB9BDE8F9
:106E9000F087B5FA85F327FA03F2D2431B3B91B290
:106EA00031821540042BF1D8DFE803F02925211A9F
:106EB0000300D9F8244084B1013CA4B2C9F824806D
:106EC000D9F820A0BAF1000FE0D0DAF8003050462F
:106ED00021469847DAF804A0F4E7B48DA4B2EFE7AE
:106EE000D9F80000B18E036889B29847CEE7D9F887
:106EF0000400318FF7E7D9F80800B18FF3E7D9F82C
:106F00000C00B6F84010EEE72DE9F04F0025E44CF8
:106F100085B040F2145200212046DFF8B08306F01D
:106F20002AFB04F5CC73C8F80030DE4BDE4E1D7032
:106F300004F2EE430A2733606A234FF48040237043
:106F4000677101F0D7F84FF4006001F0D3F8022028
:106F500001F0D0F84FF4807001F0CCF84FF41673C4
:106F6000A4F8F230FA23A4F8F4302A23A4F8F0307D
:106F7000C823A4F8FA30012384F8EE3084F80A31EB
:106F80002B2384F80B31232384F80C31242384F839
:106F90000D311023A4F810311E23A4F80E314FF444
:106FA000AF732022A4F81431022384F8F62084F869
:106FB000097184F81231002705230D2284F8EC545E
:106FC000A4F8FE50A4F8FC50A4F8005184F8E45052
:106FD00084F8E55084F8E650A4F8E850A4F8EA50A4
:106FE000A4F8EC5084F8EF5084F8F75084F8F85087
:106FF00084F8895184F8885184F80821C4F88C7188
:10700000C4F8907184F8973140F2DC53A4F824312D
:1070100040F24C43A4F8263140F26C73A4F82831B6
:1070200040F27533A4F82A3140F6430384F89451B2
:1070300084F8955184F8965184F81E5184F81F51B4
:10704000A4F82C312B4625460096032BCCBF0121FA
:10705000002184F82E1114BF1E2105210133122BAB
:1070600084F82F1104F10204EFD1FF2485F8714157
:10707000C824A5F8724140F24C44A5F8D04040F233
:107080009E74A5F8D24040F27E54A5F8D84040F254
:10709000EA544FF47A734FF4FA61A5F8DA4040F2FB
:1070A000B45400264FF001094FF01E0B4FF0320A86
:1070B0000520A5F85231A5F85411A5F85631A5F8C8
:1070C0005811A5F85A31A5F85C11A5F85E31A5F85C
:1070D0006011A5F8D430192140F2DC53A5F8DC404A
:1070E0004FF47A5485F86E01039085F86F11029180
:1070F000A5F8D630019385F821B185F8239185F85C
:107100006D9185F8709185F87491A5F8DEA085F8E9
:10711000206185F8226185F8626185F86C61A5F8C7
:10712000E04040F6AC54A5F8E2A0FCF7D5FF2322DE
:10713000AC81D8F80040AE73E27222735022E27044
:10714000462262730F2262712222A2710E222274E1
:107150003522A276212262745322E2760A22029913
:107160004FF0260EE171A2747821642284F801E0C8
:1071700084F802E022774FF05A0E2822A1722D21C6
:10718000039884F815B084F816B0E07584F804A06C
:1071900084F818B084F808E02670A673E673667663
:1071A000627221754FF4FA71A4F84E103F494048BD
:1071B000A163E1633F49E0622063A1623E484FF072
:1071C0007E51A0644FF07F5C4B2061633B4984F8A3
:1071D0001E90C4F820C0C4F824C084F84C0084F881
:1071E000506084F8516084F852602764616484F8C8
:1071F000536085F8EEE44FF0410E019B85F8EFE413
:10720000A5F8F8344FF0030E202385F8F0A485F894
:10721000F30485F8F16485F8F56485F8F66485F87B
:10722000F26485F8F464A4F85860A4F85A6084F80D
:10723000796084F87AE084F87C3084F88430042320
:1072400084F85C30152310204FF0300C84F881E076
:107250004FF0020E84F86830194B84F87D90E36695
:10726000184B84F878902367DFF86490164BDFF8AA
:1072700064A084F87B0084F87E6084F87F6084F8E2
:1072800080C084F882E084F88300A4F85660216608
:1072900084F8642084F86520636709F1080B1BE01B
:1072A00064080020DD010020BC0D00208FC2F53CE9
:1072B000CDCCCC3E00002040000040400000A0406B
:1072C0009A99193FF6287C3F1F856B3F3C1600209A
:1072D000A8D900089CDB000816F80A10002947D13D
:1072E000282384F813314FF44873A4F816310A2385
:1072F00084F8111184F8121184F8141184F818110B
:1073000040F2145285F86431C823A5F8662185F847
:10731000653185F86811A5F86A316B181031C029FC
:107320001F61FAD121464FF48E72184806F018F901
:1073300021464FF48E72164806F012F9009B1A6827
:10734000144B1168C5F8FA14516859609168996036
:107350001168C5F8061551681961916859610123D2
:1073600085F80833022385F8243405B0BDE8F08F92
:10737000094806F008F930B158453EBFA0EB0900B6
:10738000401980F816610136A6E700BF180B0020EF
:10739000340C00205E0D0020A8D90008F8B5344C4C
:1073A000A368C01A00280CDB0026237BA660012BF3
:1073B00014D007D3022B23D000F042FCA36818445A
:1073C000A060F8BD2B4DAB689847EB689847012348
:1073D000A26823736B881344A360EDE7254D2B69E6
:1073E00098476B689847A2682B8804F110011344F2
:1073F000A36004F114006B69984702232373DBE751
:107400001D4FA1693F684D1C3F782673BD4204BFE4
:1074100001271A4D636904BF2F703546E669184885
:10742000771C032F02BF012784F82070002704EB8C
:107430008606736294F820600268E7616EB1666A3E
:10744000A36AE76A9E42DEBF9E4633467646BE4248
:10745000A8BF3E46B342B8BF334604EB81010B637D
:1074600004EB8501096BA561521A13440360A3E77D
:1074700064160020D80500205407002005020020D3
:107480005007002001490248F4E400BF2014002006
:107490000008004001490248ECE400BFF813002056
:1074A0000004004001494FF08040E3E4D013002085
:1074B00001490248DEE400BFA8130020002C01406F
:1074C000FFF7F6BF254B10B55343254A254C1268EC
:1074D0000139B2FBF3F20388013AA04289B292B2B9
:1074E0009BB212D004F50064A0420ED0B0F1804FE0
:1074F0000BD0A4F59834A04207D004F58064A042D4
:1075000003D004F58064A04202D123F070039BB243
:10751000154CA04206D004F58064A0421CBF23F4A1
:1075200040739BB203800F4B8185984202850FD038
:1075300003F5006398420BD003F54063984207D0EF
:1075400003F58063984203D003F58063984201D12C
:10755000002303860123838210BD00BF40420F0039
:1075600014000020002C0140001000400B4B800A4A
:1075700098420FD004D8B0F5801F09D0FE20704784
:10758000074B984208D049339842F7D10020704702
:10759000012070470220704703207047010010004F
:1075A00002001000F8B5046805462046FFF7DEFF2C
:1075B000032841D8AB7A4FEA930E39B975460227B2
:1075C000A689AF40B6B226EA0706A6810A2505FBC2
:1075D00000E51D4E46F82510043546F825203246B4
:1075E00031B199080223A5898B402B439BB2A3811B
:1075F0002823434303F120011144EFF31286502561
:1076000085F312880425103313441F6817B10F60E7
:1076100019680431013D03F10403F6D10D60F3B2A2
:1076200083F31188282303FB0020036A2BB1A3896D
:107630009BB243F00103A381F8BDA38923F00103AA
:107640001B041B0CF7E700BFA81300200148FDF73F
:10765000DFBB00BF541700200148FDF7D9BB00BFB6
:10766000A81700204FF400520C480D4B5A60D0F878
:107670007821136823F001031B041B0C1360D0F85E
:107680006821D0F86C319A4203D000F5A270FDF762
:10769000F1BB012380F88831704700BF64160020D9
:1076A00000000240044A536823B192F9002082424C
:1076B00000D11847704700BFFC1700200022024B82
:1076C0001A70FCF723BC00BF180800202DE9F04118
:1076D00000240A274FF47A761A4D82781FFA82FE28
:1076E000A4EB0E031BB2002B29DDC2F16402D2B25F
:1076F00003FB03FC90F80380524308FB0CFC9CFB4B
:10770000F2F2C8F164084244534393FBF7F30EEBE3
:107710008E0E03EB4E031BB26B800A88B1F802E0B9
:107720000A34AEEB020E03FB0EF393FBF6F3A4B2A6
:107730001344782C25F8023FCFD1BDE8F08108BF73
:107740000122D5E70218002030B5002340F6C41509
:10775000094C03FB03F2A2F1190142784A4302F6F5
:10776000C4125A4301784A4392FBF5F224F81320DD
:107770000133072BEDD130BD1C1800200F4B043016
:1077800033F9102040F633039A42A8BF1A46192352
:10779000B2F5617FB8BF4FF461720878584300F2C8
:1077A0008330904208DA4878584300F283309042A0
:1077B000B4BF00200120704700207047900D0020CA
:1077C0000C4B1B6813F4805F0B4B0BD0C089B3F9D3
:1077D0000630421A93420ADD08448342B4BF0020B7
:1077E00001207047B3F90610008A8142F6E70120B4
:1077F000704700BF00160020900D00200022034BB0
:1078000083F82E201A639A869A637047FC1700202B
:1078100030B408B930BCF1E70D4A0023114612F824
:107820003350DC00854204D00133102BF7D130BC3B
:107830007047084B986B20B12244557842789542A6
:10784000F5D20022214499639A861A63EFE700BFBC
:10785000C0D90008FC1700204000142870B4A8BF4D
:107860001420002302261425084A02F13C015E542C
:107870000233CC18984204F8015CF8DC1344FF2270
:1078800083F83C200F2070BCC2E700BFFC1700202B
:10789000F8B50E46141E0546CCBF02200120FFF7A6
:1078A000DBFF731E132B00F2BE81DFE813F0140020
:1078B0002000290037004B005100A100F1004101D8
:1078C00071019701BC01370042005100A100F10095
:1078D0007B00CB001B012A781444FA2CA8BFFA24A1
:1078E00024EAE4742C702846BDE8F8402CE76A7856
:1078F0001444642CA8BF642424EAE4746C70F2E796
:10790000EA789E4B1444642CA8BF642424EAE474EF
:10791000EC7019682846BDE8F840D7E66B79234437
:10792000642BA8BF64230D2E23EAE3736B7100F070
:107930007A812A791444642CA8BF642424EAE4746C
:107940002C71F8BDAA79144484F30804AC71F8BD15
:107950008B4B1D682B78022B19D1204601F0EAFBD6
:10796000884901F0EFFC696A01F030FB002107460D
:1079700001F0D2FD48B98449384601F0EBFD00B171
:10798000814F0F2E6F6212D1F8BD0027F9E7AB7857
:107990002344C82BA8BFC8230F2E23EAE373AB7080
:1079A0001DD1F8BD764B1D682B78022B17D12046D0
:1079B00001F0C0FB734901F0C5FC296A01F006FB28
:1079C0000021044601F0A8FD38B96F49204601F0B6
:1079D000C1FD00B16C4C2C62F8BD0024FBE76A7855
:1079E0001444C82CA8BFC82424EAE4746C70F8BD01
:1079F000634B1D682B78022B19D1204601F09AFBAE
:107A0000614901F09FFC296B01F0E0FA0021074673
:107A100001F082FD48B95C49384601F09BFD00B198
:107A2000594F102E2F6312D1F8BD0027F9E72B7B99
:107A30002344C82BA8BFC823102E23EAE3732B735B
:107A40001DD1F8BD4E4B1D682B78022B17D1204657
:107A500001F070FB4C4901F075FCE96A01F0B6FADF
:107A60000021044601F058FD38B94749204601F08D
:107A700071FD00B1444CEC62F8BD0024FBE7EA7AEA
:107A80001444C82CA8BFC82424EAE474EC72F8BDDE
:107A90003B4B1D682B78022B19D1204601F04AFB85
:107AA0003A4901F04FFCE96B01F090FA00210746DA
:107AB00001F032FD48B93449384601F04BFD00B1C0
:107AC000314F112EEF6312D1F8BD0027F9E7AB7DDE
:107AD0002344C82BA8BFC823112E23EAE373AB7538
:107AE0001DD1F8BD264B1D682B78022B17D12046DF
:107AF00001F020FB254901F025FCA96B01F066FA95
:107B00000021044601F008FD38B91F49204601F064
:107B100021FD00B11C4CAC63F8BD0024FBE76A7D7D
:107B20001444C82CA8BFC82424EAE4746C75F8BDBA
:107B3000134B1D682B78022B17D1204601F0FAFA5F
:107B4000104901F0FFFBA96A01F040FA0021044648
:107B500001F0E2FC38B90C49204601F0FBFC00B111
:107B6000094CAC62F8BD0024FBE7EA781444C82C49
:107B7000A8BFC82424EAE474EC70F8BD780D002096
:107B80007C0D0020000020410000C84200007A4423
:107B9000254B1D682B78022B17D1204601F0CAFA1D
:107BA000224901F0CFFB696B01F010FA0021044675
:107BB00001F0B2FC38B91D49204601F0CBFC00B100
:107BC0001A4C6C63F8BD0024FBE76A7B1444C82C94
:107BD000A8BFC82424EAE4746C73F8BD124B1D6876
:107BE0002B78022B17D1204601F0A4FA104901F09E
:107BF000A9FB296C01F0EAF90021044601F08CFC94
:107C000038B90A49204601F0A5FC00B1074C2C64A4
:107C1000F8BD0024FBE7EA7D1444C82CA8BFC824A3
:107C200024EAE474EC75F8BD7C0D00200000C84225
:107C300000007A44014B1868704700BFC40D002053
:107C400010B50A490A480A68846800BF0B689A425E
:107C5000F9D14FF47A70074B596D00FB01F31B1BF0
:107C6000B3FBF1F300FB023010BD00BFC40D0020D8
:107C700010E000E0FC17002038B50446FFF7E0FFF5
:107C80000546FFF7DDFF401BA042FAD338BD10B513
:107C9000044604B910BD4FF47A70FFF7EDFF013CC4
:107CA000F7E706462DE98748294C0B27013FFCD012
:107CB0004FF01E0905254FF0020806F0400A06F0B5
:107CC000200B00E00025BAF1000F03D0E36883F435
:107CD0000043E360BBF1000F03D0E36883F480430B
:107CE000E36016F0020218BFE36848461CBF83F445
:107CF0000053E3600192FFF7CAFF019ABAF1000F47
:107D000003D0E36883F40043E360BBF1000F03D0CA
:107D1000E36883F48043E3601AB1E36883F40053BB
:107D2000E3604846FFF7B3FF7DB1013DCBD14FF48F
:107D3000FA70FFF7ACFF4FF09609B8F1000FC1D110
:107D40004FF47A70FFF7A3FFB0E708F1FF38F4E7CC
:107D500000100140024A136801331360704700BFEE
:107D6000C40D002009209DE428209BE4174B2DE939
:107D7000F0410746B3F8580090460C4601F0D6F99A
:107D8000134901F02BFA0646404601F0D3F9114998
:107D900001F024FA01464FF07E5001F0D3FA31464B
:107DA00001F014F90146304601F0CCFA2568064688
:107DB0002946384601F008F90146304601F00EFA2E
:107DC000294601F003F92060BDE8F081FC1700208E
:107DD000BD378635DB0FC94000231B68FFDE00225C
:107DE0000123184291B206D101325B00082A9BB2EE
:107DF000F7D14FF6FF710846704780EAE073A3EBB6
:107E0000E0738B4206DB002801DD401A704702D088
:107E1000084470470020704770B5044601F0BAFB73
:107E2000203040285BD82F4D2F4E2946204601F0A8
:107E300091FB00283AD12D4D2B4E2946204601F0CA
:107E40006BFB002838D12A49204601F083FB00282B
:107E500038D02749204601F0B7F80146244801F000
:107E6000B3F804462146204601F0B8F905462149F9
:107E700001F0B4F9204901F0A7F8294601F0AEF964
:107E80001E4901F0A3F8294601F0A8F91C4901F0A8
:107E90009BF829460646204601F0A0F901463046E7
:107EA00001F09CF9214601F091F870BD2046314661
:107EB00001F08AF80446B8E72046314601F086F81A
:107EC0000446BAE70F49204601F026FB0028C9D036
:107ED0000749204601F07AF801460A48BFE700202A
:107EE00070BD00BFDB0F4940DB0FC940DB0F49C04D
:107EF000DB0FC93F9A7C2E36FAAF4F393587083CE5
:107F0000A4AA2A3EDB0FC9BF2DE9F04F056885B052
:107F10000C4681463A49284601F058F8FFF77CFFA5
:107F200080462846FFF778FFD9F8045006463449C2
:107F3000284601F04BF8FFF76FFF07462846FFF78A
:107F40006BFFD9F8089005462D49484601F03EF8E8
:107F5000FFF762FF82464846FFF75EFF41468146D3
:107F6000504601F03BF941460190484601F036F990
:107F700051460290304601F031F9494603903046AF
:107F800001F02CF939468346504601F027F949465D
:107F9000206007F1004001F021F903996060A560BD
:107FA000284601F01BF9029901F010F85946E060EB
:107FB000284601F013F90146019801F005F8394609
:107FC000206106F1004001F009F90199606128463D
:107FD00001F004F90146584600F0F6FF0299A0614D
:107FE000284601F0FBF8039900F0F0FF4146E061FC
:107FF000384601F0F3F8206205B0BDE8F08F00BF0D
:10800000DB0FC93F2DE9F04104468AB027680846D6
:1080100001A96668A568FFF777FF0199384601F066
:10802000DDF804998046304601F0D8F80146404614
:1080300000F0CCFF07998046284601F0CFF80146B2
:10804000404600F0C3FF02992060384601F0C6F8B0
:1080500005998046304601F0C1F80146404600F0DF
:10806000B5FF08998046284601F0B8F80146404619
:1080700000F0ACFF03996060384601F0AFF8069954
:108080000746304601F0AAF80146384600F09EFF48
:1080900009990646284601F0A1F80146304600F04D
:1080A00095FFA0600AB0BDE8F08110B5054C2288AC
:1080B00022EA00008242208002D00120FFF7CCFBA0
:1080C000208810BDA007002010B5054C2288104361
:1080D0008242208002D00120FFF7BEFB208810BD25
:1080E000A0070020024A936823EA000090607047CE
:1080F00064080020024A936818439060704700BFEC
:108100006408002038B50E4C19252068FFF71CFBC9
:10811000002220680B4C02FB02F3A3F11901037A41
:108120004B4303F6C413534393FBF5F324F8123087
:108130000132072AEFD1BDE838400349FFF7C6BA3C
:10814000BC0D0020C00200203409002010B5104BE7
:108150001A786A2A1AD140F214525988914215D1DC
:108160001A79BE2A12D193F81225EF2A0ED10022D5
:10817000084C13F8010B80EA0201A342C9B203D1F3
:10818000831A5842584110BD0A46F2E7002010BD3C
:1081900000F8000814FD00082DE9F743FEF7DEF9AA
:1081A0006A234A4E40F214513370BE233371EF23D9
:1081B00086F8123500231846718086F81335F25C74
:1081C00001338B4280EA0200F9D186F813050427B7
:1081D00000203F4C3F4BDFF80491636003F188338C
:1081E0006360013F17F0FF0739D034233A4DE36055
:1081F00005F17848A8F57848C8F30903002B3BD06F
:1082000000234FF4005056F808800193FCF702FA5F
:108210000428E6D123694FF4005043F001032361A1
:108220001FFA88F32B80FCF7F5F9042842D1AB1C28
:108230000193019B4FEA1848A3F800804FF40050C7
:10824000FCF7E8F92369042823F001034FEAC3434C
:108250004FEAD3432361C4D104354D45C8D11C4AEC
:108260000428136943F08003136102D1FFF76EFF06
:1082700038BB0420FFF715FD4FF43020FCF7CAF996
:108280000428AED123694FF4302043F00203236168
:108290006561236943F040032361FCF7BBF923695F
:1082A000042823F002034FEAC3434FEAD343236178
:1082B000A6D096E7236923F00103DB04DB0C2361DE
:1082C0008FE7FEF735F903B0BDE8F08364080020BE
:1082D000002002402301674500F8000814FD000853
:1082E0002DE9F041FFF732FF10B90320FFF7D9FC69
:1082F0009B4CFEF733F940F214529A49204605F0A0
:108300002FF994F8EC344FF48E71022B84BF0023C4
:1083100084F8EC3494F8EC24934D01FB02F303F55C
:10832000CC7020442344286093F8EC0101FB024206
:10833000022884BF002083F8EC0192F8EC318B4ACC
:1083400013700C2202FB0343894A03F2EE431360CD
:1083500046F20902A3681A4203D14FF40050FFF716
:10836000C9FEA368D80703D54FF40050FFF7BAFE43
:10837000A368590409D50820FFF7B4FE4FF4005054
:10838000FFF7B0FE0120FFF7ADFEA3681A0706D580
:108390004FF40050FFF7A6FE0120FFF7A3FEA368ED
:1083A0009B0412D54FF40040FFF79CFE94F8123165
:1083B000012B03D14FF40060FFF794FE4FF480309F
:1083C000FFF790FE4020FFF78DFE94F86C312BB143
:1083D00094F8703113B1002384F870310020FF2726
:1083E0000246644E644B1E602318B3F87A114B08A2
:1083F00003F077334FEA910C0CF0333CCB1AA3EB2C
:108400000C034FEAD10C0CF0113CA3EB0C0303EB73
:10841000231303F00F3393FBF7FC11F0010ECCEBA9
:108420000C2C18BF0132A3EB0C0318BFD2B2012BE6
:108430000ADD022B40F09080BEF1000F00F08C802E
:1084400011F0BC0F00F0888008301028CCD1013A20
:10845000012A00F28180FFF755FE302200214748B3
:1084600005F089F82968464F01F17900FBF756FEBF
:10847000444BA7F126081F602B681878FDF7A0FE73
:10848000414B07F16E021A60642294F864113F4B6D
:108490004A43C8325A6000229A60DA601A615A610F
:1084A0009A61DA6183F8202083F82120384BBA1DC5
:1084B0001A60384BA7F11E021A60374B7A37C3F89F
:1084C0000080364BB4F8F2001F60354B1E6000F0A0
:1084D0002DFE344E7060B4F8F40000F027FE2D68D5
:1084E000B06095F85C3005F16402337095F878302F
:1084F000286E737094F86F312B4933732B4BB5F89A
:1085000016411E602A4B1A6000F068FE01464FF0CB
:108510007C5000F017FF274B1860204600F00AFE41
:108520000146254800F00EFF244900F057FE244A7A
:10853000244B1560244A186005F168031360234A30
:1085400005F211151560224AC2F80080214ABDE8E3
:10855000F0411360FDF7ECBFFBF7BEFD7BE700BF0A
:108560006408002000F800083C160020DD0100200F
:10857000BC0D00207A090020FC150020AC01002071
:108580005A09002010020020380700200C16002095
:10859000AC0E0020481400204C140020B40300202E
:1085A0007804002058180020DB0F494058140020A0
:1085B0006814002064140020000061444C3D0F4406
:1085C00078070020B00300206C070020A4030020DF
:1085D000AC0300205407002008B5FFF7DDFDFFF7CE
:1085E0007FFEBDE808400120FFF736B90C4A13783A
:1085F000590713D523F0040313700123094A0A49CC
:10860000136000220A60094904200A60084A1380A6
:108610004B22084B1B685A71FFF7FAB8704700BF2E
:108620003416002030000020CC0D0020C80D0020A2
:108630008A0D0020BC0D002008B5044B1B7803F008
:108640000503052B01D1FDF775FCFEE76818002036
:10865000034613F8012B002AFBD1181A0138704782
:10866000D0400B1C1141203A03D49C4613411843BF
:108670006346524293401843704700BF81F0004167
:1086800002E000BF83F0004330B54FEA41044FEAF7
:10869000430594EA050F08BF90EA020F1FBF54EA92
:1086A000000C55EA020C7FEA645C7FEA655C00F02E
:1086B000E2804FEA5454D4EB5555B8BF6D420CDDFF
:1086C0002C4480EA020281EA030382EA000083EA82
:1086D000010180EA020281EA0303362D88BF30BD22
:1086E00011F0004F4FEA01314FF4801C4CEA113178
:1086F00002D0404261EB410113F0004F4FEA0333D7
:108700004CEA133302D0524263EB430394EA050F61
:1087100000F0A780A4F10104D5F1200E0DDB02FAD0
:108720000EFC22FA05F2801841F1000103FA0EF264
:10873000801843FA05F359410EE0A5F120050EF12A
:10874000200E012A03FA0EFC28BF4CF0020C43FA5B
:1087500005F3C01851EBE37101F0004507D54FF068
:10876000000EDCF1000C7EEB00006EEB0101B1F5B8
:10877000801F1BD3B1F5001F0CD349085FEA3000FE
:108780004FEA3C0C04F101044FEA445212F5800F09
:1087900080F09A80BCF1004F08BF5FEA500C50F1A6
:1087A000000041EB045141EA050130BD5FEA4C0C89
:1087B000404141EB010111F4801FA4F10104E9D112
:1087C00091F0000F04BF01460020B1FA81F308BF09
:1087D0002033A3F10B03B3F120020CDA0C3208DDD5
:1087E00002F1140CC2F10C0201FA0CF021FA02F1B0
:1087F0000CE002F11402D8BFC2F1200C01FA02F120
:1088000020FA0CFCDCBF41EA0C019040E41AA2BF44
:1088100001EB0451294330BD6FEA04041F3C1CDA0C
:108820000C340EDC04F11404C4F1200220FA04F02C
:1088300001FA02F340EA030021FA04F345EA0301D6
:1088400030BDC4F10C04C4F1200220FA02F001FA98
:1088500004F340EA0300294630BD21FA04F029461A
:1088600030BD94F0000F83F4801306BF81F48011B3
:108870000134013D4EE77FEA645C18BF7FEA655C26
:1088800029D094EA050F08BF90EA020F05D054EAF8
:10889000000C04BF1946104630BD91EA030F1EBFFD
:1088A0000021002030BD5FEA545C05D14000494101
:1088B00028BF41F0004130BD14F580043CBF01F5F4
:1088C000801130BD01F0004545F0FE4141F47001DA
:1088D0004FF0000030BD7FEA645C1ABF19461046B5
:1088E0007FEA655C1CBF0B46024650EA013406BFB6
:1088F00052EA033591EA030F41F4002130BD00BF75
:1089000090F0000F04BF0021704730B54FF4806431
:1089100004F132044FF000054FF0000150E700BFB2
:1089200090F0000F04BF0021704730B54FF4806411
:1089300004F1320410F0004548BF40424FF00001FE
:108940003EE700BF42004FEAE2014FEA31014FEA41
:1089500002701FBF12F07F4393F07F4F81F0605190
:10896000704792F0000F14BF93F07F4F704730B5FF
:108970004FF4607401F0004521F0004120E700BF92
:1089800050EA010208BF704730B54FF000050AE019
:1089900050EA010208BF704730B511F0004502D51A
:1089A000404261EB41014FF4806404F132045FEA1C
:1089B000915C3FF4DCAE4FF003025FEADC0C18BFC1
:1089C00003325FEADC0C18BF033202EBDC02C2F1B7
:1089D000200300FA03FC20FA02F001FA03FE40EA49
:1089E0000E0021FA02F11444C1E600BF70B54FF049
:1089F000FF0C4CF4E06C1CEA11541DBF1CEA13552B
:108A000094EA0C0F95EA0C0F00F0DEF82C4481EA92
:108A1000030621EA4C5123EA4C5350EA013518BFB2
:108A200052EA033541F4801143F4801338D0A0FB9F
:108A300002CE4FF00005E1FB02E506F00042E0FB4C
:108A400003E54FF00006E1FB03569CF0000F18BF52
:108A50004EF0010EA4F1FF04B6F5007F64F54074FA
:108A600004D25FEA4E0E6D4146EB060642EAC6218D
:108A700041EA55514FEAC52040EA5E504FEACE2EFA
:108A8000B4F1FD0C88BFBCF5E06F1ED8BEF1004FFD
:108A900008BF5FEA500E50F1000041EB045170BD79
:108AA00006F0004646EA010140EA020081EA0301BD
:108AB000B4EB5C04C2BFD4EB0C0541EA045170BDB9
:108AC00041F480114FF0000E013C00F3AB8014F133
:108AD000360FDEBF002001F0004170BDC4F100047C
:108AE000203C35DA0C341BDC04F11404C4F12005FD
:108AF00000FA05F320FA04F001FA05F240EA020058
:108B000001F0004221F0004110EBD37021FA04F68D
:108B100042EB06015EEA430E08BF20EAD37070BD47
:108B2000C4F10C04C4F1200500FA04F320FA05F0A6
:108B300001FA04F240EA020001F0004110EBD370A8
:108B400041F100015EEA430E08BF20EAD37070BD18
:108B5000C4F1200500FA05F24EEA020E20FA04F3F1
:108B600001FA05F243EA020321FA04F001F00041A0
:108B700021FA04F220EA020000EBD3705EEA430E11
:108B800008BF20EAD37070BD94F0000F0FD101F040
:108B90000046400041EB010111F4801F08BF013C79
:108BA000F7D041EA060195F0000F18BF704703F0B7
:108BB0000046520043EB030313F4801F08BF013D3E
:108BC000F7D043EA0603704794EA0C0F0CEA1355FA
:108BD00018BF95EA0C0F0CD050EA410618BF52EAB4
:108BE0004306D1D181EA030101F000414FF00000BA
:108BF00070BD50EA410606BF1046194652EA4306C8
:108C000019D094EA0C0F02D150EA013613D195EA3B
:108C10000C0F05D152EA03361CBF104619460AD183
:108C200081EA030101F0004141F0FE4141F470018D
:108C30004FF0000070BD41F0FE4141F4780170BD7D
:108C400070B54FF0FF0C4CF4E06C1CEA11541DBFE2
:108C50001CEA135594EA0C0F95EA0C0F00F0A7F8E4
:108C6000A4EB050481EA030E52EA03354FEA013111
:108C700000F088804FEA03334FF0805545EA131324
:108C800043EA12634FEA022245EA111545EA1065EC
:108C90004FEA00260EF000419D4208BF964244F183
:108CA000FD0404F5407402D25B084FEA3202B61AA2
:108CB00065EB03055B084FEA32024FF480104FF476
:108CC000002CB6EB020E75EB030E22BFB61A7546EA
:108CD00040EA0C005B084FEA3202B6EB020E75EB7D
:108CE000030E22BFB61A754640EA5C005B084FEAE5
:108CF0003202B6EB020E75EB030E22BFB61A7546B2
:108D000040EA9C005B084FEA3202B6EB020E75EBBC
:108D1000030E22BFB61A754640EADC0055EA060E7D
:108D200018D04FEA051545EA16754FEA06164FEAC0
:108D3000C30343EA52734FEAC2025FEA1C1CC0D16C
:108D400011F4801F0BD141EA00014FF000004FF0F9
:108D5000004CB6E711F4801F04BF01430020B4F1BA
:108D6000FD0C88BFBCF5E06F3FF6AFAEB5EB030C72
:108D700004BFB6EB020C5FEA500C50F1000041EB6F
:108D8000045170BD0EF0004E4EEA113114EB5C043C
:108D9000C2BFD4EB0C0541EA045170BD41F480110F
:108DA0004FF0000E013C90E645EA060E8DE60CEA17
:108DB000135594EA0C0F08BF95EA0C0F3FF43BAF34
:108DC00094EA0C0F0AD150EA01347FF434AF95EAEB
:108DD0000C0F7FF425AF104619462CE795EA0C0FCF
:108DE00006D152EA03353FF4FDAE1046194622E79C
:108DF00050EA410618BF52EA43067FF4C5AE50EA76
:108E000041047FF40DAF52EA43057FF4EBAE12E765
:108E10004FF0FF3C06E000BF4FF0010C02E000BF46
:108E20004FF0010C4DF804CD4FEA410C7FEA6C5C29
:108E30004FEA430C18BF7FEA6C5C1BD001B050EACC
:108E4000410C0CBF52EA430C91EA030F02BF90EAB7
:108E5000020F0020704710F1000F91EA030F58BF76
:108E6000994208BF90422CBFD8176FEAE37040F0D8
:108E7000010070474FEA410C7FEA6C5C02D150EA76
:108E8000013C07D14FEA430C7FEA6C5CD6D152EA31
:108E9000033CD3D05DF8040B704700BF84461046F6
:108EA00062468C461946634600E000BF01B5FFF7F5
:108EB000B7FF002848BF10F1000F01BD4DF808EDC5
:108EC000FFF7F4FF0CBF012000205DF808FB00BF96
:108ED0004DF808EDFFF7EAFF34BF012000205DF8F0
:108EE00008FB00BF4DF808EDFFF7E0FF94BF01203D
:108EF00000205DF808FB00BF4DF808EDFFF7CEFF3E
:108F000094BF012000205DF808FB00BF4DF808ED7C
:108F1000FFF7C4FF34BF012000205DF808FB00BF4D
:108F20004FEA4102B2F1E04324BFB3F5001CDCF18B
:108F3000FE5C0DD901F0004C4FEAC0024CEA5070C3
:108F4000B2F1004F40EB830008BF20F001007047F2
:108F500011F0804F21D113F13872BCBF01F00040F5
:108F6000704741F480114FEA5252C2F11802C2F127
:108F7000200C10FA0CF320FA02F018BF40F00100A8
:108F80004FEAC1234FEAD32303FA0CFC40EA0C005A
:108F900023FA02F34FEA4303CCE77FEA625307D197
:108FA00050EA01331EBF4FF0FE4040F440007047CE
:108FB00001F0004040F0FE4040F40000704700BF68
:108FC00080F0004002E000BF81F0004142001FBF7E
:108FD0005FEA410392EA030F7FEA226C7FEA236C87
:108FE0006AD04FEA1262D2EB1363C1BFD21841407C
:108FF00048404140B8BF5B42192B88BF704710F012
:10900000004F40F4000020F07F4018BF404211F0B4
:10901000004F41F4000121F07F4118BF494292EA1C
:10902000030F3FD0A2F1010241FA03FC10EB0C0048
:10903000C3F1200301FA03F100F0004302D54942D5
:1090400060EB4000B0F5000F13D3B0F1807F06D382
:1090500040084FEA310102F10102FE2A51D2B1F17A
:10906000004F40EBC25008BF20F0010040EA03006F
:109070007047490040EB000010F4000FA2F101021C
:10908000EDD1B0FA80FCACF1080CB2EB0C0200FAA6
:109090000CF0AABF00EBC25052421843BCBFD040F4
:1090A0001843704792F0000F81F4000106BF80F46E
:1090B00000000132013BB5E74FEA41037FEA226C31
:1090C00018BF7FEA236C21D092EA030F04D092F0FC
:1090D000000F08BF0846704790EA010F1CBF002030
:1090E000704712F07F4F04D1400028BF40F000408D
:1090F000704712F100723CBF00F50000704700F0AD
:10910000004343F0FE4040F4000070477FEA2262D3
:1091100016BF08467FEA23630146420206BF5FEAA4
:10912000412390EA010F40F4800070474FF00003A4
:1091300004E000BF10F0004348BF40425FEA000C6B
:1091400008BF704743F0964301464FF000001CE013
:1091500050EA010208BF70474FF000030AE000BF69
:1091600050EA010208BF704711F0004302D54042A7
:1091700061EB41015FEA010C02BF84460146002019
:1091800043F0B64308BFA3F18053A3F50003BCFA34
:109190008CF2083AA3EBC25310DB01FA02FC6344E1
:1091A00000FA02FCC2F12002BCF1004F20FA02F2E8
:1091B00043EB020008BF20F00100704702F12002DB
:1091C00001FA02FCC2F1200250EA4C0021FA02F23C
:1091D00043EB020008BF20EADC7070474FF0FF0C41
:1091E0001CEAD0521EBF1CEAD15392EA0C0F93EA3C
:1091F0000C0F6FD01A4480EA010C400218BF5FEADE
:1092000041211ED04FF0006343EA501043EA511150
:10921000A0FB01310CF00040B1F5000F3EBF49004A
:1092200041EAD3715B0040EA010062F17F02FD2A4E
:109230001DD8B3F1004F40EBC25008BF20F0010031
:10924000704790F0000F0CF0004C08BF49024CEA48
:10925000502040EA51207F3AC2BFD2F1FF0340EADA
:10926000C250704740F400004FF00003013A5DDC4B
:1092700012F1190FDCBF00F000407047C2F100028C
:10928000410021FA02F1C2F1200200FA02FC5FEA79
:10929000310040F1000053EA4C0308BF20EADC70C3
:1092A000704792F0000F00F0004C02BF400010F435
:1092B000000F013AF9D040EA0C0093F0000F01F0E2
:1092C000004C02BF490011F4000F013BF9D041EA04
:1092D0000C018FE70CEAD15392EA0C0F18BF93EA06
:1092E0000C0F0AD030F0004C18BF31F0004CD8D130
:1092F00080EA010000F00040704790F0000F17BFB7
:1093000090F0004F084691F0000F91F0004F14D0FC
:1093100092EA0C0F01D142020FD193EA0C0F03D154
:109320004B0218BF084608D180EA010000F0004057
:1093300040F0FE4040F40000704740F0FE4040F432
:10934000400070474FF0FF0C1CEAD0521EBF1CEAD1
:10935000D15392EA0C0F93EA0C0F69D0A2EB0302EF
:1093600080EA010C49024FEA402037D04FF0805389
:1093700043EA111143EA10130CF000408B4238BF4E
:109380005B0042F17D024FF4000C8B4224BF5B1A5C
:1093900040EA0C00B3EB510F24BFA3EB510340EAAA
:1093A0005C00B3EB910F24BFA3EB910340EA9C0058
:1093B000B3EBD10F24BFA3EBD10340EADC001B01C8
:1093C00018BF5FEA1C1CE0D1FD2A3FF650AF8B426C
:1093D00040EBC25008BF20F0010070470CF0004C79
:1093E0004CEA50207F32C2BFD2F1FF0340EAC250A4
:1093F000704740F400004FF00003013A37E792F065
:10940000000F00F0004C02BF400010F4000F013AC2
:10941000F9D040EA0C0093F0000F01F0004C02BFBD
:10942000490011F4000F013BF9D041EA0C0195E726
:109430000CEAD15392EA0C0F08D142027FF47DAFBF
:1094400093EA0C0F7FF470AF084676E793EA0C0FAF
:1094500004D14B023FF44CAF08466EE730F0004CAD
:1094600018BF31F0004CCAD130F000427FF45CAF3D
:1094700031F000437FF43CAF5FE700BF4FF0FF3CAB
:1094800006E000BF4FF0010C02E000BF4FF0010CFE
:109490004DF804CD4FEA40024FEA41037FEA226CC7
:1094A00018BF7FEA236C11D001B052EA530C18BFE9
:1094B00090EA010F58BFB2EB030088BFC81738BF4E
:1094C0006FEAE17018BF40F0010070477FEA226C3C
:1094D00002D15FEA402C05D17FEA236CE4D15FEA38
:1094E000412CE1D05DF8040B704700BF844608466C
:1094F0006146FFE70FB5FFF7C9FF002848BF10F12D
:10950000000F0FBD4DF808EDFFF7F4FF0CBF012071
:1095100000205DF808FB00BF4DF808EDFFF7EAFFFB
:1095200034BF012000205DF808FB00BF4DF808EDB6
:10953000FFF7E0FF94BF012000205DF808FB00BFAB
:109540004DF808EDFFF7D2FF94BF012000205DF831
:1095500008FB00BF4DF808EDFFF7C8FF34BF01203E
:1095600000205DF808FB00BF4FEA40024FEA4103CC
:109570007FEA226C02D15FEA402C08D17FEA236C9B
:1095800002D15FEA412C02D14FF0000070474FF04A
:10959000010070474FEA4002B2F1FE4F0FD34FF087
:1095A0009E03B3EB12620DD94FEA002343F0004350
:1095B00010F0004F23FA02F018BF404270474FF0FE
:1095C0000000704712F1610F01D1420205D110F085
:1095D000004008BF6FF0004070474FF00000704738
:1095E00042000ED2B2F1FE4F0BD34FF09E03B3EB0D
:1095F000126209D44FEA002343F0004323FA02F039
:1096000070474FF00000704712F1610F01D1420224
:1096100002D14FF0FF3070474FF00000704700BF9D
:109620007BB972B90029BEBF00204FF0004106E0AF
:1096300008BF00281CBF6FF000414FF0FF3000F062
:10964000E7B9ADF1080C6DE904CE002909DB002B68
:109650001ADB00F06FF8DDF804E0DDE9022304B066
:109660007047404261EB4101002B1BDB00F062F8C8
:10967000DDF804E0DDE9022304B0404261EB410182
:10968000524263EB43037047524263EB430300F0E3
:1096900051F8DDF804E0DDE9022304B0404261EB5B
:1096A00041017047524263EB430300F043F8DDF899
:1096B00004E0DDE9022304B0524263EB4303704748
:1096C00010B500210446FFF727FF20B92046BDE86A
:1096D000104000F009B804F1004000F005F84042E5
:1096E00061EB410110BD00BFD0B5FFF72BF900229F
:1096F0000E4B06460F46FFF779F900F08BF904464A
:10970000FFF7FEF800220A4BFFF770F902460B46FE
:1097100030463946FEF7B6FF00F07CF923460022BA
:1097200042EA000210461946D0BD00BF0000F03DDD
:109730000000F0412DE9F0478C460E460446089D96
:10974000002B50D18A4217466CD9B2FA82FEBEF184
:10975000000F0BD0CEF1200C01FA0EF620FA0CFC13
:1097600002FA0EF74CEA060C00FA0EF43A0CBCFBB7
:10977000F2F9BBB202FB19CC09FB03FA4FEA144819
:1097800048EA0C46B2450AD9F61909F1FF3180F0D2
:109790002581B24540F22281A9F102093E44A6EB9F
:1097A0000A06B6FBF2F002FB106600FB03F3A4B25C
:1097B00044EA0644A34209D9E41900F1FF3280F0DB
:1097C0000B81A34240F2088102383C440021E41A94
:1097D00040EA0940002D62D0002324FA0EF42C60E8
:1097E0006B60BDE8F0878B4207D9002D55D0002172
:1097F00085E841000846BDE8F087B3FA83F1002907
:1098000040F08F80B34202D3824200F2FC80841A7F
:1098100066EB03060120B446002D40D085E8101009
:10982000BDE8F08712B90127B7FBF2F7B7FA87FE58
:10983000BEF1000F35D10121F61B4FEA174C1FFA7C
:1098400087F8B6FBFCF20CFB126608FB02F0230C57
:1098500043EA0646B04207D9F61902F1FF3302D2B5
:10986000B04200F2D2801A46361AB6FBFCF00CFB6E
:10987000106608FB00F8A3B243EA0644A04507D9E6
:10988000E41900F1FF3302D2A04500F2B980184676
:10989000A4EB080440EA02409CE729462846BDE8BC
:1098A000F08707FA0EF7CEF1200326FA03F24FEA0B
:1098B000174CB2FBFCF11FFA87F80CFB112206FAD9
:1098C0000EF620FA03F301FB08F933431E0C46EAB7
:1098D0000246B14500FA0EF409D9F61901F1FF323A
:1098E00080F08C80B14540F2898002393E44A6EB7D
:1098F0000906B6FBFCF00CFB106200FB08F99EB2F7
:1099000046EA0246B14507D9F61900F1FF3371D294
:10991000B1456FD902383E44A6EB090640EA014141
:109920008FE7C1F1200722FA07F88B4048EA0303CA
:1099300026FA07F44FEA134EB4FBFEF91FFA83FC34
:109940000EFB19448E4020FA07F809FB0CFA48EA8E
:1099500006084FEA184646EA0444A24502FA01F214
:1099600000FA01F608D9E41809F1FF3044D2A24503
:1099700042D9A9F102091C44A4EB0A04B4FBFEF08D
:109980000EFB104400FB0CFC1FFA88F848EA044464
:10999000A44507D9E41800F1FF3E29D2A44527D9F0
:1099A00002381C4440EA0940A0FB0289A4EB0C0CDD
:1099B000CC45C246CE4615D312D055B1B6EB0A03FC
:1099C0006CEB0E0606FA07F7CB401F43CE402F6024
:1099D0006E600021BDE8F0871046F7E68946DEE6B6
:1099E0004645EAD2B8EB020A69EB030E0138E4E718
:1099F0007046D7E718468FE78146BDE7114676E700
:109A000002383C4444E7084606E7023A3E442BE766
:109A1000704700BF4A0011D212F5001211D20DD5C5
:109A20006FF47873B3EB62520ED44FEAC12343F064
:109A3000004343EA505323FA02F070474FF000000E
:109A4000704750EA013002D14FF0FF3070474FF0BD
:109A50000000704719481A49026800608A4217D00E
:109A6000002103E0174B5B58435004311648174B55
:109A700042189A42F6D3164A02E0002342F8043B09
:109A8000144B9A42F9D3FAF76DFE00F033F8FEE773
:109A9000114E4FF0090030601048016821F07061EC
:109AA0000160410201600E4C182020600D490E48F3
:109AB00008600E48D0F800D040680047F04F002002
:109AC000EFBEADDE00DC000800000020A800002092
:109AD000A80000206C18002018100240040001406B
:109AE000140C0140000C01404434434400F0FF1FBB
:109AF000FEE700002DE980488FB0F6F709FB714CB6
:109B00002379256833B1A368EB1A002BA2BF002389
:109B1000237123736C4B1E6842F20103334008BF6C
:109B20006373330740F12781684B1B681B7A062B50
:109B30000BD8DFE813F0070007003300DF00A601B1
:109B4000D101D101624B1A780AB90023FFE000224B
:109B50001A7002225F4B604993F800E05F4BDFF818
:109B600090911B6893F800C05D4B93F800808B5C6C
:109B7000501C43FA0EF303F00F03634509D20B2B7D
:109B800007D88F5C085C07EA080700EB072049F854
:109B900023000232102AEAD10123D8E0514B1A786F
:109BA000002AD2D000221A704F4B504A9978587828
:109BB00001F0070740EA0720DF78106007F03F0058
:109BC000400140EAD10019795060890041EA9711BB
:109BD0005F7993F809E007F0010041EA8021916084
:109BE000997901F00F00C00140EA5700DF79D06099
:109BF00007F07F00000140EA1110197A1061490056
:109C00000EF0030041EAD71141EA40219F7A5161E9
:109C1000D97A07F01F00C90041EA5711800140EAD4
:109C20009E00D161597B9061187B01F0070740EAE3
:109C300007209F7B106207F03F00400140EAD100FF
:109C4000D97B5062890041EA97111F7C07F001001F
:109C500041EA80219162597C01F00F00C00140EA85
:109C600057009F7CD06207F07F00000140EA11108E
:109C70001063D97C93F814E0490041EAD7110EF043
:109C8000030041EA40215163997D5F7DDB7DC9007E
:109C900041EA571107F01F00DF07D1634CBF40F2C4
:109CA0001471AD21800140EA9E0090639807116411
:109CB0004CBF40F21471AD21516419077FF56CAFB0
:109CC000032344E0A800002000160020FC1500201B
:109CD00089150020860D002079150020800D0020B8
:109CE000870D0020F6150020DD150020F01400205F
:109CF000801400207C4A1378002B3FF426AF002309
:109D000013707A4A7A4910787A4FB1F800E007EB7D
:109D1000400191F803C0097941EA0C218E457FF496
:109D200014AF7978012900F0A08081290FD1032395
:109D3000102884BF10211170177800226E49DFF8B7
:109D4000ECE1D0B2874201F1020100F29080DA0723
:109D500011D5012203F00203002B14BF1346002388
:109D60006273664A13700CBF01230023237105F54B
:109D7000C333A033A360730410D5614A13780BB1C9
:109D80000021117063734BB10123237100235B4ADF
:109D9000137005F5F42303F59073A360F7070DD551
:109DA000A27BE37B934209D0012323730023534911
:109DB000E2734B7005F5C333A033A360B60409D535
:109DC0000023504A32F81310002942F05081013329
:109DD0000C2BF7D14C4B1B7858072ED54B4AB2F9B8
:109DE000001081EAE173A3EBE173B3F52F7F1BDC75
:109DF000B2F9022082EAE273A3EBE273B3F52F7F9C
:109E000012DC4349B1F9002082EAE273A3EBE2736A
:109E100041F28832934207DCB1F9021081EAE17322
:109E2000A3EBE173934208DD3A4B1B88012B04D866
:109E30004022394B1A70FEF7D9FBFDF7FBFE2F4B82
:109E400005465B68C31A632B40F38380324B187856
:109E5000FDF7C5FF062879D8DFE810F0F0006E00A6
:109E6000EA0010011901FB0004010B4660E711F83C
:109E700002CC11F8010C40EA0C202EF8120001323D
:109E80005FE7264B1A78002A3FF45FAE00221A7073
:109E9000234B1A789A46A82A7FF457AEDF7C002F0E
:109EA0007FF453AEDFF88890DFF888800AEB070371
:109EB000D8781B7903EB0020FFF738F91949FFF731
:109EC00041FA4146FFF780F8FFF78AFB49F817008F
:109ED0000237102FEAD15FE6134B1A78002A3FF4BD
:109EE00034AE00221A7057E6AD150020B0150020E0
:109EF000AE150020B1150020B41500200000002090
:109F0000381600205C15002034160020B80D002003
:109F1000BE0700208A0D002025000020A615002085
:109F200091150020CDCCCC40F8150020D014002095
:109F3000B01400200080BB434FF48042574B5A615D
:109F40004FF400521A614FF400421A61544B6435C9
:109F50005D60637B206823B92369C31A002BC0F2BC
:109F6000938600F59C43203323614E4B1E78002ED0
:109F700040F0AC804C4FDFF83C91DFF84CA197F8F3
:109F80000080F5B24545C0F0A88242F20102474B7D
:109F900047491B68096813400391059305D0237B4B
:109FA0003F4A23713E4B5B78137026791EB13C4BC0
:109FB0001E7886F001060F2384F838303D4B94F864
:109FC00039901B68002504930323B9FBF3F303EBDB
:109FD0004303A9EB0303DBB25B000693364B039A02
:109FE00003F1280B012302F51672DFF8D8A00792BF
:109FF0000BF148024545C0F2A58294F838302C4A4E
:10A000000F2B2E4B40F0F5822D490968490100F1D4
:10A01000F0821268D9689A60521AC82A02D90122BD
:10A0200083F8212094F83930013384F8393053E033
:10A030001A4BDA6882F48042DA6081E74FF480429A
:10A04000164B5A614FF400525A614FF400425A6164
:10A050007CE74FF48042114B1A61DA6882F40052B7
:10A06000DA6006E04FF480420C4B1A614FF4005264
:10A070001A61DA6882F40042DA6067E74FF48042DE
:10A08000064B1A61DA6882F40052DA605BE7034B30
:10A09000DA6882F48042DA60DFE700BF0010014036
:10A0A0000000002008160020840D0020001600206B
:10A0B000C40D0020FC150020BC0000200C16002060
:10A0C0008C0D0020900D00202C000020B24A126858
:10A0D000904201D9013E1E70B04B1B68DA0405D5D1
:10A0E000AF4B1B68DB0701D4FEF780FAAD4B256848
:10A0F0001968887A002800F09782AB4A0B7B0138F8
:10A1000032F910001BB1C0F53B60083000B2A0F579
:10A110007A70B0F57A7FA8BF4FF47A7020EAE070C9
:10A12000FFF708F8A149FFF70DF9A149FFF756F825
:10A13000FFF756FA9F4B1880984B1B68DE050BD52E
:10A140009D4B9D429D4B03D99A780AB901229A7082
:10A150009B780BB1F8F784FD994DB5F8DE1005F545
:10A160008B70FDF72DFB814668B9F8F74DFD002295
:10A17000944BC3F80090C3F80490C3F80890924B36
:10A180001A605A609A60914E3378580721D5834BF4
:10A190001B68D9061DD58E4B1B78DA0619D48D4B5A
:10A1A0001B78002B00F08C8295F86E31B9F1000F0E
:10A1B00040F07482002B00F08682874B1A68874B30
:10A1C0001B689B1A002B80F27E82FEF70FFA84F840
:10A1D000FD900022134695F86CA195F86D01B5F835
:10A1E00026E1B5F828C1704F37F912109B08714568
:10A1F000C4BF63F07F03DBB201326145B8BF43F0F7
:10A200004003042AF0D194F8FE209A4240F0628282
:10A2100094F8FF20F92A02D8013284F8FF20DFF8F1
:10A22000B48184F8FE3098F8003063B95C4B1B6849
:10A23000DB0740F15182B9F1000F04D13378D80720
:10A2400001D5F9F73FF894F8FF30DFF8B091142BFF
:10A2500034D198F80030C3B194F8FE305F2B06D1AA
:10A26000337813F0040B00F06B82FEF7BFF9BAF1FC
:10A27000000F0AD094F8FE307D2B06D1337813F00E
:10A28000040B00F06382FEF7B1F9337813F0040297
:10A2900014D194F8FE30572B40F05E824FF47A735D
:10A2A000A4F800314E4B1B685A0742BF0A214D4AA1
:10A2B000118013F0080301D14B4A1380374BDFF8AC
:10A2C000E0801B6813F0040F25D094F8023193B19D
:10A2D000337859070FD5B7F90620B5F826319A42D9
:10A2E00009DDD8F8003013F0010301BF32213F4AE5
:10A2F00084F802311180D8F80030DA0340F19882F6
:10A300003B4B1A782AB93B4A127812B93221374AA4
:10A31000118001221A7000234FF0010AD9F8007051
:10A32000C8F8003007F17B0607F1CB093278737863
:10A330009A420ED2314616F8010CFDF71FFA40B1D1
:10A3400016F8023CD8F800200AFA03F31343C8F8C1
:10A3500000300436B145E9D14FF00C094FF0000A46
:10A360004FF0010BDFF8988007F1C90607F21117CB
:10A370007278B3789A425CD2711C3078FDF7FEF99E
:10A38000002856D01C4A7179F37809FB0120013B63
:10A3900003EB430336E000BF041600200016002044
:10A3A0008C0D0020FC150020900D002000007A4448
:10A3B00000C07F44F4070020404B4C000C160020E6
:10A3C00064080020EC1200205C13002034160020EA
:10A3D0005A16002028000020C40D002090070020FD
:10A3E0009C07002048070020E8070020AA0E002054
:10A3F000CE0E0020CF0E0020A80000203C1600202A
:10A40000A2D50008D0F808214344934296F804E00E
:10A410000FD0C0F80831BB4B0BFA01F193F834317F
:10A4200080F804E123EA0101B64BC0F80CA183F8DF
:10A4300034110636B7429BD1B34B4FF000089B4610
:10A440001A68B24F0392B24AA7F58276D2F800A0FA
:10A45000227904927A68002A00F00A821178002991
:10A4600000F00682BB68AAEB0303002B0BDB0AF5A6
:10A47000FA73BB60012303FA08F096F8343123EA3B
:10A48000000386F83431049B002B00F0F1813B7807
:10A4900050780433DBB2002840F00F829D4830F939
:10A4A00013009D4BB3F8243103F1C80E704540F3FF
:10A4B000CD81927896F8343143FA08F3DB0700F146
:10A4C000D7810398FDF7E4F9012396F8342103FAC4
:10A4D00008F3134386F83431CAE1072D96BFD9F843
:10A4E00000302946595D3846DAF800309847032D88
:10A4F000034621D8D9F8002002EB8501C86B0A90E9
:10A50000D3B105F10F0002EB800132F82020981A38
:10A510004FF47A7358434B889B1A90FBF3F040F248
:10A52000EE2300F57A709842B8BF184640F6CA0389
:10A530009842A8BF184683B2724A013602EB45051D
:10A54000AB821CE54FEA450EC6B1744931F91500DE
:10A55000049980B2898A814203D80499C98A8142C8
:10A5600021D25BF825100398814209D93AF80E00F0
:10A570000599E1B92AF8150001353BE53046E7E7D2
:10A58000E8B209920893FBF7ABFF032D089B099AE9
:10A59000EEDC5C4F03FA05F197F838E02EEA010192
:10A5A00087F83810E4E707994BF82510E0E7062113
:10A5B0006943069F02EB010E2EF80700514F97F8F2
:10A5C000CCC0BCF1000F04D1B9F1020FD2D987F889
:10A5D000CC30515ABEF802000844BEF804100844BA
:10A5E0004F4900B221F81500032190FBF1F080B231
:10A5F000C0E701214B481268417001709968DA6028
:10A60000521A596800258A4288BF0022414E88BFED
:10A6100083F82120A8457FF705ADE8B2FBF760FF7E
:10A6200026F815000135F5E73F4B1B681F047FF541
:10A6300083ADD4F8E830EB1A002BFFF67DAD05F5BD
:10A640009C432033C4F8E830384B5A79384B33F800
:10A650001220CB7A92B292FBF3F294F8EC302949B3
:10A66000013303F00F0384F8EC300B4483F8ED2042
:10A670000346ED315A5C01331044102B00B2F9D17E
:10A6800090FBF3F000B2002806DB6428A8BF64202A
:10A69000FEF750FD274946E50020F9E73BB14FF4AE
:10A6A0007A711B4A126801FB0323234A136094F852
:10A6B000FD30002B3FF48DADFDF7A0F8002306E040
:10A6C000B9F1000FF3D11020FDF7A2F8012384F8AF
:10A6D000FD307EE50022A0E5337859077FF5B3AD64
:10A6E0002379002B3FF4AFAD144BDB78002B7FF4C4
:10A6F000AAAD10B1FDF77AFFA5E5B9F1000F7FF41F
:10A70000A2ADF7E7A8000020BC0D0020AC0100209E
:10A71000C40D0020900D002064080020BC00002023
:10A72000760100200000002000160020000E00200E
:10A73000100E00200000C842900700200C160020D8
:10A740000B20FDF765F884F8FFB090E50B20FDF7CE
:10A750005FF884F8FFB098E574490968480716D592
:10A760005A2B14D1724B197821B11A700122714BF6
:10A770001A70A3E594F8023183F0010384F80231E2
:10A780001BB10C20FDF744F898E50D20FAE75D2B8E
:10A7900001F078845B2B01F085845E2B41F084848A
:10A7A000032001F070BCBAF1000F02D07E2B01F043
:10A7B0008B8498F8FE30972B04D14FF4C8725E4B0F
:10A7C0001A807BE5A72B05D15C4A137843F004037C
:10A7D000137073E50022BB2B0B9218D10223ADF846
:10A7E0002E30D9F80020BDF82C10B2F858300B44A8
:10A7F000A2F85830BDF82E10B2F85A300B44A2F827
:10A800005A30FDF7E9FE002388F8FF3056E5B72BF4
:10A8100002D14FF6FE73E2E7BE2B03D10223ADF85F
:10A820002C30DEE7BD2B7FF449AD4FF6FE73F6E723
:10A830003F4A1378002B3FF46EAD337813F00403D6
:10A840007FF469AD137001223A4B63E5C83B98422F
:10A8500002DA927852422DE6012303FA08F296F8C2
:10A86000343123EA020386F834310AF5FA73BB6007
:10A8700008F10108B8F1040F07F10C077FF4EAAD05
:10A880002F4E304F336813F0020F07D1274B1B6850
:10A89000D80561D52C4BDB78002B5DD03B68990740
:10A8A0005AD52A4B1B8813F0010804D1F8F7ACF9EC
:10A8B0000120FDF709FC002352E001287FF404AEDB
:10A8C0000C297FF401AE2248927830F9130040F64B
:10A8D00033039842A8BF18464FF49663B0F5617FE2
:10A8E000B8BF4FF4617093FBF2F3A0F5617090FB79
:10A8F000F3F096F835315FFA80F94B453FF4E4AD5B
:10A90000B9F1030F94BF4B460223124A86F8353142
:10A9100001FB032303F2EE43CBF80030FDF7F2FB1B
:10A9200009F10100C0B2FCF797FFCDE50016002049
:10A93000CF0E0020D00E0020581600205A160020FE
:10A940008C0D00209C0700200C160020A007002082
:10A95000900D0020640800200120FDF7A6FB0123D4
:10A960003268520740F15781002B00F054810120DA
:10A97000FDF79BFBAF4B1B889B0704D4F8F744F90A
:10A980000220FDF7A1FB3B6813F00A0F20D03368CB
:10A99000D80640F14481A74B1B88590706D40420F0
:10A9A000FDF792FBA44B1A88A44B1A8033689A06D1
:10A9B00040F139819F4B1B885B0602D44020FDF794
:10A9C00083FB3368580641BF9B4B1A889C4B1A8007
:10A9D00033684FF48070190540F12981FDF774FB4D
:10A9E0006B79082B01D00E2B02D14020FDF75DFBC7
:10A9F0000122944B83F8362193F8373123B13B6819
:10AA00005A0701D5F8F736FCFDF71AF98E4B20608E
:10AA10009B892BB1D4F86021821A002AFFF66FA817
:10AA20008A4D0344C4F860312B6889480393894BED
:10AA30005B6898470595002840F0CD81864B874D8F
:10AA40001B6813F0020300F00684D4F8C0312846D6
:10AA50009847002861D0824F94F8C821294628469B
:10AA6000F9F7A6FE3B887F4E002B41D000231A4603
:10AA70003068DFF80CE239884FEA830CB1F5C87F03
:10AA800008BF4EF8232035F913805EF80C1025F826
:10AA9000132041444EF80C1020F813200133032BEF
:10AAA000E9D16F4F3B88012B1FD14FF4C87ED4F8FA
:10AAB000CC31C83393FBFEF30380D4F8D011C831F6
:10AAC00091FBFEF14180D4F8D431C83393FBFEFEF4
:10AAD000654B1B88AEEB030E039BA0F804E0A3F8C4
:10AAE0005820A3F85A20FDF777FD3B88013B3B80B7
:10AAF0005E4B1B68580703D503985830FAF738F8AF
:10AB000032682B8811885B1A2B8051886B885B1AFE
:10AB10006B809288AB889B1AAB80FDF791F8002779
:10AB20000546D4F8D8614FF07E5B861B3046FEF7B1
:10AB3000FDFAD4F8DC11FEF751FBC4F8D8513D46BC
:10AB40004B4BDFF840811B68DFF810A11B780490A5
:10AB500003930DF12C096B0006933D4B33F915005F
:10AB6000FEF7E8FA0499FEF739FB039B49F8250044
:10AB7000002B00F0DB811846FEF7DCFA0146584650
:10AB8000FEF7E0FB014607905846FEF71DFA394BE9
:10AB900053F82510FEF722FB06903AF91500FEF750
:10ABA000C9FA079B1946FEF719FB069A014610469B
:10ABB000FEF70CFA2F4B43F82500FEF7EBFC28F8C4
:10ABC00015006B0033F908300135032D03FB0377C3
:10ABD000C1D164235F43244B0BA91B8826485B43E8
:10ABE00097FBF3F7493FBFB2FDF70CFA3B2F40F25A
:10ABF000A281B4F9F801FEF79DFAD4F8F4510146A8
:10AC00002846FEF7A7FC1D4B002840F0DB811A7890
:10AC100022F00802D9E10220FDF747FAB3E604204A
:10AC2000FDF743FAC2E64020FDF73FFAC9E6FDF71B
:10AC30003CFAD5E6A0070020E807002036160020E1
:10AC40008E070020A8000020640800203C16002089
:10AC5000C4070020040700209C070020C80E002025
:10AC600058160020AC0E00203A00002000160020EC
:10AC70005814002088020020940200205A16002058
:10AC800074020020BE070020D4F838516B1C012D3F
:10AC9000C4F8383100F08A80022D00F08F80002D3A
:10ACA00069D1BA4B1B681B077FF5AEAED4F83C31B7
:10ACB000C31A002BFFF6A8AE00F5C330A030C4F8CD
:10ACC0003C01D4F84431B2489847B14994F848213E
:10ACD0000846F9F76DFDAF490A78570718D5D4F83B
:10ACE0003C31AC46C4F84C312B46AB4DAB4EDFF893
:10ACF000A0E2AF1D3EF9130026F802CF25F813009D
:10AD000027F813000133032BF4D122F004020A7058
:10AD100094F85C3183B19E4AA1491388B1F80201CD
:10AD20001B1A1380B1F804015388B1F806111B1ADD
:10AD3000538093885B1A9380D4F84C21DAB1D4F80D
:10AD40003C3195499B1A974A881D93424FF0000366
:10AD500019D88F4E36F9132031F913705D009742E0
:10AD6000475FC8BF21F81320974203F10103B8BF22
:10AD70004253032BEED1D4F83831032BC4BF002348
:10AD8000C4F8383140E60226844DC4F84C3131F91C
:10AD9000132030F9137001333A4492FBF6F2032B7F
:10ADA00025F8022FF3D1FDF717FCE4E7774B1B687A
:10ADB0005E077FF529AEFCF7F1FADCE7734B1B6801
:10ADC0005D077FF521AE94F85D31002B3FF41CAE9A
:10ADD000F8F742F8CFE7744994F864210846F9F788
:10ADE000E7FCB4F80031002B50D00027BA46D4F865
:10ADF00068316E4E1B7806F10C0504936C4BB3F86A
:10AE000000917B00B9F57A7F0693674B08BFC6F8BF
:10AE100000A033F91700336808BFC5F810A0034439
:10AE20003360FEF787F92A6902F10108B8F1010FD2
:10AE3000C5F8108038D1002368602860AB605A4B99
:10AE4000DFF870817A00B9F1010F22F803A022F82F
:10AE500008A059D1286901284ADD0138FEF76AF9AE
:10AE60000146E868FEF76EFA01F04EFB049B83464C
:10AE7000002B3FD01846FEF75DF95946FEF74CFB14
:10AE8000002837D04FF47A73A4F8003100234649E4
:10AE9000484D31F8132035F81300121A21F8132009
:10AEA0000133032BF5D1C9E52A68079011460692B4
:10AEB000FEF78AF883464046FEF73CF901465846BD
:10AEC000FEF740FA069A1146FEF780F8079B014606
:10AED000804668601846FEF777F85946FEF77EF917
:10AEE000A968FEF773F8C5F80080E860A860A6E7D7
:10AEF0000020B9E74FF47A72336803F5FA7393FBD5
:10AF0000F2F37A0028F802300137032F06F1040625
:10AF100005F114057FF472AFB9F1010F02D1484673
:10AF2000FCF776FCB4F80031013BADE73AF8153098
:10AF300028F8153045E6204B4FF07E511B684FF046
:10AF4000000A5F681D4D3846FEF740F801464FF095
:10AF50007E50FEF7F7F98046194B33F91A00FEF7D9
:10AF6000E9F855F82A1083463846FEF737F90146C6
:10AF70005846FEF72BF84146FEF730F945F82A000F
:10AF80000AF1010ABAF1030FE6D132E69C0700206C
:10AF9000CA0700205A160020F8010020640900208A
:10AFA000640800207FC3C901C407002014020020E8
:10AFB000A80000205C020020581400209402002009
:10AFC000BE0700201A7842F008022946D4F8F001A2
:10AFD0001A7001F017F9B14DD4F8F0112860084645
:10AFE000FEF7FCF8D4F8F4A1804651465046FEF72F
:10AFF000F5F801464046FDF7E9FFD4F8EC7101F0A1
:10B0000083FA07F100470146384601F0FBF8A449EE
:10B0100068602868FEF7E2F801F06AF8A14FA049DD
:10B0200038806868FEF7DAF801F062F89E4B7880A5
:10B030001B68190740F1D2800BA99C48FCF7E2FF7E
:10B040009B4B4FF07E511B680025D3F80880974F2B
:10B050004046FDF7BBFF01464FF07E50FEF772F908
:10B060008146DFF88CB23BF91500FEF763F857F81C
:10B07000251082464046FEF7B1F801465046FDF7DE
:10B08000A5FF4946FEF7AAF847F825000135032D2C
:10B09000E9D18648FAF774FF864B18803046FAF7F4
:10B0A000DDFFFCF7CDFDD4F808322060824AC4F8F9
:10B0B0000802824CC31A1380236893F85230002B85
:10B0C00040F0CD807E4BB3F906007E4B1F687B8934
:10B0D0009842C0F2DE80B0F5FA6FFA79BFBFC61AA7
:10B0E0005643C3F5FA6396FBF3F6ACBFC2F16406B0
:10B0F000C6F16406744B2268B3F824E193F9EE308C
:10B1000000215B429BB206931346642501336F4CCA
:10B110000492059340F2E632694B4FEA410833F955
:10B1200011C0ACEB0E0303F2F319914500F2B380AA
:10B13000002BB8BF5B4202290393049B00F0DC8024
:10B1400093F811212AB1039B9A42ACBF00239B1AAA
:10B150000393039B6FF0630B93FBF5F25C4B02F1DF
:10B16000010933F912A033F91990039BA9EB0A09DD
:10B170000BFB023202FB09F292FBF5F2524424F877
:10B1800008207A1812795343524A93FBF2F364333E
:10B190009BB2734393FBF5F9059B022913F8012B2E
:10B1A00009FB02F292FBF5F205934B4B5A54059BB7
:10B1B000DA7C09FB02F393FBF5F3484A5354484BFE
:10B1C00040F0C880F4459D70C0F2C7803E4FB7F88C
:10B1D0002621904280F2CB801046CDE0494641487E
:10B1E000FCF710FF404B9B68039303993E4B0846C6
:10B1F000D3F80C801F69FDF7F1FF41460546404634
:10B20000FDF7ECFF01462846FDF7E0FE394605460E
:10B210003846FDF7E3FF01462846FDF7D7FE01F06B
:10B2200073F900210546FEF76DF990B92E4B2946BA
:10B230009868FEF787F82C4B29469860D868FEF787
:10B2400081F8294B2946D8601869FEF77BF8264B10
:10B25000186124481EE72B806B80AB8021E7002516
:10B26000224EDFF89080059BB6F902001B6808EBC0
:10B27000050793F85290FDF75DFF4A463946FCF703
:10B2800075FDFEF787F904350C2D26F8020FEAD17B
:10B2900018E764262EE74FF4FA734CE750140020A9
:10B2A0004C3D0F44B80D00209C070020A402002054
:10B2B00058140020E8070020541800203C160020F5
:10B2C000900D0020BC0D002064080020D412002046
:10B2D0001C1800200CFEFFFF381300205013002024
:10B2E000DC1200200800002000000020C20700201F
:10B2F000CA070020B402002093F812212AB1039B50
:10B300009342D4BF00239B1A0393039B6FF0630BFC
:10B3100093FBF5F2BD4B03EB4209039BB9F918A26D
:10B320000BFB0232B9F91A92069BA9EB0A0902FB40
:10B3300009F292FBF5F252445A43039BA280BA7978
:10B34000002BB8BF5B425343B14A93FBF2F303F1C6
:10B35000640921E7F4455E5404DA34F808305B42AE
:10B3600024F80830013103297FF4D4AE2EE7B0F57C
:10B37000FA6FA8BF4FF4FA604FF47A73801A5843FB
:10B38000C2F5FA62B0FBF2F0642690FBF6F2A14B34
:10B39000511C33F9125033F911106FF0630303FBA2
:10B3A0000203491B4B4393FBF6F32B44E3809A4B78
:10B3B0001B885A063ED5994B1888994B1B88C01A92
:10B3C00000B2FDF7B7FE9749FDF708FF964905461D
:10B3D000FDF7FCFDFCF720FD80462846FCF71CFD30
:10B3E0000546B4F90200FDF7A5FE0646B4F90000D3
:10B3F000FDF7A0FE41468146FDF7F0FE314682464C
:10B400002846FDF7EBFE01465046FDF7DDFDFEF751
:10B41000C1F8414620803046FDF7E0FE4946064629
:10B420002846FDF7DBFE01463046FDF7CFFDFEF76F
:10B43000B1F860807D4B7E4E1B687E4D13F0020F8D
:10B4400041D045F20721DFF8C481D8F80020D8F8B0
:10B450002832D31A8B4236DDC8F82822F9F786FA4B
:10B4600098F82C32DFF8EC91032BB9F8003040F05B
:10B47000A2800A2B1DD90023282088F82C32FCF743
:10B4800006FCF9F773FA6C4B1888F9F74FFA6B4B17
:10B490001A68D37890FBF3F001300828A8BF082081
:10B4A000537980B24343A8F82E3213795843A8F851
:10B4B000300298F82C32012B00F09780C0F0878082
:10B4C000022B00F0E880594B1A68130537D54F4915
:10B4D000D1F834020B68A3EB000B45F2072083453B
:10B4E0002DDDC1F83432554BB4F90680D3F800A0F5
:10B4F000A8F57A789AF80A30DFF85C91012B00F011
:10B50000D380C0F01E81022B00F0F280D9F8003009
:10B510004B4A03FB0BFB4FF47A739BFBF3FB494B4A
:10B52000D3E9000110EB0B0841EBEB79C3E900898B
:10B53000404600234946FEF773F8434B1860DFF896
:10B540001C91D9F80030D80402D50A20FCF760F924
:10B550003E4B1968002900F0FD80DFF804B1DFF8E8
:10B5600004A1DBF80000DAF80020824200F2F28049
:10B57000374ADFF8F4801078002840F0E48001209A
:10B580001070B8F800004A68125C42B138B90A7805
:10B59000053A012A03D80393FCF752FB039B1B686F
:10B5A000B8F800105B685A5CFE2A40F0CF80002398
:10B5B000A8F80030CEE00A2B3FF67BAF032388F8D3
:10B5C0002C320023A8F82E32A8F8303271E7B8F8F0
:10B5D0002E22B9F800309A427FF775AF0123082078
:10B5E00088F82C32FCF714F96DE73378B9F80020AD
:10B5F00023F002033370B8F83032934236DD022371
:10B60000072088F82C32FCF703F937E0A800002067
:10B610000CFEFFFF04180020A0070020E807002010
:10B620008E07002035FA8E3CDB0FC93F0016002044
:10B630003416002025000020180E0020FC0D0020EC
:10B64000407E0500E8020020F007002034180020AA
:10B650002A180020A80E0020F80700208C0D0020DA
:10B66000C40D00202C18002030180020B8F82E320D
:10B6700001339A420DDD002388F82C32854B1B885C
:10B68000B3F5A67F3FF61FAFF7F7CCFA10232B7068
:10B6900019E70820B7E7B8F83032B9F800200133CD
:10B6A0009A429BDC07209DE77B4AD1F83832507BD9
:10B6B0007A4A32F81020082093FBF0FE92B2A3EBF6
:10B6C0000E031A44C1F8382292FBF0F240F6E4402F
:10B6D00092B25043BAF80820BAF90630C2EB1030E3
:10B6E0004FF47A72424392FBF3F2C9F800200DE75F
:10B6F0003078BAF808304007B7F8DE10C9F80030E3
:10B700007FF504AF664804930392FCF759F8039A57
:10B71000049B20B912F0100F18BF4FF0000832211F
:10B7200008FB08F292FBF1F24244BAF9068008FBEA
:10B7300002F84FF47A7298FBF2F84344C9F80030EB
:10B74000E4E60023FAE70021117028E7FF2A36D14A
:10B75000FCF754F832782B78510739D543F00103C0
:10B760002B700025DFF8549109EB050393F84A206C
:10B77000012A40F0FE80DFF848814A4AC2469346DB
:10B78000C8F8003059F805301360DBF80000036892
:10B790005B689847002800F0C280DBF8000003686F
:10B7A000DB689847DAF8003093F8481000294DD14B
:10B7B000242840F08B82012183F8481096E00A206B
:10B7C000DBF8003000FB0233CAF800304B1CEFE618
:10B7D00023F001012970D9F80010C8071FD432499D
:10B7E0000978090755BF23F0030323F0050343F04D
:10B7F000040343F002032B70264B58BF22F00102D2
:10B800001B884ABF42F0010232703270B3F5AA7F42
:10B810002B788CBF23F0400343F040032B70234B65
:10B820001B685D0702D5224A128842B9214A128854
:10B830000AB1980703D4204BB3F800311BB1337819
:10B8400023F001033370FCF7FBF98AE7012905D1E6
:10B850004D2808BF022118BF0021ADE7022903D1FE
:10B860003C2808BF0321F6E7032909D1002140281D
:10B870009FBF1971D9715871987198BF04219BE7C6
:10B8800004291FD1997983F849004840987105210E
:10B8900092E700BFB40D0020000E0020100E002023
:10B8A0007A090020940700205A1600209C070020E7
:10B8B0004807002058160020A8000020F0020020B1
:10B8C00030160020052911D193F805E019798E452D
:10B8D00093F806E040F2F48180EA0E0E83F806E069
:10B8E00001F1010E194483F804E0087293F848103E
:10B8F00006297FF44AAF93F84900F7F772FD20B9A3
:10B90000FAF742FE08B9F8F769FCD8F800309879E0
:10B91000F7F722FD0022D8F8003083F84820BC4B0E
:10B920001B7833B359F80580D8F8003040465B697E
:10B930009847002800F0DB81FAF7FCFAB54BB648CF
:10B94000197800239E46DAB2914200F2D481322067
:10B95000FCF79DF9B14B1B685A0307D5B04B9B68A8
:10B960005B0303D440F2DC50FCF791F9AD4AAE4BD7
:10B97000DA604C35982D7FF4F5AEAC4B9B680BB17B
:10B98000AB48984797F82331AA4E002B52D0AA4BC8
:10B99000B6F8E2521888FDF7C9FB06F539710122A5
:10B9A000FCF7E4F9FDF71CFE80B2B5FBF0F096F869
:10B9B0003631411C09B2A6F8E812002B00F0A28132
:10B9C0000023B6F9EA9206F53B7806F53D7E38F994
:10B9D000132034F913C009FB02F292FBF1F23EF896
:10B9E00013502EF813C0ACEB05052A4428F8132099
:10B9F0000133042BEBD10023A6F8EA0286F8363196
:10BA00008C4A0023B2F9EA52002D40F38181B2F949
:10BA1000E8C202F53D7E02F53B7232F913103EF8A2
:10BA20001300694391FBFCF1411A24F81310013310
:10BA3000042BF2D101237F4DDFF8348285F83731B2
:10BA40007E4B196811F0080F3BD0A3887C4803F1A6
:10BA5000450292B28A2ADFF81CC200F25C81794A60
:10BA6000B2F800E01EF0040F00F055810088BCF829
:10BA70000020821A92B20FFA82FE1EF1B30FBCBFF1
:10BA800002F5B4720FFA82FEBEF1B30FC4BFAEF579
:10BA9000B4720FFA82FE6C4A1278100711D597F92A
:10BAA000EE00D8F80020404200FB0EF092F809E0CA
:10BAB00002B26FF01D0002FB0EF292FBF0F2134493
:10BAC000A38011F0140F12D05E4B1B8803F4027395
:10BAD0006BB15D4B197811F0100100F020815B4BC8
:10BAE000628897F974111B6801FB03236380584B2C
:10BAF0001B7843B1574BB3F90620B7F826319A4269
:10BB0000DCBF0023A380D8F8003093F818A1BAF165
:10BB1000000F4FD04B4B1B889A074BD0D6F8EC1137
:10BB2000D6F8F03108460393FDF758FB039B834694
:10BB300019461846FDF752FB01465846FDF746FAEE
:10BB4000D6F8F491834649464846FDF747FB01463F
:10BB50005846FDF73BFA00F0D7FC01464846FDF792
:10BB6000F1FB3D498146FDF7E1FC002840F064818E
:10BB7000484600F0F7FAD6F80813FDF72FFB00F05F
:10BB8000B7FAB0F5617FA8BF4FF46170FDF7D2FA44
:10BB90003249FDF7D7FBFCF73FF906465046FDF763
:10BBA000C9FA3146FDF71AFB00F0A2FA00B2E388A9
:10BBB0001844E0802A4BD8F80000B7F8FA20294949
:10BBC0000093294B09681E6800F15803B047114BD8
:10BBD00026491E78032E4FD9D5F80C33B3F802E06E
:10BBE000BEF5FA7F48D2B4F90430B1F9047083EAA3
:10BBF000E370A0EBE370CEF10002131A9F4204DB66
:10BC00000EEB0003BB42A8BF3B468B8034E000BF75
:10BC10006016002053130020781300200016002027
:10BC2000640800200400FA0500ED00E0040700208D
:10BC300088030020A8000020541800209C07002042
:10BC4000E8070020A00700205A16002084070020E3
:10BC500028000020900D00208FC2753CEFB6B04444
:10BC60007A090020BC0D00203C0000202813002091
:10BC70003C160020361600200027D5F80C33B4F906
:10BC800006800393B1F90290B1F900A0B1F904B0B4
:10BC9000AD4CAE4BB74204F11004C0F0CF80AC4BBA
:10BCA0001B7813F0040340F00481A84AA9499E427E
:10BCB00040F2258131F8130022F813000133F6E732
:10BCC000864501D1062177E5002175E531784907E0
:10BCD0003FF50CAEA0490968097881427FF406AEB1
:10BCE0009E4A9F4911609F499F4ACA60FEE50A200B
:10BCF000FBF7CDFF18E650F8232001331268A2F8B5
:10BD000000E020E6B6F8EA32013BA6F8EA3277E630
:10BD1000A2F8EA328EE60388ACF80030D1E6D5F816
:10BD2000FC02924A90F803E0914B8078BEF1000F3C
:10BD300040D0B2F906E0B3F90020AEEB020383EA8B
:10BD4000E37CACEBE37C844519DD012285F800231C
:10BD500040F24B4296450FDD062293FBF2F3502B47
:10BD6000A8BF50236FF04F01B5F802238B42ACBF40
:10BD7000D3185318E380BAE640F27E43FAE795F809
:10BD800000332BB17B4B85F8001318687A4B186091
:10BD90007A4BD5F804131B681A440B8849889A42D9
:10BDA00003DB91420B46A8BF13461BB2E380A5F804
:10BDB00002339CE6B2F90620B3F90010531A83EA65
:10BDC000E37CACEBE37C844525DD062093FBF0F3BC
:10BDD000782BA8BF78236FF0770E69487345ACBF06
:10BDE0000360C0F800E00123664885F80033037063
:10BDF000624BD5F804031B681944038840889942B4
:10BE000003DB88420346A8BF0B4640F27D418A42CD
:10BE1000B0DCE2806BE695F80033002BE8D001201F
:10BE2000574B85F800E3C3F800E0564B1870514BB0
:10BE30001868514B1860DBE70020B8E640460593D0
:10BE4000FDF778F954F8101CFDF7C8F9049048463E
:10BE5000FDF770F954F8081CFDF7C0F9049A014683
:10BE60001046FDF7B3F804905046FDF763F954F817
:10BE70000C1CFDF7B3F9049A01461046FDF7A6F82D
:10BE8000039B049093F9010040420BFB00F0FDF787
:10BE900051F954F8041CFDF7A1F9049A0146104623
:10BEA000FDF794F8FDF776FB059B23F817000137A3
:10BEB000F0E60122344BDB780493244BB3F90010F5
:10BEC000964239D8314A294C1068B4F90670428834
:10BED00003EB46039142D4BF0021891A2C4AD5F8BE
:10BEE000D0831268C8BF89B202F4805B02F0100EE2
:10BEF000284A05931468154A059B93424ED195F83C
:10BF0000D4330BB1F9F7BEFF184BB3F90A2040F256
:10BF1000A4639A4240F39980F8F764F995F83731B1
:10BF2000002B3DF4ECAD1C4B1B685B077DF5E7ADCA
:10BF3000F7F7A0F9FDF7E3BD33F9120001328142B2
:10BF4000B8BF0146BCE700BFB8030020D0070020FF
:10BF500034160020401600205C160020F04F002010
:10BF6000EFBEADDE00ED00E00400FA05900D00200C
:10BF70008C070020EC0700207407002084070020B5
:10BF80007C070020240000200C1600204C14002008
:10BF900000160020481400209C07002013885B1A1C
:10BFA0001BB222F8023BBBF1000F2CD0039E96F887
:10BFB00000C0BCF1000F0AD1B8F80E90B4F806C06A
:10BFC000A9EB0C0ABA4502DACC44BC4514DCB8F83B
:10BFD0000EC0BC45B9BFB4F802C0B0F80290B0F8CA
:10BFE00004C0B4F80090634503DB9945CC46A8BF74
:10BFF0009C4622F802CC7FE7B945B4BF638823880A
:10C0000022F8023C78E7049EB0F8029016B1B0F82E
:10C0100004C0E8E7B0F800C0634503DB9945CC46AF
:10C02000A8BF9C4622F802CCB8F810309F42BFF659
:10C0300063AFBEF1000F01D08388E1E7039B1B785B
:10C04000002B7FF459AF0388DAE70123204A214906
:10C05000136000220A6020490A60204A13804B22A4
:10C060001F4B1B685A7105221E4B1A8056E701238D
:10C07000237300231C4A05F5C335A0355370A56012
:10C08000FDF7A8BE01205FFA80F808F1FF3385F8BC
:10C09000EC34FCF781F8FCF723F94046FBF7DCFBB6
:10C0A000FEF70CB90220EEE7562B01D1FCF794FA0B
:10C0B00098F80030DFF83480002B3EF47AAB98F823
:10C0C000FE306F2B7EF46FABF7F7FCF8FEF7F6B897
:10C0D00030000020CC0D0020C80D00208A0D00206B
:10C0E000BC0D0020B60D002000000020A80000209C
:10C0F00030B5C0F3C751A1F17F021E2A83B020DC06
:10C10000531C1BDB162A4FEAD07409DDC0F316005E
:10C1100040F400009639884004B1404203B030BD7D
:10C120000F4B53F824502946FCF750FF019001981B
:10C130002946FCF749FF30F0004306D1002003B048
:10C1400030BDFDF727FA03B030BDC0F31603C0F3CE
:10C15000C75243F40000C2F19603D840DCE700BFA9
:10C16000A8DB0008F0B58BB0044600F01DFA224EA3
:10C17000054696F9003001332FD021462046FDF7C1
:10C18000F3F9074648BB204601F076F94FF07E519F
:10C19000FDF7E0F908B30122184B20468DE80C00AA
:10C1A0000897FCF7CFFB02460B461548CDE9042360
:10C1B000CDE9022300F0B6FF96F90030CDE9060183
:10C1C000022B0DD0684600F0ABFF48B1089B73B955
:10C1D000DDE90601FCF7A4FE054628460BB0F0BDDC
:10C1E00001F0B8F921230360089B002BF0D001F087
:10C1F000B1F9089B0360EBE740000020B0DB0008CA
:10C20000BCDB000800F034BB2DE9F0478AB00546DE
:10C210000C4600F0BFFBDFF8EC82064698F9007090
:10C220007B1C31D021462046FDF79EF9824658BB43
:10C2300029462846FDF798F900218146002840F05C
:10C2400099802846FDF75EF910B300212046FDF7DE
:10C2500059F98246002854D00122A44B28468DE883
:10C260000C00CDF82090FCF76DFBCDE902012046D3
:10C27000FCF768FB00220023CDE90401CDE9062389
:10C28000002F62D04FF07E5630460AB0BDE8F087EE
:10C29000304601F0F5F80746002800F087800021BD
:10C2A0003046FDF72FF90028EED0284601F0E8F8D7
:10C2B0000028E9D0204601F0E3F80028E4D000226D
:10C2C00004218A4B2846019308920091FCF73AFB1F
:10C2D000CDE902012046FCF735FB0024002598F942
:10C2E0000030CDE90401022BCDE9064504D06846B3
:10C2F00000F016FF00282ED101F02CF92223036054
:10C3000029E0204601F0BCF80028BDD000212046DD
:10C31000FDF702F90028B7D00122744B28468DE8BA
:10C320000C00CDF820A0FCF70DFBCDE90201204662
:10C33000FCF708FB98F90030CDE90401002B40F030
:10C34000938000220023CDE90623684600F0E8FE32
:10C35000002800F08480089B1BB101F0FBF8089BCB
:10C360000360DDE90601FCF7DBFD064630460AB056
:10C37000BDE8F0872046FDF7C5F8002884D00122EB
:10C380005A4B28468DE80C00CDF820A0FCF7DAFACD
:10C39000CDE902012046FCF7D5FA0022544B022FCA
:10C3A000CDE90401CDE90623CFD16BE7284601F0A2
:10C3B00067F800283FF473AF204601F061F80028C9
:10C3C0003FF46DAF31463046FDF7CEF80346002806
:10C3D00074D10321454A284608938DE80600FCF7EE
:10C3E000B1FACDE902012046FCF7ACFA98F90060F9
:10C3F000CDE90401002E3ED14FF060423D4B28466E
:10C400000021CDE90623FDF787F800283FF46FAF40
:10C4100020464FF07C51FCF7E1FEFCF793FA04460E
:10C420000D4600F085FE02460B4620462946FCF7E5
:10C4300045FD00283FD14FF060422F4B98F9006036
:10C44000CDE90623022E7FF452AF55E71046194678
:10C45000FCF7F6FB022CCDE906017FF476AF01F084
:10C4600079F82123036076E700202449022BCDE9E7
:10C470000601F4D069E70022214B28460021CDE9CE
:10C480000623FDF749F80028DCD020464FF07C5108
:10C49000FCF7A4FEFCF756FA04460D4600F048FEF1
:10C4A00002460B4620462946FCF708FD18B9002233
:10C4B000124BCDE9062398F90060C3E701220B4B2C
:10C4C00028468DE80C000897FCF73CFACDE90201FC
:10C4D0002046FCF737FA98F90040CDE90401002224
:10C4E0000023002CB2D1CDE906232EE7B8DB0008EB
:10C4F0000000F03FFFFFEF47FFFFEFC70000F0FF36
:10C500000000F07F40000020F0B58BB0044600F042
:10C51000B3FD234B064693F900506B1C0AD021460D
:10C520002046FDF721F8074620B900212046FCF7F8
:10C53000F3FF10B930460BB0F0BD0122194B204675
:10C540008DE80C000897FCF7FDF90022CDE9040105
:10C55000CDE902010023ADB110461946FCF770FB8E
:10C56000022DCDE906010FD100F0F4FF2123036075
:10C57000089B7BB9DDE90601FCF7D2FC0646304694
:10C580000BB0F0BDCDE90623684600F0C9FD0028D8
:10C59000EED1E9E700F0DEFF089B0360EAE700BFA9
:10C5A00040000020C0DB0008F8B520F00043B3F1E4
:10C5B0007E5F11D0044608DCB3F17C5F11DAB3F181
:10C5C0000C5F00F383809B48F8BD0146FCF7FCFC40
:10C5D0000146FCF7B7FEF8BD002840F3CB800020F1
:10C5E000F8BD0028C0F2C88001464FF07E50FCF72D
:10C5F000EBFC4FF07C51FCF7F1FD044600F03CFDF4
:10C600008D4906462046FCF7E9FD8C49FCF7DEFC27
:10C610002146FCF7E3FD8A49FCF7D6FC2146FCF7EE
:10C62000DDFD8849FCF7D2FC2146FCF7D7FD8649A1
:10C63000FCF7CAFC2146FCF7D1FD8449FCF7C6FC97
:10C640002146FCF7CBFD824905462046FCF7C6FD96
:10C650008049FCF7B9FC2146FCF7C0FD7E49FCF798
:10C66000B5FC2146FCF7BAFD7C49FCF7ADFC214640
:10C67000FCF7B4FD4FF07E51FCF7A8FC01462846BC
:10C68000FCF760FE3146FCF7A9FD26F47F6525F036
:10C690000F05074629462846FCF7A0FD014620461F
:10C6A000FCF792FC314604462846FCF78FFC014615
:10C6B0002046FCF747FE01463846FCF787FC294632
:10C6C000FCF784FC0146FCF781FCF8BD0146FCF751
:10C6D00085FD05465849FCF781FD5849FCF776FC75
:10C6E0002946FCF77BFD5649FCF76EFC2946FCF712
:10C6F00075FD5449FCF76AFC2946FCF76FFD524969
:10C70000FCF762FC2946FCF769FD5049FCF75EFC2A
:10C710002946FCF763FD4E4906462846FCF75EFDB8
:10C720004C49FCF751FC2946FCF758FD4A49FCF7F7
:10C730004DFC2946FCF752FD4849FCF745FC2946CB
:10C74000FCF74CFD4FF07E51FCF740FC01463046B3
:10C75000FCF7F8FD2146FCF741FD01464048FCF797
:10C7600033FC01462046FCF72FFC01463D48FCF710
:10C770002BFCF8BD3C48F8BD4FF07E51FCF726FC81
:10C780004FF07C51FCF72AFD04462B49FCF726FDAF
:10C790002A49FCF71BFC2146FCF720FD2849FCF741
:10C7A00013FC2146FCF71AFD2649FCF70FFC214635
:10C7B000FCF714FD2449FCF707FC2146FCF70EFDAD
:10C7C0002249FCF703FC2146FCF708FD06462046FB
:10C7D00000F052FC1E4905462046FCF7FFFC1D49AF
:10C7E000FCF7F2FB2146FCF7F9FC1B49FCF7EEFBDA
:10C7F0002146FCF7F3FC1949FCF7E6FB2146FCF760
:10C80000EDFC4FF07E51FCF7E1FB01463046FCF7B2
:10C8100099FD2946FCF7E2FC1149FCF7D5FB2946B6
:10C82000FCF7D4FB0146FCF7D1FB01460F48FCF7AF
:10C83000CBFBF8BDDB0FC93F08EF1138047F4F3A3F
:10C840004611243DA80A4E3E90B0A63EABAA2A3E11
:10C850002EC69D3D6133303F2D57014039D11940DF
:10C860006821A233DA0FC93FDB0F4940DA0F494094
:10C87000F8B50C4621F00041B1F1FF4F034614DC3E
:10C8800020F00046B6F1FF4F07460EDCB4F17E5FA4
:10C890003DD0A51705F0020545EAD07556B9022D21
:10C8A00030D0032D30D13248F8BD19462046FCF770
:10C8B0008DFBF8BD01B3B1F1FF4F2CD0B6F1FF4FA6
:10C8C0001AD0711AC9153C291ADC002C39DB214613
:10C8D0001846FCF737FD00F0CFFD00F0B7FC012D46
:10C8E0002CD0022D22D0002D2FD02249FCF76EFB38
:10C8F0002149FCF769FBF8BD002F06DB1F48F8BD96
:10C900001E48ECE71C48F8BDF8BD1D48F8BDBDE861
:10C91000F84000F09BBCB6F1FF4F17D0022DF1D0CC
:10C92000032DC0D0012D19D00020F8BD1149FCF70E
:10C930004DFB01461048FCF747FBF8BD00F10040F5
:10C94000F8BD3C31C3DA0020C9E7F8BD022D0CD098
:10C95000032D08D0012D04D00A48F8BD4FF0004047
:10C96000F8BD0948F8BD0948F8BD0948F8BD00BF41
:10C97000DB0F49C02EBDBB33DB0F4940DB0FC93F86
:10C98000DB0FC9BFDB0F493FDB0F49BFE4CB16C04C
:10C99000E4CB16402DE9F04F31F0004987B011D0BB
:10C9A00020F0004ABAF1FF4F054605DD4F4807B0B9
:10C9B000BDE8F04F00F06CBDB9F1FF4F07DDBAF1F3
:10C9C0007E5FF3D14FF07E5007B0BDE8F08F0028B6
:10C9D0000C4647DB0026B9F1FF4F3BD0B9F17E5F33
:10C9E00080460F4651D0B4F1804F67D0B4F17C5FE0
:10C9F0001BD000F041FDBAF1FF4F4ED0BAF1000F4D
:10CA00004BD0BAF17E5F48D0ED0F013D56EA0503E9
:10CA100064D0B9F19A4F6DDD354B9A4500F35B82D6
:10CA2000002CC0F25E820020CEE7002D4ADA00F032
:10CA300023FDBAF1FF4F02D0BAF1000FE1D1AAF104
:10CA40007E5A5AEA060342D0012EBDD100F10041C0
:10CA50000846B9E7BAF17E5FB4D02ADD002CE2DBEC
:10CA60000846B1E7B9F1974F21DAB9F17E5F0ADBE9
:10CA70004FEAE953C3F1960349FA03F202FA03F3CA
:10CA8000994500F023820026A8E7002C9CDA014695
:10CA90004FF07E50FCF756FC96E7002C04DA014676
:10CAA0004FF07E50FCF74EFC002D8DDAC7E70226D2
:10CAB00091E7002CB7DA01F1004085E70146FCF769
:10CAC0008DFB81E707B0BDE8F04F00F0D5BA014615
:10CAD000FCF77AFA0146FCF735FC75E7414640461B
:10CAE000FCF772FA0146FCF72DFC6DE7BCDB000891
:10CAF000F7FF7F3FBAF5000F80F2FF814FF09741BB
:10CB0000FCF76CFB6FF0170182464FEAEA53B34A19
:10CB1000CAF3160A7F3B0B449245194602934AF02A
:10CB20007E5840F3E381AE4B9A4540F33A820023AE
:10CB30001A4601930B4603924FF07E5B00220133AD
:10CB40000293A8F50008594640460092FCF73CFACB
:10CB5000594682464046FCF739FA01464FF07E506E
:10CB6000FCF7F0FB014605905046FCF737FB4FEA17
:10CB70006801009A41F00051C14601F5802120F47E
:10CB80007F6828F00F080A4411460090404604923E
:10CB9000FCF724FB01465046FCF716FA049A82463D
:10CBA00059461046FCF710FA01464846FCF70CFAC5
:10CBB0004146FCF713FB01465046FCF705FA059B7E
:10CBC0001946FCF70BFB009B834619461846FCF7F9
:10CBD00005FB81468349FCF701FB8349FCF7F6F925
:10CBE0004946FCF7FBFA8149FCF7F0F94946FCF7A6
:10CBF000F5FA7F49FCF7EAF94946FCF7EFFA7D4977
:10CC0000FCF7E4F94946FCF7E9FA7B49FCF7DEF961
:10CC1000494682464846FCF7E1FA01465046FCF791
:10CC2000DDFA814600994046FCF7D0F95946FCF7F9
:10CC3000D5FA4946FCF7CAF9414682464046FCF718
:10CC4000CDFA6E490490FCF7C1F95146FCF7BEF9E4
:10CC500020F47F6929F00F0949464046FCF7BEFAE7
:10CC6000664980464846FCF7AFF9049B1946FCF735
:10CC7000ABF901465046FCF7A7F90099FCF7AEFA6C
:10CC8000594682464846FCF7A9FA01465046FCF749
:10CC90009DF9834601464046FCF798F920F47F6AE7
:10CCA0002AF00F0A50465649FCF798FA4146814649
:10CCB0005046FCF789F901465846FCF785F9514979
:10CCC000FCF78CFA504980465046FCF787FA01463B
:10CCD0004046FCF77BF90399FCF778F98046029807
:10CCE000FCF728FA824641464846FCF76FF901995D
:10CCF000FCF76CF95146FCF769F920F47F6B2BF0D7
:10CD00000F0B51465846FCF75FF90199FCF75CF9A7
:10CD10004946FCF759F901464046FCF755F924F419
:10CD20007F64013E24F00F0456EA05038046214645
:10CD3000384614BF4FF07E56344EFCF745F959463D
:10CD4000FCF74CFA394605464046FCF747FA0146DF
:10CD50002846FCF73BF9214607465846FCF73EFAC1
:10CD6000804638464146FCF731F9002881460446A2
:10CD7000C24620F0004540F3FE80B5F1864F00F337
:10CD8000CC8000F0BC80B5F17C5F00F3CE80002544
:10CD9000A94624F47F6424F00F0420461C49FCF7C4
:10CDA0001DFA514680462046FCF70EF901463846EA
:10CDB000FCF70AF91749FCF711FA1749074620460C
:10CDC000FCF70CFA01463846FCF700F90746014625
:10CDD0004046FCF7FBF8414604461FE071C41C00C6
:10CDE000D6B35D0042F1533E55326C3E05A38B3EF7
:10CDF000ABAAAA3EB76DDB3E9A99193F00004040AE
:10CE00000038763F4F38763FA0C39D36000080BF84
:10CE10000072313F1872313F8CBEBF35FCF7D4F839
:10CE200001463846FCF7D0F8214680462046FCF7FC
:10CE3000D5F907467F49FCF7D1F97F49FCF7C4F8DB
:10CE40003946FCF7CBF97D49FCF7C0F83946FCF7C9
:10CE5000C5F97B49FCF7B8F83946FCF7BFF97949C1
:10CE6000FCF7B4F83946FCF7B9F901462046FCF75F
:10CE7000ABF8074601462046FCF7B0F94FF0804179
:10CE800082463846FCF7A0F801465046FCF75AFAAD
:10CE9000414607462046FCF7A1F94146FCF796F8C3
:10CEA00001463846FCF790F82146FCF78DF801461C
:10CEB0004FF07E50FCF788F84319B3F5000FC0F22D
:10CEC000B48018463146FCF789F97DE502F001028D
:10CED000C2F1020682E55C4B9A456BDD002C7FF7C0
:10CEE000A2AD5A490846FCF779F96DE50023002206
:10CEF000019303934FF07E5B25E6002105E654493C
:10CF00003846FCF763F8414682464846FCF75CF831
:10CF100001465046FCF71EFB38B130464B49FCF742
:10CF20005DF94A49FCF75AF94EE54FF40003ED1557
:10CF30007E3D43FA05F52B19C3F3C7524549C3F3A8
:10CF400016097F3A114149F40009C2F1170249FA62
:10CF500002F9002C23EA01014046B8BFC9F10009DB
:10CF6000FCF732F8014682463846FCF72FF84FEAC4
:10CF7000C95504460DE7384B9D420ADC7FF403AFE8
:10CF80004146FCF721F801463846FCF7CFFA002865
:10CF9000CBD030463149FCF721F93049FCF71EF976
:10CFA00012E52F4B4FF4001201932E4B4FF07F5B95
:10CFB0000393C8E54FF07E51FCF706F82A498046F6
:10CFC000FCF70CF9294981464046FCF707F94FF078
:10CFD0007A5182464046FCF701F901462448FBF7A6
:10CFE000F3FF4146FCF7FAF801464FF07C50FBF79F
:10CFF000EBFF414683464046FCF7F0F801465846B1
:10D00000FCF7ECF81B49FCF7E9F801465046FBF742
:10D01000DBFF014680464846FBF7D8FF20F47F6BD4
:10D020002BF00F0B4946584673E6494600F034FA98
:10D0300048E700BF4CBB31330EEADD3555B38A38C3
:10D04000610B363BABAA2A3E0700803FCAF249710A
:10D050003CAA3833FFFF7F00000016436042A20D58
:10D0600000C0153FDCCFD13500AAB83F70A5EC3623
:10D07000ABAAAA3E3BAAB83F20F00042B2F1FF4F54
:10D08000F8B504462FD26AB3002803463EDBB2F55A
:10D09000000F4FEAE0502DD300267F38C2074FF033
:10D0A000190431464FF08072C3F3160343F40003B2
:10D0B00048BF5B0047105B008D189D4202DC5B1B84
:10D0C000A9181644013C4FEA43034FEA5202F3D138
:10D0D00013B1013626F00106701000F17C5000EB10
:10D0E000C750F8BDF8BD0146FCF778F82146FBF7BC
:10D0F0006DFFF8BD14F4000201D00EE00A465B009B
:10D100001C0202F10101F9D5801AC5E70146FBF7BF
:10D110005BFF0146FCF716F9F8BD4FF0FF32F3E76D
:10D120000020704700200149704700BF0000F87FD1
:10D13000F0B5C1F30A5EAEF2FF36132E83B002469D
:10D140000B460C464FEAD17507462DDC002E48DB16
:10D150003C49314103EA010010432AD049080B4001
:10D1600053EA02070BD04FF48023132E0CBF4FF06D
:10D170000047002724EA010143FA06F40C43324B2E
:10D18000214603EBC505D5E90045384622462B4626
:10D19000FBF77AFACDE90001DDE9000122462B46D2
:10D1A000FBF770FA03B0F0BD332E06DDB6F5806FE5
:10D1B00044D01046194603B0F0BD4FF0FF31AEF237
:10D1C000134E21FA0EF10842F3D049080842D6D096
:10D1D0004FF0804320EA010143FA0EFE4EEA0107B8
:10D1E000CDE721F0004101431946E4D0C3F3130316
:10D1F00043EA000CCCF1000343EA0C03640C1B0B64
:10D2000003F40023640443EA04010F4B03EBC5035A
:10D21000D3E9006732463B46FBF736FACDE9000119
:10D22000DDE9000132463B46FBF72CFA024621F0CD
:10D23000004141EAC57310461946BCE7FBF724FAE2
:10D24000B9E700BFFFFF0F00C8DB00082DE9F04180
:10D2500020F00045B5F1A14F0446064608DBB5F1C4
:10D26000FF4F6FDC002840F3A0806F48BDE8F081DD
:10D270006E4B9D4277DCB5F1445F68DB4FF0FF37C2
:10D2800021462046FBF7AAFF01468046FBF7A6FF92
:10D2900005466749FBF7A2FF6649FBF797FE29465B
:10D2A000FBF79CFF6449FBF791FE2946FBF796FFCD
:10D2B0006249FBF78BFE2946FBF790FF6049FBF7BD
:10D2C00085FE2946FBF78AFF5E49FBF77FFE414654
:10D2D000FBF784FF5C4980462846FBF77FFF5B49EC
:10D2E000FBF772FE2946FBF779FF5949FBF76CFE05
:10D2F0002946FBF773FF5749FBF766FE2946FBF704
:10D300006DFF5549FBF760FE2946FBF767FF7B1C65
:10D31000014640464CD0FBF759FE2146FBF75EFF25
:10D320004E4B4F4D53F82710FBF74EFE2146FBF7AF
:10D330004BFE014655F82700FBF746FE002E30DB7A
:10D34000BDE8F0810146FBF741FEBDE8F0814549AB
:10D35000FBF73CFE4FF07E51FCF7FCF800288DD027
:10D360002046BDE8F08100F087F83F4B04469D421F
:10D3700029DCA3F5D0039D4244DC0146FBF726FEE1
:10D380004FF07E51FBF720FE4FF0804105462046CE
:10D39000FBF71CFE01462846FBF7D4FF0027044696
:10D3A0006EE700F10040BDE8F0813048BDE8F08153
:10D3B000FBF70CFE2146FBF711FF01462046FBF769
:10D3C00003FEBDE8F0812A4B9D4214DC4FF07F51F3
:10D3D000FBF7FAFD4FF07F5105462046FBF7FEFEB6
:10D3E0004FF07E51FBF7F2FD01462846FBF7AAFFFE
:10D3F0000227044644E701461E48FBF7A3FF032724
:10D4000004463DE74FF07E51FBF7DEFD4FF07E51C5
:10D4100005462046FBF7DAFD01462846FBF792FF5A
:10D42000012704462CE700BFDB0FC93FFFFFDF3EAB
:10D43000D769853C59DA4B3D356B883D6E2EBA3D38
:10D440002549123EABAAAA3E21A215BD6BF16E3D45
:10D4500095879D3D388EE33DCDCC4C3EE8DB000802
:10D46000D8DB0008CAF24971FFFF973FDB0FC9BF45
:10D47000FFFF1B40000080BF20F00040704700BF4E
:10D4800020F00040B0F1FF4FACBF002001207047FA
:10D49000004870470000C07F30F0004238B50346B6
:10D4A00016D0B2F1FF4F0FD2B2F5000F0D4610D3D8
:10D4B0000446D00D2844FE282EDC00281DDD24F073
:10D4C000FF4444EAC05038BD0146FBF77FFD38BD3C
:10D4D00038BD4FF09841FBF781FE184A034695424C
:10D4E00007DB0446C0F3C7501938E3E7144800F0DF
:10D4F0002BF81349FBF772FE38BD10F1160F13DA43
:10D500004CF2503295421946F0DD0E4800F01CF8FE
:10D510000C49FBF763FE38BD19460A4800F014F8C1
:10D520000849FBF75BFE38BD24F0FF44193044EA9C
:10D53000C0504FF04C51FBF751FE38BDB03CFFFFDF
:10D540006042A20DCAF2497101F0004120F0004092
:10D5500008437047014B1868704700BF4400002023
:10D5600010B5431E0A44914200D110BD11F8014B81
:10D5700003F8014FF7E703460244934200D1704796
:10D5800003F8011BF9E7C9B2034610F8012B1AB1E1
:10D590009142F9D11846704700290CBF1846002067
:10D5A00070470100010200010300010400010500B1
:10D5B000010600010700010800010900010A00013D
:10D5C0000B00010C01030D00010E00010F00011002
:10D5D00000011100011200011300011400010000FC
:10D5E0000000000000000000010203040607080913
:10D5F0000010014000401002001001400020100205
:10D600000010014000801002000C014020001002B8
:10D61000000C014010001002000801401000100230
:10D6200000080140200010020008014040001002E4
:10D63000B4D70008A4D70008A2D70008A0D70008D4
:10D6400000000040000801400100001C002800000C
:10D6500000000040000801400200041C00280000F7
:10D6600000000040000801400400081C00280000E1
:10D67000000000400008014008000C1C00280000C9
:10D6800000040040000801404000001D0028000088
:10D6900000040040000801408000041D0028000034
:10D6A00000040040000C01400100081D002800009B
:10D6B00000040040000C014002000C1D0028000086
:10D6C000002C0140000801400001001B012800005F
:10D6D000002C01400008014000080C1B012800003C
:10D6E00000080040000C01404000001E002800001F
:10D6F00000080040000C01408000041E00280000CB
:10D7000000080040000C01400001081E0028000035
:10D7100000080040000C014000020C1E0028000020
:10D720000000803F000000BFD0B35D3F0000803F9D
:10D730000000803F000000BFD0B35DBF0000803F0D
:10D740000000803F0000003FD0B35D3F000080BF7D
:10D750000000803F0000003FD0B35DBF000080BFED
:10D760000000803F000080BF00000000000080BF7C
:10D770000000803F0000803F000000000000803F6C
:10D780000000000080250000004B00000096000013
:10D7900000E1000000C201000084030090D00300FB
:10D7A000FFFFFFFF00010D030903010307030C0343
:10D7B0000603FFFF00020202030208020D03090331
:10D7C000010307030C030603FFFF000000540040A1
:10D7D000000C0140400080001F20000000002000DD
:10D7E00000580040000C0140000400082122000005
:10D7F00000004000524F4C4C3B50495443483B5969
:10D8000041573B414C543B506F733B506F73523BFD
:10D810004E6176523B4C4556454C3B4D41473B563D
:10D82000454C3B0000000000010203040102030418
:10D83000060708090204060800010000AB4E0008B4
:10D84000DF4C0008B74C0008714C00080D4E000872
:10D85000A14C0008094E000800000000BADA0008D8
:10D860000000000001000000BFDA00080100000015
:10D8700002000000C6DA00080200000003000000F9
:10D88000CFDA00080300000004000000D5DA000829
:10D890000500000005000000DADA000806000000BC
:10D8A00006000000E4DA000807000000070000009E
:10D8B000EDDA00080800000008000000F6DA0008B1
:10D8C0000900000009000000FFDA00080A0000005B
:10D8D0000A00000009DB00080B0000000B0000003C
:10D8E00013DB00080C0000000C0000001DDB00082A
:10D8F0000D0000000D00000025DB00080E000000F8
:10D900000E0000002DDB00080F0000000F000000DB
:10D9100035DB000810000000100000003EDB0008AE
:10D92000110000001100000045DB0008120000009B
:10D93000120000004FDB000813000000130000007D
:10D9400057DB0008140000001400000062DB000830
:10D95000150000001500000069DB0008160000003B
:10D960001600000070DB0008170000001700000020
:10D9700078DB0008180000001800000080DB0008B9
:10D98000190000001900000088DB00081A000000E0
:10D990001A00000092DB00081B0000001B000000C2
:10D9A00000000000FF000000414552543132333482
:10D9B0003536373861626364656667680000000069
:10D9C0000100000094DA00080201000081DA00087A
:10D9D000030200007EDA00080403000079DA000880
:10D9E0000504000074DA0008060500006BDA000880
:10D9F0000706000068DA00080807000065DA00087A
:10DA000009080000381800200A09000062DA00083E
:10DA10000C0A00005DDA00080D0B000058DA00085F
:10DA20000E0C000049DA00080F0D00003818002025
:10DA30000B0E000045DA0008100F000040DA000865
:10DA400000F50A05FF00640AFF0405040508050F38
:10DA500005080504050405FF140F2305FF0505054A
:10DA600005FF0A0AFF1932FF3202FF05050F0505FF
:10DA7000050F1EFF1E050505FF0F050F05FF3232BE
:10DA8000FF0A0A0A0A0A28280A280A28280A0A0A6B
:10DA90000A0A46FF140A140A140AFF434C464C00B3
:10DAA000434A4D31005365702031332032303137D5
:10DAB0000031313A30383A30380041524D3B004164
:10DAC0004E474C453B00484F52495A4F4E3B00424F
:10DAD00041524F3B004D41473B004845414446526F
:10DAE00045453B004845414441444A3B0043414D84
:10DAF000535441423B0043414D545249473B004738
:10DB0000505320484F4D453B0047505320484F4C01
:10DB1000443B0050415353544852553B0042454505
:10DB20005045523B004C45444D41583B004C454408
:10DB30004C4F573B004C4C49474854533B004341E2
:10DB40004C49423B00474F5645524E4F523B004FC7
:10DB500053442053573B0054454C454D455452596E
:10DB60003B004754554E453B00534F4E41523B00FE
:10DB7000534552564F313B00534552564F323B00AE
:10DB8000534552564F333B00424C41434B424F5852
:10DB90003B004641494C534146453B0041455452A8
:10DBA00031323334000000000000004B000000CB95
:10DBB00061636F7366000000706F7766000000009D
:10DBC00073717274660000000000000000003043B2
:10DBD00000000000000030C33863ED3EDA0F493F1B
:10DBE0005E987B3FDA0FC93F6937AC316821223339
:08DBF000B40F14336821A233C5
:08DBF8003CBBFF7F01000000AF
:10DC000001010000F40100000000803F000000005E
:10DC10000000000000A24A040000803F0000803F96
:10DC20000000803F0101000001000000BD6200080B
:10DC30000100000000127A000100000135260008F2
:10DC4000010000004800002000000000000000006B
:10DC500000000000000000000000000000000000C4
:10DC600000000000000000000000000000000000B4
:10DC700000000000000000000000000000000000A4
:10DC80000000000000000000000000000000000094
:10DC90000000000000000000000000000000000084
:08DCA00000000000000000007C
:0400000508000000EF
:00000001FF
